Component: ARM Compiler 5.05 update 1 (build 106) Tool: armlink [4d0efa]

==============================================================================

Section Cross References

    main.o(i.cdc_acm_user_ev_handler) refers to boards.o(i.bsp_board_led_off) for bsp_board_led_off
    main.o(i.cdc_acm_user_ev_handler) refers to boards.o(i.bsp_board_led_on) for bsp_board_led_on
    main.o(i.cdc_acm_user_ev_handler) refers to app_usbd_cdc_acm.o(i.app_usbd_cdc_acm_read) for app_usbd_cdc_acm_read
    main.o(i.cdc_acm_user_ev_handler) refers to app_error.o(i.app_error_handler_bare) for app_error_handler_bare
    main.o(i.cdc_acm_user_ev_handler) refers to boards.o(i.bsp_board_led_invert) for bsp_board_led_invert
    main.o(i.cdc_acm_user_ev_handler) refers to main.o(i.requestTx) for requestTx
    main.o(i.cdc_acm_user_ev_handler) refers to app_usbd_cdc_acm.o(i.app_usbd_cdc_acm_rx_size) for app_usbd_cdc_acm_rx_size
    main.o(i.cdc_acm_user_ev_handler) refers to nrf_assert.o(i.assert_nrf_callback) for assert_nrf_callback
    main.o(i.cdc_acm_user_ev_handler) refers to main.o(.data) for .data
    main.o(i.cdc_acm_user_ev_handler) refers to main.o(.bss) for .bss
    main.o(i.cdc_acm_user_ev_handler) refers to main.o(.constdata) for .constdata
    main.o(i.main) refers to nrf_drv_clock.o(i.nrf_drv_clock_init) for nrf_drv_clock_init
    main.o(i.main) refers to app_error.o(i.app_error_handler_bare) for app_error_handler_bare
    main.o(i.main) refers to nrf_drv_power.o(i.nrf_drv_power_init) for nrf_drv_power_init
    main.o(i.main) refers to nrf_log_frontend.o(i.nrf_log_init) for nrf_log_init
    main.o(i.main) refers to nrf_log_frontend.o(i.nrf_log_frontend_std_0) for nrf_log_frontend_std_0
    main.o(i.main) refers to boards.o(i.bsp_board_leds_init) for bsp_board_leds_init
    main.o(i.main) refers to boards.o(i.bsp_board_buttons_init) for bsp_board_buttons_init
    main.o(i.main) refers to printf8.o(i.__0snprintf$8) for __2snprintf
    main.o(i.main) refers to app_usbd.o(i.app_usbd_init) for app_usbd_init
    main.o(i.main) refers to app_usbd.o(i.app_usbd_class_append) for app_usbd_class_append
    main.o(i.main) refers to nrf_drv_power.o(i.nrf_drv_power_usbevt_init) for nrf_drv_power_usbevt_init
    main.o(i.main) refers to app_usbd.o(i.app_usbd_start) for app_usbd_start
    main.o(i.main) refers to app_usbd.o(i.app_usbd_disable) for app_usbd_disable
    main.o(i.main) refers to nrf_log_frontend.o(i.nrf_log_frontend_dequeue) for nrf_log_frontend_dequeue
    main.o(i.main) refers to boards.o(i.bsp_board_button_state_get) for bsp_board_button_state_get
    main.o(i.main) refers to main.o(i.requestTx) for requestTx
    main.o(i.main) refers to nrf_log_frontend.o(i.nrf_log_frontend_std_2) for nrf_log_frontend_std_2
    main.o(i.main) refers to main.o(i.nrf_delay_us) for nrf_delay_us
    main.o(i.main) refers to main.o(.bss) for .bss
    main.o(i.main) refers to main.o(.constdata) for .constdata
    main.o(i.main) refers to main.o(.data) for .data
    main.o(i.nrf_delay_us) refers to system_nrf52840.o(.data) for SystemCoreClock
    main.o(i.power_usb_event_handler) refers to nrf_assert.o(i.assert_nrf_callback) for assert_nrf_callback
    main.o(i.power_usb_event_handler) refers to nrf_log_frontend.o(i.nrf_log_frontend_std_0) for nrf_log_frontend_std_0
    main.o(i.power_usb_event_handler) refers to nrf_drv_usbd.o(i.nrf_drv_usbd_is_enabled) for nrf_drv_usbd_is_enabled
    main.o(i.power_usb_event_handler) refers to app_usbd.o(i.app_usbd_enable) for app_usbd_enable
    main.o(i.power_usb_event_handler) refers to main.o(.data) for .data
    main.o(i.requestTx) refers to printf8.o(i.__0sprintf$8) for __2sprintf
    main.o(i.requestTx) refers to strlen.o(.text) for strlen
    main.o(i.requestTx) refers to app_usbd_cdc_acm.o(i.app_usbd_cdc_acm_write) for app_usbd_cdc_acm_write
    main.o(i.requestTx) refers to nrf_assert.o(i.assert_nrf_callback) for assert_nrf_callback
    main.o(i.requestTx) refers to main.o(.data) for .data
    main.o(i.requestTx) refers to main.o(.bss) for .bss
    main.o(i.requestTx) refers to main.o(.constdata) for .constdata
    main.o(i.usbd_user_ev_handler) refers to boards.o(i.bsp_board_leds_off) for bsp_board_leds_off
    main.o(i.usbd_user_ev_handler) refers to boards.o(i.bsp_board_led_off) for bsp_board_led_off
    main.o(i.usbd_user_ev_handler) refers to boards.o(i.bsp_board_led_on) for bsp_board_led_on
    main.o(.constdata) refers to main.o(i.usbd_user_ev_handler) for usbd_user_ev_handler
    main.o(.constdata) refers to main.o(i.power_usb_event_handler) for power_usb_event_handler
    main.o(.constdata) refers to main.o(.bss) for m_app_cdc_acm_data
    main.o(.constdata) refers to app_usbd_cdc_acm.o(.constdata) for app_usbd_cdc_acm_class_methods
    main.o(.constdata) refers to main.o(.constdata) for m_cdc_acm_class_descriptors
    main.o(.constdata) refers to main.o(i.cdc_acm_user_ev_handler) for cdc_acm_user_ev_handler
    boards.o(i.bsp_board_button_idx_to_pin) refers to boards.o(.constdata) for .constdata
    boards.o(i.bsp_board_button_state_get) refers to boards.o(i.nrf_gpio_pin_port_decode) for nrf_gpio_pin_port_decode
    boards.o(i.bsp_board_button_state_get) refers to boards.o(.constdata) for .constdata
    boards.o(i.bsp_board_buttons_init) refers to boards.o(i.nrf_gpio_cfg) for nrf_gpio_cfg
    boards.o(i.bsp_board_buttons_init) refers to boards.o(.constdata) for .constdata
    boards.o(i.bsp_board_led_idx_to_pin) refers to boards.o(.constdata) for .constdata
    boards.o(i.bsp_board_led_invert) refers to boards.o(i.nrf_gpio_pin_port_decode) for nrf_gpio_pin_port_decode
    boards.o(i.bsp_board_led_invert) refers to boards.o(.constdata) for .constdata
    boards.o(i.bsp_board_led_off) refers to boards.o(i.nrf_gpio_pin_write) for nrf_gpio_pin_write
    boards.o(i.bsp_board_led_off) refers to boards.o(.constdata) for .constdata
    boards.o(i.bsp_board_led_on) refers to boards.o(i.nrf_gpio_pin_write) for nrf_gpio_pin_write
    boards.o(i.bsp_board_led_on) refers to boards.o(.constdata) for .constdata
    boards.o(i.bsp_board_led_state_get) refers to boards.o(i.nrf_gpio_pin_port_decode) for nrf_gpio_pin_port_decode
    boards.o(i.bsp_board_led_state_get) refers to boards.o(.constdata) for .constdata
    boards.o(i.bsp_board_leds_init) refers to boards.o(i.nrf_gpio_cfg) for nrf_gpio_cfg
    boards.o(i.bsp_board_leds_init) refers to boards.o(i.bsp_board_leds_off) for bsp_board_leds_off
    boards.o(i.bsp_board_leds_init) refers to boards.o(.constdata) for .constdata
    boards.o(i.bsp_board_leds_off) refers to boards.o(i.bsp_board_led_off) for bsp_board_led_off
    boards.o(i.bsp_board_leds_on) refers to boards.o(i.bsp_board_led_on) for bsp_board_led_on
    boards.o(i.bsp_board_pin_to_button_idx) refers to boards.o(.constdata) for .constdata
    boards.o(i.bsp_board_pin_to_led_idx) refers to boards.o(.constdata) for .constdata
    boards.o(i.nrf_gpio_cfg) refers to boards.o(i.nrf_gpio_pin_port_decode) for nrf_gpio_pin_port_decode
    boards.o(i.nrf_gpio_pin_write) refers to boards.o(i.nrf_gpio_pin_port_decode) for nrf_gpio_pin_port_decode
    bsp.o(i.alert_timer_handler) refers to boards.o(i.bsp_board_led_invert) for bsp_board_led_invert
    bsp.o(i.bsp_button_event_handler) refers to boards.o(i.bsp_board_pin_to_button_idx) for bsp_board_pin_to_button_idx
    bsp.o(i.bsp_button_event_handler) refers to app_timer.o(i.app_timer_start) for app_timer_start
    bsp.o(i.bsp_button_event_handler) refers to app_timer.o(i.app_timer_stop) for app_timer_stop
    bsp.o(i.bsp_button_event_handler) refers to bsp.o(.constdata) for .constdata
    bsp.o(i.bsp_button_event_handler) refers to bsp.o(.data) for .data
    bsp.o(i.bsp_button_event_handler) refers to bsp.o(.bss) for .bss
    bsp.o(i.bsp_button_is_pressed) refers to boards.o(i.bsp_board_button_state_get) for bsp_board_button_state_get
    bsp.o(i.bsp_buttons_disable) refers to app_button.o(i.app_button_disable) for app_button_disable
    bsp.o(i.bsp_buttons_enable) refers to app_button.o(i.app_button_enable) for app_button_enable
    bsp.o(i.bsp_event_to_button_action_assign) refers to bsp.o(.bss) for .bss
    bsp.o(i.bsp_indication_set) refers to bsp.o(i.bsp_led_indication) for bsp_led_indication
    bsp.o(i.bsp_indication_set) refers to bsp.o(.data) for .data
    bsp.o(i.bsp_init) refers to bsp.o(i.bsp_event_to_button_action_assign) for bsp_event_to_button_action_assign
    bsp.o(i.bsp_init) refers to app_button.o(i.app_button_init) for app_button_init
    bsp.o(i.bsp_init) refers to app_button.o(i.app_button_enable) for app_button_enable
    bsp.o(i.bsp_init) refers to app_timer.o(i.app_timer_create) for app_timer_create
    bsp.o(i.bsp_init) refers to boards.o(i.bsp_board_leds_init) for bsp_board_leds_init
    bsp.o(i.bsp_init) refers to bsp.o(.data) for .data
    bsp.o(i.bsp_init) refers to bsp.o(.constdata) for .constdata
    bsp.o(i.bsp_init) refers to bsp.o(i.button_timer_handler) for button_timer_handler
    bsp.o(i.bsp_init) refers to bsp.o(i.leds_timer_handler) for leds_timer_handler
    bsp.o(i.bsp_init) refers to bsp.o(i.alert_timer_handler) for alert_timer_handler
    bsp.o(i.bsp_led_indication) refers to bsp.o(i.leds_off) for leds_off
    bsp.o(i.bsp_led_indication) refers to boards.o(i.bsp_board_led_state_get) for bsp_board_led_state_get
    bsp.o(i.bsp_led_indication) refers to boards.o(i.bsp_board_led_off) for bsp_board_led_off
    bsp.o(i.bsp_led_indication) refers to boards.o(i.bsp_board_led_on) for bsp_board_led_on
    bsp.o(i.bsp_led_indication) refers to uldiv.o(.text) for __aeabi_uldivmod
    bsp.o(i.bsp_led_indication) refers to app_timer.o(i.app_timer_start) for app_timer_start
    bsp.o(i.bsp_led_indication) refers to boards.o(i.bsp_board_led_invert) for bsp_board_led_invert
    bsp.o(i.bsp_led_indication) refers to app_timer.o(i.app_timer_stop) for app_timer_stop
    bsp.o(i.bsp_led_indication) refers to boards.o(i.bsp_board_leds_on) for bsp_board_leds_on
    bsp.o(i.bsp_led_indication) refers to bsp.o(.data) for .data
    bsp.o(i.bsp_led_indication) refers to bsp.o(.constdata) for .constdata
    bsp.o(i.bsp_wakeup_button_disable) refers to boards.o(i.bsp_board_button_idx_to_pin) for bsp_board_button_idx_to_pin
    bsp.o(i.bsp_wakeup_button_disable) refers to bsp.o(i.nrf_gpio_cfg_sense_set) for nrf_gpio_cfg_sense_set
    bsp.o(i.bsp_wakeup_button_enable) refers to boards.o(i.bsp_board_button_idx_to_pin) for bsp_board_button_idx_to_pin
    bsp.o(i.bsp_wakeup_button_enable) refers to bsp.o(i.nrf_gpio_cfg_sense_set) for nrf_gpio_cfg_sense_set
    bsp.o(i.button_timer_handler) refers to bsp.o(i.bsp_button_event_handler) for bsp_button_event_handler
    bsp.o(i.leds_off) refers to boards.o(i.bsp_board_led_off) for bsp_board_led_off
    bsp.o(i.leds_off) refers to boards.o(i.bsp_board_leds_off) for bsp_board_leds_off
    bsp.o(i.leds_off) refers to bsp.o(.data) for .data
    bsp.o(i.leds_timer_handler) refers to bsp.o(i.bsp_led_indication) for bsp_led_indication
    bsp.o(i.leds_timer_handler) refers to bsp.o(.data) for .data
    bsp.o(.constdata) refers to bsp.o(.bss) for m_leds_timer_id_data
    bsp.o(.constdata) refers to bsp.o(.bss) for m_alert_timer_id_data
    bsp.o(.constdata) refers to bsp.o(.bss) for m_button_timer_id_data
    bsp.o(.constdata) refers to bsp.o(i.bsp_button_event_handler) for bsp_button_event_handler
    bsp_nfc.o(i.bsp_nfc_btn_deinit) refers to bsp.o(i.bsp_event_to_button_action_assign) for bsp_event_to_button_action_assign
    bsp_nfc.o(i.bsp_nfc_btn_init) refers to bsp.o(i.bsp_event_to_button_action_assign) for bsp_event_to_button_action_assign
    bsp_nfc.o(i.bsp_nfc_sleep_mode_prepare) refers to app_util_platform.o(i.app_util_critical_region_enter) for app_util_critical_region_enter
    bsp_nfc.o(i.bsp_nfc_sleep_mode_prepare) refers to app_util_platform.o(i.app_util_critical_region_exit) for app_util_critical_region_exit
    app_usbd.o(i.app_usbd_all_call) refers to app_usbd.o(i.class_event_handler) for class_event_handler
    app_usbd.o(i.app_usbd_all_call) refers to app_usbd.o(.data) for .data
    app_usbd.o(i.app_usbd_all_until_served_call) refers to app_usbd.o(i.class_event_handler) for class_event_handler
    app_usbd.o(i.app_usbd_all_until_served_call) refers to app_usbd.o(.data) for .data
    app_usbd.o(i.app_usbd_class_append) refers to app_usbd.o(i.app_usbd_ep_instance_get) for app_usbd_ep_instance_get
    app_usbd.o(i.app_usbd_class_append) refers to app_usbd.o(i.app_usbd_class_iface_ep_get) for app_usbd_class_iface_ep_get
    app_usbd.o(i.app_usbd_class_append) refers to app_usbd.o(i.app_usbd_class_iface_get) for app_usbd_class_iface_get
    app_usbd.o(i.app_usbd_class_append) refers to app_usbd.o(i.app_usbd_ep_instance_set) for app_usbd_ep_instance_set
    app_usbd.o(i.app_usbd_class_append) refers to app_usbd.o(.data) for .data
    app_usbd.o(i.app_usbd_class_append) refers to app_usbd.o(.constdata) for .constdata
    app_usbd.o(i.app_usbd_class_first_get) refers to app_usbd.o(.data) for .data
    app_usbd.o(i.app_usbd_class_remove) refers to app_usbd.o(i.class_event_handler) for class_event_handler
    app_usbd.o(i.app_usbd_class_remove) refers to app_usbd.o(i.app_usbd_ep_instance_get) for app_usbd_ep_instance_get
    app_usbd.o(i.app_usbd_class_remove) refers to app_usbd.o(i.app_usbd_ep_instance_set) for app_usbd_ep_instance_set
    app_usbd.o(i.app_usbd_class_remove) refers to app_usbd.o(.data) for .data
    app_usbd.o(i.app_usbd_class_remove) refers to app_usbd.o(.constdata) for .constdata
    app_usbd.o(i.app_usbd_class_remove_all) refers to app_usbd.o(i.app_usbd_class_remove) for app_usbd_class_remove
    app_usbd.o(i.app_usbd_class_remove_all) refers to app_usbd.o(.data) for .data
    app_usbd.o(i.app_usbd_class_sof_first_get) refers to app_usbd.o(.data) for .data
    app_usbd.o(i.app_usbd_class_sof_register) refers to app_usbd.o(.data) for .data
    app_usbd.o(i.app_usbd_class_sof_unregister) refers to app_usbd.o(.data) for .data
    app_usbd.o(i.app_usbd_core_handler_call) refers to app_usbd.o(.bss) for .bss
    app_usbd.o(i.app_usbd_disable) refers to nrf_drv_usbd.o(i.nrf_drv_usbd_is_started) for nrf_drv_usbd_is_started
    app_usbd.o(i.app_usbd_disable) refers to app_usbd.o(i.app_usbd_stop) for app_usbd_stop
    app_usbd.o(i.app_usbd_disable) refers to nrf_drv_usbd.o(i.nrf_drv_usbd_disable) for nrf_drv_usbd_disable
    app_usbd.o(i.app_usbd_enable) refers to nrf_drv_usbd.o(i.nrf_drv_usbd_enable) for nrf_drv_usbd_enable
    app_usbd.o(i.app_usbd_endpoint_std_req_handle) refers to app_usbd_core.o(i.app_usbd_core_setup_transfer_buff_get) for app_usbd_core_setup_transfer_buff_get
    app_usbd.o(i.app_usbd_endpoint_std_req_handle) refers to nrf_drv_usbd.o(i.nrf_drv_usbd_ep_stall_check) for nrf_drv_usbd_ep_stall_check
    app_usbd.o(i.app_usbd_endpoint_std_req_handle) refers to app_usbd_core.o(i.app_usbd_core_setup_rsp) for app_usbd_core_setup_rsp
    app_usbd.o(i.app_usbd_endpoint_std_req_handle) refers to nrf_drv_usbd.o(i.nrf_drv_usbd_ep_stall) for nrf_drv_usbd_ep_stall
    app_usbd.o(i.app_usbd_endpoint_std_req_handle) refers to app_usbd.o(i.nrf_usbd_dtoggle_get) for nrf_usbd_dtoggle_get
    app_usbd.o(i.app_usbd_endpoint_std_req_handle) refers to app_usbd.o(i.nrf_usbd_dtoggle_set) for nrf_usbd_dtoggle_set
    app_usbd.o(i.app_usbd_endpoint_std_req_handle) refers to nrf_drv_usbd.o(i.nrf_drv_usbd_ep_stall_clear) for nrf_drv_usbd_ep_stall_clear
    app_usbd.o(i.app_usbd_ep_call) refers to app_usbd.o(i.app_usbd_ep_conf_access) for app_usbd_ep_conf_access
    app_usbd.o(i.app_usbd_ep_conf_access) refers to app_usbd.o(.bss) for .bss
    app_usbd.o(i.app_usbd_ep_handler_set) refers to app_usbd.o(i.app_usbd_ep_instance_get) for app_usbd_ep_instance_get
    app_usbd.o(i.app_usbd_ep_handler_set) refers to app_usbd.o(i.app_usbd_ep_conf_access) for app_usbd_ep_conf_access
    app_usbd.o(i.app_usbd_ep_instance_get) refers to app_usbd.o(i.app_usbd_ep_conf_access) for app_usbd_ep_conf_access
    app_usbd.o(i.app_usbd_ep_instance_set) refers to app_usbd.o(i.app_usbd_ep_conf_access) for app_usbd_ep_conf_access
    app_usbd.o(i.app_usbd_event_handler) refers to app_usbd.o(i.class_event_handler) for class_event_handler
    app_usbd.o(i.app_usbd_event_handler) refers to app_usbd.o(i.app_usbd_core_handler_call) for app_usbd_core_handler_call
    app_usbd.o(i.app_usbd_event_handler) refers to app_usbd.o(i.app_usbd_all_call) for app_usbd_all_call
    app_usbd.o(i.app_usbd_event_handler) refers to app_usbd.o(i.app_usbd_ep_conf_access) for app_usbd_ep_conf_access
    app_usbd.o(i.app_usbd_event_handler) refers to nrf_drv_usbd.o(i.nrf_drv_usbd_ep_stall) for nrf_drv_usbd_ep_stall
    app_usbd.o(i.app_usbd_event_handler) refers to app_usbd.o(i.user_event_handler) for user_event_handler
    app_usbd.o(i.app_usbd_event_handler) refers to app_usbd.o(.data) for .data
    app_usbd.o(i.app_usbd_iface_call) refers to app_usbd.o(i.app_usbd_class_iface_get) for app_usbd_class_iface_get
    app_usbd.o(i.app_usbd_iface_call) refers to app_usbd.o(.data) for .data
    app_usbd.o(i.app_usbd_init) refers to nrf_drv_usbd.o(i.nrf_drv_usbd_init) for nrf_drv_usbd_init
    app_usbd.o(i.app_usbd_init) refers to memseta.o(.text) for __aeabi_memclr4
    app_usbd.o(i.app_usbd_init) refers to app_usbd.o(i.app_usbd_ep_instance_set) for app_usbd_ep_instance_set
    app_usbd.o(i.app_usbd_init) refers to app_usbd.o(i.app_usbd_class_iface_ep_get) for app_usbd_class_iface_ep_get
    app_usbd.o(i.app_usbd_init) refers to app_usbd.o(i.app_usbd_class_iface_get) for app_usbd_class_iface_get
    app_usbd.o(i.app_usbd_init) refers to app_usbd.o(i.app_usbd_event_handler) for app_usbd_event_handler
    app_usbd.o(i.app_usbd_init) refers to app_usbd.o(.constdata) for .constdata
    app_usbd.o(i.app_usbd_init) refers to app_usbd.o(.data) for .data
    app_usbd.o(i.app_usbd_init) refers to app_usbd.o(.bss) for .bss
    app_usbd.o(i.app_usbd_init) refers to app_usbd_core.o(.constdata) for app_usbd_core_inst
    app_usbd.o(i.app_usbd_interface_std_req_handle) refers to app_usbd_core.o(i.app_usbd_core_setup_transfer_buff_get) for app_usbd_core_setup_transfer_buff_get
    app_usbd.o(i.app_usbd_interface_std_req_handle) refers to app_usbd_core.o(i.app_usbd_core_setup_rsp) for app_usbd_core_setup_rsp
    app_usbd.o(i.app_usbd_req_std_set_interface) refers to app_usbd.o(i.app_usbd_class_iface_get) for app_usbd_class_iface_get
    app_usbd.o(i.app_usbd_req_std_set_interface) refers to app_usbd.o(i.app_usbd_class_iface_ep_get) for app_usbd_class_iface_ep_get
    app_usbd.o(i.app_usbd_req_std_set_interface) refers to app_usbd.o(i.nrf_usbd_dtoggle_get) for nrf_usbd_dtoggle_get
    app_usbd.o(i.app_usbd_req_std_set_interface) refers to app_usbd.o(i.nrf_usbd_dtoggle_set) for nrf_usbd_dtoggle_set
    app_usbd.o(i.app_usbd_req_std_set_interface) refers to nrf_drv_usbd.o(i.nrf_drv_usbd_ep_stall_clear) for nrf_drv_usbd_ep_stall_clear
    app_usbd.o(i.app_usbd_start) refers to nrf_drv_usbd.o(i.nrf_drv_usbd_ep_enable) for nrf_drv_usbd_ep_enable
    app_usbd.o(i.app_usbd_start) refers to app_usbd.o(i.app_usbd_core_handler_call) for app_usbd_core_handler_call
    app_usbd.o(i.app_usbd_start) refers to app_usbd.o(i.app_usbd_all_call) for app_usbd_all_call
    app_usbd.o(i.app_usbd_start) refers to app_usbd.o(i.user_event_handler) for user_event_handler
    app_usbd.o(i.app_usbd_start) refers to nrf_drv_usbd.o(i.nrf_drv_usbd_start) for nrf_drv_usbd_start
    app_usbd.o(i.app_usbd_start) refers to app_usbd.o(.constdata) for .constdata
    app_usbd.o(i.app_usbd_start) refers to app_usbd.o(.bss) for .bss
    app_usbd.o(i.app_usbd_start) refers to app_usbd.o(.data) for .data
    app_usbd.o(i.app_usbd_stop) refers to nrf_drv_usbd.o(i.nrf_drv_usbd_stop) for nrf_drv_usbd_stop
    app_usbd.o(i.app_usbd_stop) refers to app_usbd.o(i.app_usbd_all_call) for app_usbd_all_call
    app_usbd.o(i.app_usbd_stop) refers to app_usbd.o(i.app_usbd_core_handler_call) for app_usbd_core_handler_call
    app_usbd.o(i.app_usbd_stop) refers to app_usbd.o(i.user_event_handler) for user_event_handler
    app_usbd.o(i.app_usbd_stop) refers to app_usbd.o(.constdata) for .constdata
    app_usbd.o(i.app_usbd_uninit) refers to nrf_drv_usbd.o(i.nrf_drv_usbd_uninit) for nrf_drv_usbd_uninit
    app_usbd.o(i.app_usbd_uninit) refers to memseta.o(.text) for __aeabi_memclr4
    app_usbd.o(i.app_usbd_uninit) refers to app_usbd.o(.data) for .data
    app_usbd.o(i.app_usbd_uninit) refers to app_usbd.o(.bss) for .bss
    app_usbd.o(i.nrf_usbd_dtoggle_get) refers to app_usbd.o(i.nrf_usbd_dtoggle_set) for nrf_usbd_dtoggle_set
    app_usbd.o(i.user_event_handler) refers to app_usbd.o(.data) for .data
    app_usbd_core.o(i.app_usbd_core_class_rwu_pend) refers to app_usbd_core.o(.emb_text) for __asm___15_app_usbd_core_c_a97d2587__nrf_atomic_internal_orr
    app_usbd_core.o(i.app_usbd_core_class_rwu_pend) refers to app_usbd_core.o(i.nrf_usbd_task_trigger) for nrf_usbd_task_trigger
    app_usbd_core.o(i.app_usbd_core_class_rwu_pend) refers to app_usbd_core.o(.data) for .data
    app_usbd_core.o(i.app_usbd_core_class_rwu_register) refers to app_usbd_core.o(.data) for .data
    app_usbd_core.o(i.app_usbd_core_class_rwu_unregister) refers to app_usbd_core.o(.data) for .data
    app_usbd_core.o(i.app_usbd_core_ep_transfer) refers to nrf_drv_usbd.o(i.nrf_drv_usbd_ep_transfer) for nrf_drv_usbd_ep_transfer
    app_usbd_core.o(i.app_usbd_core_ep_transfer) refers to app_usbd_core.o(.data) for .data
    app_usbd_core.o(i.app_usbd_core_event_handler) refers to app_usbd_core.o(.emb_text) for __asm___15_app_usbd_core_c_a97d2587__nrf_atomic_internal_and
    app_usbd_core.o(i.app_usbd_core_event_handler) refers to app_usbd_core.o(i.nrf_usbd_task_trigger) for nrf_usbd_task_trigger
    app_usbd_core.o(i.app_usbd_core_event_handler) refers to app_usbd_core.o(i.app_usbd_core_setup_req_handler) for app_usbd_core_setup_req_handler
    app_usbd_core.o(i.app_usbd_core_event_handler) refers to nrf_drv_usbd.o(i.nrf_drv_usbd_setup_stall) for nrf_drv_usbd_setup_stall
    app_usbd_core.o(i.app_usbd_core_event_handler) refers to app_usbd_core.o(i.usb_core_ep0_handler_check) for usb_core_ep0_handler_check
    app_usbd_core.o(i.app_usbd_core_event_handler) refers to nrf_drv_usbd.o(i.nrf_drv_usbd_setup_data_clear) for nrf_drv_usbd_setup_data_clear
    app_usbd_core.o(i.app_usbd_core_event_handler) refers to nrf_drv_usbd.o(i.nrf_drv_usbd_setup_clear) for nrf_drv_usbd_setup_clear
    app_usbd_core.o(i.app_usbd_core_event_handler) refers to app_usbd_core.o(.data) for .data
    app_usbd_core.o(i.app_usbd_core_setup_data_handler_set) refers to nrf_drv_usbd.o(i.nrf_drv_usbd_last_setup_dir_get) for nrf_drv_usbd_last_setup_dir_get
    app_usbd_core.o(i.app_usbd_core_setup_data_handler_set) refers to app_usbd_core.o(.data) for .data
    app_usbd_core.o(i.app_usbd_core_setup_data_transfer) refers to nrf_drv_usbd.o(i.nrf_drv_usbd_ep_transfer) for nrf_drv_usbd_ep_transfer
    app_usbd_core.o(i.app_usbd_core_setup_data_transfer) refers to app_usbd_core.o(.data) for .data
    app_usbd_core.o(i.app_usbd_core_setup_req_handler) refers to nrf_drv_usbd.o(i.nrf_drv_usbd_setup_get) for nrf_drv_usbd_setup_get
    app_usbd_core.o(i.app_usbd_core_setup_req_handler) refers to app_usbd_core.o(i.setup_req_std_in) for setup_req_std_in
    app_usbd_core.o(i.app_usbd_core_setup_req_handler) refers to app_usbd_core.o(i.setup_req_std_out) for setup_req_std_out
    app_usbd_core.o(i.app_usbd_core_setup_req_handler) refers to app_usbd.o(i.app_usbd_all_until_served_call) for app_usbd_all_until_served_call
    app_usbd_core.o(i.app_usbd_core_setup_req_handler) refers to app_usbd.o(i.app_usbd_iface_call) for app_usbd_iface_call
    app_usbd_core.o(i.app_usbd_core_setup_req_handler) refers to app_usbd.o(i.app_usbd_interface_std_req_handle) for app_usbd_interface_std_req_handle
    app_usbd_core.o(i.app_usbd_core_setup_req_handler) refers to app_usbd.o(i.app_usbd_ep_call) for app_usbd_ep_call
    app_usbd_core.o(i.app_usbd_core_setup_req_handler) refers to app_usbd.o(i.app_usbd_endpoint_std_req_handle) for app_usbd_endpoint_std_req_handle
    app_usbd_core.o(i.app_usbd_core_setup_req_handler) refers to nrf_drv_usbd.o(i.nrf_drv_usbd_setup_stall) for nrf_drv_usbd_setup_stall
    app_usbd_core.o(i.app_usbd_core_setup_req_handler) refers to app_usbd_core.o(i.usb_core_ep0_handler_check) for usb_core_ep0_handler_check
    app_usbd_core.o(i.app_usbd_core_setup_req_handler) refers to nrf_drv_usbd.o(i.nrf_drv_usbd_setup_data_clear) for nrf_drv_usbd_setup_data_clear
    app_usbd_core.o(i.app_usbd_core_setup_req_handler) refers to nrf_drv_usbd.o(i.nrf_drv_usbd_setup_clear) for nrf_drv_usbd_setup_clear
    app_usbd_core.o(i.app_usbd_core_setup_rsp) refers to nrf_drv_usbd.o(i.nrf_drv_usbd_ep_max_packet_size_get) for nrf_drv_usbd_ep_max_packet_size_get
    app_usbd_core.o(i.app_usbd_core_setup_rsp) refers to app_util_platform.o(i.app_util_critical_region_enter) for app_util_critical_region_enter
    app_usbd_core.o(i.app_usbd_core_setup_rsp) refers to app_usbd_core.o(i.app_usbd_core_setup_data_transfer) for app_usbd_core_setup_data_transfer
    app_usbd_core.o(i.app_usbd_core_setup_rsp) refers to app_usbd_core.o(i.app_usbd_core_setup_data_handler_set) for app_usbd_core_setup_data_handler_set
    app_usbd_core.o(i.app_usbd_core_setup_rsp) refers to app_util_platform.o(i.app_util_critical_region_exit) for app_util_critical_region_exit
    app_usbd_core.o(i.app_usbd_core_setup_rsp) refers to app_usbd_core.o(.constdata) for .constdata
    app_usbd_core.o(i.app_usbd_core_setup_transfer_buff_get) refers to app_usbd_core.o(.bss) for .bss
    app_usbd_core.o(i.app_usbd_core_state_get) refers to app_usbd_core.o(.data) for .data
    app_usbd_core.o(i.app_usbd_ep_handled_transfer) refers to nrf_drv_usbd.o(i.nrf_drv_usbd_ep_handled_transfer) for nrf_drv_usbd_ep_handled_transfer
    app_usbd_core.o(i.app_usbd_ep_handled_transfer) refers to app_usbd_core.o(.data) for .data
    app_usbd_core.o(i.app_usbd_setup_data_handled_transfer) refers to nrf_drv_usbd.o(i.nrf_drv_usbd_ep_handled_transfer) for nrf_drv_usbd_ep_handled_transfer
    app_usbd_core.o(i.app_usbd_setup_data_handled_transfer) refers to app_usbd_core.o(.data) for .data
    app_usbd_core.o(i.setup_req_get_descriptor) refers to app_usbd.o(i.app_usbd_class_first_get) for app_usbd_class_first_get
    app_usbd_core.o(i.setup_req_get_descriptor) refers to app_usbd_core.o(i.app_usbd_core_setup_transfer_buff_get) for app_usbd_core_setup_transfer_buff_get
    app_usbd_core.o(i.setup_req_get_descriptor) refers to memcpya.o(.text) for __aeabi_memcpy
    app_usbd_core.o(i.setup_req_get_descriptor) refers to app_util_platform.o(i.app_util_critical_region_enter) for app_util_critical_region_enter
    app_usbd_core.o(i.setup_req_get_descriptor) refers to app_usbd_core.o(i.app_usbd_setup_data_handled_transfer) for app_usbd_setup_data_handled_transfer
    app_usbd_core.o(i.setup_req_get_descriptor) refers to app_usbd_core.o(i.app_usbd_core_setup_data_handler_set) for app_usbd_core_setup_data_handler_set
    app_usbd_core.o(i.setup_req_get_descriptor) refers to app_util_platform.o(i.app_util_critical_region_exit) for app_util_critical_region_exit
    app_usbd_core.o(i.setup_req_get_descriptor) refers to app_usbd_string_desc.o(i.app_usbd_string_desc_get) for app_usbd_string_desc_get
    app_usbd_core.o(i.setup_req_get_descriptor) refers to app_usbd_core.o(i.app_usbd_core_setup_rsp) for app_usbd_core_setup_rsp
    app_usbd_core.o(i.setup_req_get_descriptor) refers to app_usbd_core.o(.constdata) for .constdata
    app_usbd_core.o(i.setup_req_get_descriptor) refers to app_usbd_core.o(.data) for .data
    app_usbd_core.o(i.setup_req_get_descriptor) refers to app_usbd_core.o(.bss) for .bss
    app_usbd_core.o(i.setup_req_std_in) refers to app_usbd_core.o(i.app_usbd_core_setup_transfer_buff_get) for app_usbd_core_setup_transfer_buff_get
    app_usbd_core.o(i.setup_req_std_in) refers to app_usbd_core.o(i.setup_req_get_descriptor) for setup_req_get_descriptor
    app_usbd_core.o(i.setup_req_std_in) refers to app_usbd_core.o(i.app_usbd_core_setup_rsp) for app_usbd_core_setup_rsp
    app_usbd_core.o(i.setup_req_std_in) refers to app_usbd_core.o(.data) for .data
    app_usbd_core.o(i.setup_req_std_out) refers to app_usbd_core.o(i.setup_req_std_set_configuration) for setup_req_std_set_configuration
    app_usbd_core.o(i.setup_req_std_out) refers to app_usbd_core.o(.data) for .data
    app_usbd_core.o(i.setup_req_std_set_configuration) refers to app_usbd.o(i.app_usbd_class_first_get) for app_usbd_class_first_get
    app_usbd_core.o(i.setup_req_std_set_configuration) refers to app_usbd_core.o(i.nrf_usbd_dtoggle_set) for nrf_usbd_dtoggle_set
    app_usbd_core.o(i.setup_req_std_set_configuration) refers to nrf_drv_usbd.o(i.nrf_drv_usbd_ep_stall_clear) for nrf_drv_usbd_ep_stall_clear
    app_usbd_core.o(i.setup_req_std_set_configuration) refers to app_usbd_core.o(.data) for .data
    app_usbd_core.o(i.usb_core_ep0_handler_check) refers to app_usbd_core.o(.data) for .data
    app_usbd_core.o(i.usbd_descriptor_conf_feeder) refers to nrf_drv_usbd.o(i.nrf_drv_usbd_feeder_buffer_get) for nrf_drv_usbd_feeder_buffer_get
    app_usbd_core.o(i.usbd_descriptor_conf_feeder) refers to memcpya.o(.text) for __aeabi_memcpy
    app_usbd_core.o(.constdata) refers to app_usbd_core.o(i.setup_data_handler_empty) for setup_data_handler_empty
    app_usbd_core.o(.constdata) refers to app_usbd_core.o(i.usbd_descriptor_conf_feeder) for usbd_descriptor_conf_feeder
    app_usbd_core.o(.constdata) refers to app_usbd_core.o(.bss) for m_descriptor_conf_feed_data
    app_usbd_core.o(.constdata) refers to app_usbd_core.o(i.app_usbd_core_event_handler) for app_usbd_core_event_handler
    app_usbd_core.o(.constdata) refers to app_usbd_core.o(.data) for app_usbd_core_inst_data
    app_usbd_core.o(.constdata) refers to app_usbd_core.o(.constdata) for m_core_methods
    app_usbd_string_desc.o(i.app_usbd_string_desc_get) refers to app_usbd_string_desc.o(.data) for .data
    app_usbd_string_desc.o(i.app_usbd_string_desc_get) refers to app_usbd_string_desc.o(.constdata) for .constdata
    app_usbd_string_desc.o(.data) refers to app_usbd_string_desc.o(.constdata) for <Data2>
    app_usbd_string_desc.o(.data) refers to app_usbd_string_desc.o(.constdata) for <Data4>
    app_usbd_string_desc.o(.data) refers to app_usbd_string_desc.o(.constdata) for <Data6>
    app_usbd_string_desc.o(.data) refers to main.o(.bss) for g_extern_serial_number
    app_usbd_string_desc.o(.data) refers to app_usbd_string_desc.o(.constdata) for <Data8>
    nrf_drv_clock.o(i.clock_clk_started_notify) refers to nrf_drv_clock.o(.bss) for .bss
    nrf_drv_clock.o(i.hfclk_stop) refers to nrf_drv_clock.o(i.nrf_clock_hf_is_running) for nrf_clock_hf_is_running
    nrf_drv_clock.o(i.hfclk_stop) refers to nrf_drv_clock.o(.bss) for .bss
    nrf_drv_clock.o(i.lfclk_stop) refers to nrf_drv_clock.o(.bss) for .bss
    nrf_drv_clock.o(i.nrf_drv_clock_hfclk_is_running) refers to nrf_drv_clock.o(i.nrf_clock_hf_is_running) for nrf_clock_hf_is_running
    nrf_drv_clock.o(i.nrf_drv_clock_hfclk_release) refers to app_util_platform.o(i.app_util_critical_region_enter) for app_util_critical_region_enter
    nrf_drv_clock.o(i.nrf_drv_clock_hfclk_release) refers to nrf_drv_clock.o(i.hfclk_stop) for hfclk_stop
    nrf_drv_clock.o(i.nrf_drv_clock_hfclk_release) refers to app_util_platform.o(i.app_util_critical_region_exit) for app_util_critical_region_exit
    nrf_drv_clock.o(i.nrf_drv_clock_hfclk_release) refers to nrf_drv_clock.o(.bss) for .bss
    nrf_drv_clock.o(i.nrf_drv_clock_hfclk_request) refers to app_util_platform.o(i.app_util_critical_region_enter) for app_util_critical_region_enter
    nrf_drv_clock.o(i.nrf_drv_clock_hfclk_request) refers to nrf_drv_clock.o(i.item_enqueue) for item_enqueue
    nrf_drv_clock.o(i.nrf_drv_clock_hfclk_request) refers to nrf_drv_clock.o(i.nrf_clock_event_clear) for nrf_clock_event_clear
    nrf_drv_clock.o(i.nrf_drv_clock_hfclk_request) refers to app_util_platform.o(i.app_util_critical_region_exit) for app_util_critical_region_exit
    nrf_drv_clock.o(i.nrf_drv_clock_hfclk_request) refers to nrf_drv_clock.o(.bss) for .bss
    nrf_drv_clock.o(i.nrf_drv_clock_init) refers to nrf_drv_common.o(i.nrf_drv_common_irq_enable) for nrf_drv_common_irq_enable
    nrf_drv_clock.o(i.nrf_drv_clock_init) refers to nrf_drv_clock.o(.bss) for .bss
    nrf_drv_clock.o(i.nrf_drv_clock_init_check) refers to nrf_drv_clock.o(.bss) for .bss
    nrf_drv_clock.o(i.nrf_drv_clock_lfclk_release) refers to app_util_platform.o(i.app_util_critical_region_enter) for app_util_critical_region_enter
    nrf_drv_clock.o(i.nrf_drv_clock_lfclk_release) refers to nrf_drv_clock.o(i.lfclk_stop) for lfclk_stop
    nrf_drv_clock.o(i.nrf_drv_clock_lfclk_release) refers to app_util_platform.o(i.app_util_critical_region_exit) for app_util_critical_region_exit
    nrf_drv_clock.o(i.nrf_drv_clock_lfclk_release) refers to nrf_drv_clock.o(.bss) for .bss
    nrf_drv_clock.o(i.nrf_drv_clock_lfclk_request) refers to app_util_platform.o(i.app_util_critical_region_enter) for app_util_critical_region_enter
    nrf_drv_clock.o(i.nrf_drv_clock_lfclk_request) refers to nrf_drv_clock.o(i.item_enqueue) for item_enqueue
    nrf_drv_clock.o(i.nrf_drv_clock_lfclk_request) refers to nrf_drv_clock.o(i.nrf_clock_event_clear) for nrf_clock_event_clear
    nrf_drv_clock.o(i.nrf_drv_clock_lfclk_request) refers to app_util_platform.o(i.app_util_critical_region_exit) for app_util_critical_region_exit
    nrf_drv_clock.o(i.nrf_drv_clock_lfclk_request) refers to nrf_drv_clock.o(.bss) for .bss
    nrf_drv_clock.o(i.nrf_drv_clock_onIRQ) refers to nrf_drv_clock.o(i.nrf_clock_event_check) for nrf_clock_event_check
    nrf_drv_clock.o(i.nrf_drv_clock_onIRQ) refers to nrf_drv_clock.o(i.nrf_clock_event_clear) for nrf_clock_event_clear
    nrf_drv_clock.o(i.nrf_drv_clock_onIRQ) refers to nrf_drv_clock.o(i.clock_clk_started_notify) for clock_clk_started_notify
    nrf_drv_clock.o(i.nrf_drv_clock_onIRQ) refers to nrf_drv_clock.o(.bss) for .bss
    nrf_drv_clock.o(i.nrf_drv_clock_uninit) refers to nrf_drv_common.o(i.nrf_drv_common_clock_irq_disable) for nrf_drv_common_clock_irq_disable
    nrf_drv_clock.o(i.nrf_drv_clock_uninit) refers to nrf_drv_clock.o(i.lfclk_stop) for lfclk_stop
    nrf_drv_clock.o(i.nrf_drv_clock_uninit) refers to nrf_drv_clock.o(i.hfclk_stop) for hfclk_stop
    nrf_drv_clock.o(i.nrf_drv_clock_uninit) refers to nrf_drv_clock.o(.bss) for .bss
    nrf_drv_common.o(i.POWER_CLOCK_IRQHandler) refers to nrf_drv_clock.o(i.nrf_drv_clock_onIRQ) for nrf_drv_clock_onIRQ
    nrf_drv_common.o(i.POWER_CLOCK_IRQHandler) refers to nrf_drv_power.o(i.nrf_drv_power_onIRQ) for nrf_drv_power_onIRQ
    nrf_drv_common.o(i.nrf_drv_common_clock_irq_disable) refers to nrf_drv_power.o(i.nrf_drv_power_init_check) for nrf_drv_power_init_check
    nrf_drv_common.o(i.nrf_drv_common_clock_irq_disable) refers to nrf_drv_common.o(i.nrf_drv_common_irq_disable) for nrf_drv_common_irq_disable
    nrf_drv_common.o(i.nrf_drv_common_power_irq_disable) refers to nrf_drv_clock.o(i.nrf_drv_clock_init_check) for nrf_drv_clock_init_check
    nrf_drv_common.o(i.nrf_drv_common_power_irq_disable) refers to nrf_drv_common.o(i.nrf_drv_common_irq_disable) for nrf_drv_common_irq_disable
    nrf_drv_gpiote.o(i.GPIOTE_IRQHandler) refers to nrf_drv_gpiote.o(i.nrf_gpiote_event_is_set) for nrf_gpiote_event_is_set
    nrf_drv_gpiote.o(i.GPIOTE_IRQHandler) refers to nrf_drv_gpiote.o(i.nrf_gpiote_event_clear) for nrf_gpiote_event_clear
    nrf_drv_gpiote.o(i.GPIOTE_IRQHandler) refers to nrf_drv_gpiote.o(i.nrf_gpio_ports_read) for nrf_gpio_ports_read
    nrf_drv_gpiote.o(i.GPIOTE_IRQHandler) refers to nrf_drv_gpiote.o(i.nrf_bitmask_bit_is_set) for nrf_bitmask_bit_is_set
    nrf_drv_gpiote.o(i.GPIOTE_IRQHandler) refers to nrf_drv_gpiote.o(i.channel_port_get) for channel_port_get
    nrf_drv_gpiote.o(i.GPIOTE_IRQHandler) refers to nrf_drv_gpiote.o(i.nrf_gpio_pin_port_decode) for nrf_gpio_pin_port_decode
    nrf_drv_gpiote.o(i.GPIOTE_IRQHandler) refers to nrf_drv_gpiote.o(i.nrf_gpio_cfg_sense_set) for nrf_gpio_cfg_sense_set
    nrf_drv_gpiote.o(i.GPIOTE_IRQHandler) refers to nrf_drv_gpiote.o(.bss) for .bss
    nrf_drv_gpiote.o(i.channel_free) refers to nrf_drv_gpiote.o(.bss) for .bss
    nrf_drv_gpiote.o(i.channel_port_alloc) refers to nrf_drv_gpiote.o(.bss) for .bss
    nrf_drv_gpiote.o(i.channel_port_get) refers to nrf_drv_gpiote.o(.bss) for .bss
    nrf_drv_gpiote.o(i.nrf_drv_gpiote_clr_task_addr_get) refers to nrf_drv_gpiote.o(i.channel_port_get) for channel_port_get
    nrf_drv_gpiote.o(i.nrf_drv_gpiote_clr_task_trigger) refers to nrf_drv_gpiote.o(i.channel_port_get) for channel_port_get
    nrf_drv_gpiote.o(i.nrf_drv_gpiote_in_event_addr_get) refers to nrf_drv_gpiote.o(i.pin_in_use_by_te) for pin_in_use_by_te
    nrf_drv_gpiote.o(i.nrf_drv_gpiote_in_event_addr_get) refers to nrf_drv_gpiote.o(i.channel_port_get) for channel_port_get
    nrf_drv_gpiote.o(i.nrf_drv_gpiote_in_event_disable) refers to nrf_drv_gpiote.o(i.pin_in_use_by_port) for pin_in_use_by_port
    nrf_drv_gpiote.o(i.nrf_drv_gpiote_in_event_disable) refers to nrf_drv_gpiote.o(i.nrf_gpio_cfg_sense_set) for nrf_gpio_cfg_sense_set
    nrf_drv_gpiote.o(i.nrf_drv_gpiote_in_event_disable) refers to nrf_drv_gpiote.o(i.pin_in_use_by_te) for pin_in_use_by_te
    nrf_drv_gpiote.o(i.nrf_drv_gpiote_in_event_disable) refers to nrf_drv_gpiote.o(i.channel_port_get) for channel_port_get
    nrf_drv_gpiote.o(i.nrf_drv_gpiote_in_event_enable) refers to nrf_drv_gpiote.o(i.pin_in_use_by_port) for pin_in_use_by_port
    nrf_drv_gpiote.o(i.nrf_drv_gpiote_in_event_enable) refers to nrf_drv_gpiote.o(i.channel_port_get) for channel_port_get
    nrf_drv_gpiote.o(i.nrf_drv_gpiote_in_event_enable) refers to nrf_drv_gpiote.o(i.nrf_gpio_pin_read) for nrf_gpio_pin_read
    nrf_drv_gpiote.o(i.nrf_drv_gpiote_in_event_enable) refers to nrf_drv_gpiote.o(i.nrf_gpio_cfg_sense_set) for nrf_gpio_cfg_sense_set
    nrf_drv_gpiote.o(i.nrf_drv_gpiote_in_event_enable) refers to nrf_drv_gpiote.o(i.pin_in_use_by_te) for pin_in_use_by_te
    nrf_drv_gpiote.o(i.nrf_drv_gpiote_in_event_enable) refers to nrf_drv_gpiote.o(i.nrf_gpiote_event_clear) for nrf_gpiote_event_clear
    nrf_drv_gpiote.o(i.nrf_drv_gpiote_in_event_enable) refers to nrf_drv_gpiote.o(.bss) for .bss
    nrf_drv_gpiote.o(i.nrf_drv_gpiote_in_init) refers to nrf_drv_gpiote.o(i.channel_port_alloc) for channel_port_alloc
    nrf_drv_gpiote.o(i.nrf_drv_gpiote_in_init) refers to nrf_drv_gpiote.o(i.nrf_gpio_pin_port_decode) for nrf_gpio_pin_port_decode
    nrf_drv_gpiote.o(i.nrf_drv_gpiote_in_init) refers to nrf_drv_gpiote.o(i.nrf_gpio_cfg) for nrf_gpio_cfg
    nrf_drv_gpiote.o(i.nrf_drv_gpiote_in_init) refers to nrf_drv_gpiote.o(.bss) for .bss
    nrf_drv_gpiote.o(i.nrf_drv_gpiote_in_is_set) refers to nrf_drv_gpiote.o(i.nrf_gpio_pin_read) for nrf_gpio_pin_read
    nrf_drv_gpiote.o(i.nrf_drv_gpiote_in_uninit) refers to nrf_drv_gpiote.o(i.nrf_drv_gpiote_in_event_disable) for nrf_drv_gpiote_in_event_disable
    nrf_drv_gpiote.o(i.nrf_drv_gpiote_in_uninit) refers to nrf_drv_gpiote.o(i.pin_in_use_by_te) for pin_in_use_by_te
    nrf_drv_gpiote.o(i.nrf_drv_gpiote_in_uninit) refers to nrf_drv_gpiote.o(i.channel_port_get) for channel_port_get
    nrf_drv_gpiote.o(i.nrf_drv_gpiote_in_uninit) refers to nrf_drv_gpiote.o(i.nrf_gpio_cfg_default) for nrf_gpio_cfg_default
    nrf_drv_gpiote.o(i.nrf_drv_gpiote_in_uninit) refers to nrf_drv_gpiote.o(i.channel_free) for channel_free
    nrf_drv_gpiote.o(i.nrf_drv_gpiote_in_uninit) refers to nrf_drv_gpiote.o(.bss) for .bss
    nrf_drv_gpiote.o(i.nrf_drv_gpiote_init) refers to nrf_drv_gpiote.o(i.channel_free) for channel_free
    nrf_drv_gpiote.o(i.nrf_drv_gpiote_init) refers to nrf_drv_common.o(i.nrf_drv_common_irq_enable) for nrf_drv_common_irq_enable
    nrf_drv_gpiote.o(i.nrf_drv_gpiote_init) refers to nrf_drv_gpiote.o(i.nrf_gpiote_event_clear) for nrf_gpiote_event_clear
    nrf_drv_gpiote.o(i.nrf_drv_gpiote_init) refers to nrf_drv_gpiote.o(.bss) for .bss
    nrf_drv_gpiote.o(i.nrf_drv_gpiote_is_init) refers to nrf_drv_gpiote.o(.bss) for .bss
    nrf_drv_gpiote.o(i.nrf_drv_gpiote_out_clear) refers to nrf_drv_gpiote.o(i.nrf_gpio_pin_clear) for nrf_gpio_pin_clear
    nrf_drv_gpiote.o(i.nrf_drv_gpiote_out_init) refers to nrf_drv_gpiote.o(i.channel_port_alloc) for channel_port_alloc
    nrf_drv_gpiote.o(i.nrf_drv_gpiote_out_init) refers to nrf_drv_gpiote.o(i.nrf_gpio_pin_clear) for nrf_gpio_pin_clear
    nrf_drv_gpiote.o(i.nrf_drv_gpiote_out_init) refers to nrf_drv_gpiote.o(i.nrf_gpio_cfg) for nrf_gpio_cfg
    nrf_drv_gpiote.o(i.nrf_drv_gpiote_out_init) refers to nrf_drv_gpiote.o(i.nrf_gpio_pin_set) for nrf_gpio_pin_set
    nrf_drv_gpiote.o(i.nrf_drv_gpiote_out_init) refers to nrf_drv_gpiote.o(.bss) for .bss
    nrf_drv_gpiote.o(i.nrf_drv_gpiote_out_set) refers to nrf_drv_gpiote.o(i.nrf_gpio_pin_set) for nrf_gpio_pin_set
    nrf_drv_gpiote.o(i.nrf_drv_gpiote_out_task_addr_get) refers to nrf_drv_gpiote.o(i.channel_port_get) for channel_port_get
    nrf_drv_gpiote.o(i.nrf_drv_gpiote_out_task_disable) refers to nrf_drv_gpiote.o(.bss) for .bss
    nrf_drv_gpiote.o(i.nrf_drv_gpiote_out_task_enable) refers to nrf_drv_gpiote.o(.bss) for .bss
    nrf_drv_gpiote.o(i.nrf_drv_gpiote_out_task_force) refers to nrf_drv_gpiote.o(.bss) for .bss
    nrf_drv_gpiote.o(i.nrf_drv_gpiote_out_task_trigger) refers to nrf_drv_gpiote.o(i.channel_port_get) for channel_port_get
    nrf_drv_gpiote.o(i.nrf_drv_gpiote_out_toggle) refers to nrf_drv_gpiote.o(i.nrf_gpio_pin_port_decode) for nrf_gpio_pin_port_decode
    nrf_drv_gpiote.o(i.nrf_drv_gpiote_out_uninit) refers to nrf_drv_gpiote.o(i.pin_in_use_by_te) for pin_in_use_by_te
    nrf_drv_gpiote.o(i.nrf_drv_gpiote_out_uninit) refers to nrf_drv_gpiote.o(i.channel_port_get) for channel_port_get
    nrf_drv_gpiote.o(i.nrf_drv_gpiote_out_uninit) refers to nrf_drv_gpiote.o(i.channel_free) for channel_free
    nrf_drv_gpiote.o(i.nrf_drv_gpiote_out_uninit) refers to nrf_drv_gpiote.o(i.nrf_gpio_cfg_default) for nrf_gpio_cfg_default
    nrf_drv_gpiote.o(i.nrf_drv_gpiote_out_uninit) refers to nrf_drv_gpiote.o(.bss) for .bss
    nrf_drv_gpiote.o(i.nrf_drv_gpiote_set_task_addr_get) refers to nrf_drv_gpiote.o(i.channel_port_get) for channel_port_get
    nrf_drv_gpiote.o(i.nrf_drv_gpiote_set_task_trigger) refers to nrf_drv_gpiote.o(i.channel_port_get) for channel_port_get
    nrf_drv_gpiote.o(i.nrf_drv_gpiote_uninit) refers to nrf_drv_gpiote.o(i.nrf_drv_gpiote_in_uninit) for nrf_drv_gpiote_in_uninit
    nrf_drv_gpiote.o(i.nrf_drv_gpiote_uninit) refers to nrf_drv_gpiote.o(i.nrf_drv_gpiote_out_uninit) for nrf_drv_gpiote_out_uninit
    nrf_drv_gpiote.o(i.nrf_drv_gpiote_uninit) refers to nrf_drv_gpiote.o(.bss) for .bss
    nrf_drv_gpiote.o(i.nrf_gpio_cfg) refers to nrf_drv_gpiote.o(i.nrf_gpio_pin_port_decode) for nrf_gpio_pin_port_decode
    nrf_drv_gpiote.o(i.nrf_gpio_cfg_default) refers to nrf_drv_gpiote.o(i.nrf_gpio_cfg) for nrf_gpio_cfg
    nrf_drv_gpiote.o(i.nrf_gpio_cfg_sense_set) refers to nrf_drv_gpiote.o(i.nrf_gpio_pin_port_decode) for nrf_gpio_pin_port_decode
    nrf_drv_gpiote.o(i.nrf_gpio_pin_clear) refers to nrf_drv_gpiote.o(i.nrf_gpio_pin_port_decode) for nrf_gpio_pin_port_decode
    nrf_drv_gpiote.o(i.nrf_gpio_pin_read) refers to nrf_drv_gpiote.o(i.nrf_gpio_pin_port_decode) for nrf_gpio_pin_port_decode
    nrf_drv_gpiote.o(i.nrf_gpio_pin_set) refers to nrf_drv_gpiote.o(i.nrf_gpio_pin_port_decode) for nrf_gpio_pin_port_decode
    nrf_drv_gpiote.o(i.nrf_gpio_ports_read) refers to nrf_drv_gpiote.o(.constdata) for .constdata
    nrf_drv_gpiote.o(i.pin_in_use_by_port) refers to nrf_drv_gpiote.o(.bss) for .bss
    nrf_drv_gpiote.o(i.pin_in_use_by_te) refers to nrf_drv_gpiote.o(.bss) for .bss
    nrf_drv_power.o(i.nrf_drv_power_init) refers to nrf_drv_common.o(i.nrf_drv_common_irq_enable) for nrf_drv_common_irq_enable
    nrf_drv_power.o(i.nrf_drv_power_init) refers to nrf_drv_power.o(.data) for .data
    nrf_drv_power.o(i.nrf_drv_power_init) refers to nrf_drv_power.o(.constdata) for .constdata
    nrf_drv_power.o(i.nrf_drv_power_init_check) refers to nrf_drv_power.o(.data) for .data
    nrf_drv_power.o(i.nrf_drv_power_onIRQ) refers to nrf_drv_power.o(i.nrf_power_event_get_and_clear) for nrf_power_event_get_and_clear
    nrf_drv_power.o(i.nrf_drv_power_onIRQ) refers to nrf_drv_power.o(.data) for .data
    nrf_drv_power.o(i.nrf_drv_power_pof_init) refers to nrf_drv_power.o(i.nrf_drv_power_pof_uninit) for nrf_drv_power_pof_uninit
    nrf_drv_power.o(i.nrf_drv_power_pof_init) refers to nrf_drv_power.o(.data) for .data
    nrf_drv_power.o(i.nrf_drv_power_pof_uninit) refers to nrf_drv_power.o(.data) for .data
    nrf_drv_power.o(i.nrf_drv_power_sleepevt_init) refers to nrf_drv_power.o(i.nrf_drv_power_sleepevt_uninit) for nrf_drv_power_sleepevt_uninit
    nrf_drv_power.o(i.nrf_drv_power_sleepevt_init) refers to nrf_drv_power.o(.data) for .data
    nrf_drv_power.o(i.nrf_drv_power_sleepevt_uninit) refers to nrf_drv_power.o(.data) for .data
    nrf_drv_power.o(i.nrf_drv_power_uninit) refers to nrf_drv_power.o(i.nrf_drv_power_pof_uninit) for nrf_drv_power_pof_uninit
    nrf_drv_power.o(i.nrf_drv_power_uninit) refers to nrf_drv_power.o(i.nrf_drv_power_sleepevt_uninit) for nrf_drv_power_sleepevt_uninit
    nrf_drv_power.o(i.nrf_drv_power_uninit) refers to nrf_drv_power.o(i.nrf_drv_power_usbevt_uninit) for nrf_drv_power_usbevt_uninit
    nrf_drv_power.o(i.nrf_drv_power_uninit) refers to nrf_drv_power.o(.data) for .data
    nrf_drv_power.o(i.nrf_drv_power_usbevt_init) refers to nrf_drv_power.o(i.nrf_drv_power_usbevt_uninit) for nrf_drv_power_usbevt_uninit
    nrf_drv_power.o(i.nrf_drv_power_usbevt_init) refers to nrf_drv_power.o(.data) for .data
    nrf_drv_power.o(i.nrf_drv_power_usbevt_uninit) refers to nrf_drv_power.o(.data) for .data
    nrf_drv_systick.o(i.nrf_drv_systick_delay_ms) refers to nrf_drv_systick.o(i.nrf_drv_systick_ms_tick) for nrf_drv_systick_ms_tick
    nrf_drv_systick.o(i.nrf_drv_systick_delay_ms) refers to nrf_drv_systick.o(i.nrf_drv_systick_delay_ticks) for nrf_drv_systick_delay_ticks
    nrf_drv_systick.o(i.nrf_drv_systick_delay_us) refers to nrf_drv_systick.o(i.nrf_drv_systick_delay_ticks) for nrf_drv_systick_delay_ticks
    nrf_drv_systick.o(i.nrf_drv_systick_delay_us) refers to system_nrf52840.o(.data) for SystemCoreClock
    nrf_drv_systick.o(i.nrf_drv_systick_ms_tick) refers to system_nrf52840.o(.data) for SystemCoreClock
    nrf_drv_systick.o(i.nrf_drv_systick_test) refers to system_nrf52840.o(.data) for SystemCoreClock
    nrf_drv_uart.o(i.UARTE0_UART0_IRQHandler) refers to nrf_drv_uart.o(i.uarte_irq_handler) for uarte_irq_handler
    nrf_drv_uart.o(i.UARTE0_UART0_IRQHandler) refers to nrf_drv_uart.o(i.uart_irq_handler) for uart_irq_handler
    nrf_drv_uart.o(i.UARTE0_UART0_IRQHandler) refers to nrf_drv_uart.o(.bss) for .bss
    nrf_drv_uart.o(i.apply_config) refers to nrf_drv_uart.o(i.nrf_gpio_pin_set) for nrf_gpio_pin_set
    nrf_drv_uart.o(i.apply_config) refers to nrf_drv_uart.o(i.nrf_gpio_cfg_output) for nrf_gpio_cfg_output
    nrf_drv_uart.o(i.apply_config) refers to nrf_drv_uart.o(i.nrf_gpio_cfg_input) for nrf_gpio_cfg_input
    nrf_drv_uart.o(i.apply_config) refers to nrf_drv_uart.o(.bss) for .bss
    nrf_drv_uart.o(i.interrupts_enable) refers to nrf_drv_uart.o(i.nrf_uarte_event_clear) for nrf_uarte_event_clear
    nrf_drv_uart.o(i.interrupts_enable) refers to nrf_drv_uart.o(i.nrf_uart_event_clear) for nrf_uart_event_clear
    nrf_drv_uart.o(i.interrupts_enable) refers to nrf_drv_uart.o(i.nrf_drv_get_IRQn) for nrf_drv_get_IRQn
    nrf_drv_uart.o(i.interrupts_enable) refers to nrf_drv_common.o(i.nrf_drv_common_irq_enable) for nrf_drv_common_irq_enable
    nrf_drv_uart.o(i.interrupts_enable) refers to nrf_drv_uart.o(.bss) for .bss
    nrf_drv_uart.o(i.nrf_drv_uart_errorsrc_get) refers to nrf_drv_uart.o(i.nrf_uarte_event_clear) for nrf_uarte_event_clear
    nrf_drv_uart.o(i.nrf_drv_uart_errorsrc_get) refers to nrf_drv_uart.o(i.nrf_uart_event_clear) for nrf_uart_event_clear
    nrf_drv_uart.o(i.nrf_drv_uart_errorsrc_get) refers to nrf_drv_uart.o(.bss) for .bss
    nrf_drv_uart.o(i.nrf_drv_uart_init) refers to nrf_drv_uart.o(i.apply_config) for apply_config
    nrf_drv_uart.o(i.nrf_drv_uart_init) refers to nrf_drv_uart.o(i.interrupts_enable) for interrupts_enable
    nrf_drv_uart.o(i.nrf_drv_uart_init) refers to nrf_drv_uart.o(.bss) for .bss
    nrf_drv_uart.o(i.nrf_drv_uart_rx) refers to nrf_drv_uart.o(i.nrf_drv_is_in_RAM) for nrf_drv_is_in_RAM
    nrf_drv_uart.o(i.nrf_drv_uart_rx) refers to nrf_drv_uart.o(i.nrf_drv_uart_rx_for_uarte) for nrf_drv_uart_rx_for_uarte
    nrf_drv_uart.o(i.nrf_drv_uart_rx) refers to nrf_drv_uart.o(i.nrf_drv_uart_rx_for_uart) for nrf_drv_uart_rx_for_uart
    nrf_drv_uart.o(i.nrf_drv_uart_rx) refers to nrf_drv_uart.o(.bss) for .bss
    nrf_drv_uart.o(i.nrf_drv_uart_rx_abort) refers to nrf_drv_uart.o(.bss) for .bss
    nrf_drv_uart.o(i.nrf_drv_uart_rx_disable) refers to nrf_drv_uart.o(.bss) for .bss
    nrf_drv_uart.o(i.nrf_drv_uart_rx_enable) refers to nrf_drv_uart.o(i.rx_enable) for rx_enable
    nrf_drv_uart.o(i.nrf_drv_uart_rx_enable) refers to nrf_drv_uart.o(.bss) for .bss
    nrf_drv_uart.o(i.nrf_drv_uart_rx_for_uart) refers to nrf_drv_uart.o(i.rx_enable) for rx_enable
    nrf_drv_uart.o(i.nrf_drv_uart_rx_for_uart) refers to nrf_drv_uart.o(i.nrf_uart_event_clear) for nrf_uart_event_clear
    nrf_drv_uart.o(i.nrf_drv_uart_rx_for_uart) refers to nrf_drv_uart.o(i.nrf_uart_event_check) for nrf_uart_event_check
    nrf_drv_uart.o(i.nrf_drv_uart_rx_for_uart) refers to nrf_drv_uart.o(i.rx_byte) for rx_byte
    nrf_drv_uart.o(i.nrf_drv_uart_rx_for_uart) refers to nrf_drv_uart.o(.bss) for .bss
    nrf_drv_uart.o(i.nrf_drv_uart_rx_for_uarte) refers to nrf_drv_uart.o(i.nrf_uarte_event_clear) for nrf_uarte_event_clear
    nrf_drv_uart.o(i.nrf_drv_uart_rx_for_uarte) refers to nrf_drv_uart.o(i.nrf_uarte_event_check) for nrf_uarte_event_check
    nrf_drv_uart.o(i.nrf_drv_uart_rx_for_uarte) refers to nrf_drv_uart.o(.bss) for .bss
    nrf_drv_uart.o(i.nrf_drv_uart_rx_ready) refers to nrf_drv_uart.o(.bss) for .bss
    nrf_drv_uart.o(i.nrf_drv_uart_tx) refers to nrf_drv_uart.o(i.nrf_drv_is_in_RAM) for nrf_drv_is_in_RAM
    nrf_drv_uart.o(i.nrf_drv_uart_tx) refers to nrf_drv_uart.o(i.nrf_drv_uart_tx_in_progress) for nrf_drv_uart_tx_in_progress
    nrf_drv_uart.o(i.nrf_drv_uart_tx) refers to nrf_drv_uart.o(i.nrf_uarte_event_clear) for nrf_uarte_event_clear
    nrf_drv_uart.o(i.nrf_drv_uart_tx) refers to nrf_drv_uart.o(i.nrf_uarte_event_check) for nrf_uarte_event_check
    nrf_drv_uart.o(i.nrf_drv_uart_tx) refers to nrf_drv_uart.o(i.nrf_uart_event_clear) for nrf_uart_event_clear
    nrf_drv_uart.o(i.nrf_drv_uart_tx) refers to nrf_drv_uart.o(i.tx_byte) for tx_byte
    nrf_drv_uart.o(i.nrf_drv_uart_tx) refers to nrf_drv_uart.o(i.nrf_uart_event_check) for nrf_uart_event_check
    nrf_drv_uart.o(i.nrf_drv_uart_tx) refers to nrf_drv_uart.o(.bss) for .bss
    nrf_drv_uart.o(i.nrf_drv_uart_tx_abort) refers to nrf_drv_uart.o(i.nrf_uarte_event_clear) for nrf_uarte_event_clear
    nrf_drv_uart.o(i.nrf_drv_uart_tx_abort) refers to nrf_drv_uart.o(i.nrf_uarte_event_check) for nrf_uarte_event_check
    nrf_drv_uart.o(i.nrf_drv_uart_tx_abort) refers to nrf_drv_uart.o(i.tx_done_event) for tx_done_event
    nrf_drv_uart.o(i.nrf_drv_uart_tx_abort) refers to nrf_drv_uart.o(.bss) for .bss
    nrf_drv_uart.o(i.nrf_drv_uart_tx_in_progress) refers to nrf_drv_uart.o(.bss) for .bss
    nrf_drv_uart.o(i.nrf_drv_uart_uninit) refers to nrf_drv_uart.o(i.nrf_drv_get_IRQn) for nrf_drv_get_IRQn
    nrf_drv_uart.o(i.nrf_drv_uart_uninit) refers to nrf_drv_uart.o(i.nrf_drv_common_irq_disable) for nrf_drv_common_irq_disable
    nrf_drv_uart.o(i.nrf_drv_uart_uninit) refers to nrf_drv_uart.o(i.pins_to_default) for pins_to_default
    nrf_drv_uart.o(i.nrf_drv_uart_uninit) refers to nrf_drv_uart.o(.bss) for .bss
    nrf_drv_uart.o(i.nrf_gpio_cfg) refers to nrf_drv_uart.o(i.nrf_gpio_pin_port_decode) for nrf_gpio_pin_port_decode
    nrf_drv_uart.o(i.nrf_gpio_cfg_default) refers to nrf_drv_uart.o(i.nrf_gpio_cfg) for nrf_gpio_cfg
    nrf_drv_uart.o(i.nrf_gpio_cfg_input) refers to nrf_drv_uart.o(i.nrf_gpio_cfg) for nrf_gpio_cfg
    nrf_drv_uart.o(i.nrf_gpio_cfg_output) refers to nrf_drv_uart.o(i.nrf_gpio_cfg) for nrf_gpio_cfg
    nrf_drv_uart.o(i.nrf_gpio_pin_set) refers to nrf_drv_uart.o(i.nrf_gpio_pin_port_decode) for nrf_gpio_pin_port_decode
    nrf_drv_uart.o(i.pins_to_default) refers to nrf_drv_uart.o(i.nrf_gpio_cfg_default) for nrf_gpio_cfg_default
    nrf_drv_uart.o(i.pins_to_default) refers to nrf_drv_uart.o(.bss) for .bss
    nrf_drv_uart.o(i.rx_byte) refers to nrf_drv_uart.o(i.nrf_uart_event_clear) for nrf_uart_event_clear
    nrf_drv_uart.o(i.rx_enable) refers to nrf_drv_uart.o(i.nrf_uart_event_clear) for nrf_uart_event_clear
    nrf_drv_uart.o(i.tx_byte) refers to nrf_drv_uart.o(i.nrf_uart_event_clear) for nrf_uart_event_clear
    nrf_drv_uart.o(i.uart_irq_handler) refers to nrf_drv_uart.o(i.nrf_uart_int_enable_check) for nrf_uart_int_enable_check
    nrf_drv_uart.o(i.uart_irq_handler) refers to nrf_drv_uart.o(i.nrf_uart_event_check) for nrf_uart_event_check
    nrf_drv_uart.o(i.uart_irq_handler) refers to nrf_drv_uart.o(i.nrf_uart_event_clear) for nrf_uart_event_clear
    nrf_drv_uart.o(i.uart_irq_handler) refers to nrf_drv_uart.o(i.rx_byte) for rx_byte
    nrf_drv_uart.o(i.uart_irq_handler) refers to nrf_drv_uart.o(i.rx_done_event) for rx_done_event
    nrf_drv_uart.o(i.uart_irq_handler) refers to nrf_drv_uart.o(i.tx_byte) for tx_byte
    nrf_drv_uart.o(i.uart_irq_handler) refers to nrf_drv_uart.o(i.tx_done_event) for tx_done_event
    nrf_drv_uart.o(i.uarte_irq_handler) refers to nrf_drv_uart.o(i.nrf_uarte_event_check) for nrf_uarte_event_check
    nrf_drv_uart.o(i.uarte_irq_handler) refers to nrf_drv_uart.o(i.nrf_uarte_event_clear) for nrf_uarte_event_clear
    nrf_drv_uart.o(i.uarte_irq_handler) refers to nrf_drv_uart.o(i.rx_done_event) for rx_done_event
    nrf_drv_uart.o(i.uarte_irq_handler) refers to nrf_drv_uart.o(i.tx_done_event) for tx_done_event
    nrf_drv_usbd.o(i.USBD_IRQHandler) refers to nrf_drv_usbd.o(i.nrf_usbd_event_check) for nrf_usbd_event_check
    nrf_drv_usbd.o(i.USBD_IRQHandler) refers to nrf_drv_usbd.o(i.nrf_usbd_event_clear) for nrf_usbd_event_clear
    nrf_drv_usbd.o(i.USBD_IRQHandler) refers to nrf_drv_usbd.o(i.usbd_dmareq_process) for usbd_dmareq_process
    nrf_drv_usbd.o(i.USBD_IRQHandler) refers to nrf_drv_usbd.o(i.USBD_ISR_Setup) for USBD_ISR_Setup
    nrf_drv_usbd.o(i.USBD_IRQHandler) refers to nrf_drv_usbd.o(.data) for .data
    nrf_drv_usbd.o(i.USBD_IRQHandler) refers to nrf_drv_usbd.o(.constdata) for .constdata
    nrf_drv_usbd.o(i.USBD_ISR_EpDataStatus) refers to nrf_drv_usbd.o(i.bit2ep) for bit2ep
    nrf_drv_usbd.o(i.USBD_ISR_EpDataStatus) refers to nrf_drv_usbd.o(i.usbd_ep_data_handler) for usbd_ep_data_handler
    nrf_drv_usbd.o(i.USBD_ISR_EpDataStatus) refers to nrf_drv_usbd.o(i.usbd_dmareq_process) for usbd_dmareq_process
    nrf_drv_usbd.o(i.USBD_ISR_EpDataStatus) refers to nrf_drv_usbd.o(.data) for .data
    nrf_drv_usbd.o(i.USBD_ISR_Event) refers to nrf_drv_usbd.o(i.nrf_usbd_eventcause_clear) for nrf_usbd_eventcause_clear
    nrf_drv_usbd.o(i.USBD_ISR_Event) refers to nrf_drv_usbd.o(.constdata) for .constdata
    nrf_drv_usbd.o(i.USBD_ISR_Event) refers to nrf_drv_usbd.o(.data) for .data
    nrf_drv_usbd.o(i.USBD_ISR_Setup) refers to nrf_drv_usbd.o(i.ep2bit) for ep2bit
    nrf_drv_usbd.o(i.USBD_ISR_Setup) refers to nrf_drv_usbd.o(i.usbd_ep_abort) for usbd_ep_abort
    nrf_drv_usbd.o(i.USBD_ISR_Setup) refers to nrf_drv_usbd.o(i.nrf_atomic_u32_and) for nrf_atomic_u32_and
    nrf_drv_usbd.o(i.USBD_ISR_Setup) refers to nrf_drv_usbd.o(.data) for .data
    nrf_drv_usbd.o(i.USBD_ISR_Setup) refers to nrf_drv_usbd.o(.constdata) for .constdata
    nrf_drv_usbd.o(i.USBD_ISR_SetupData) refers to nrf_drv_usbd.o(i.ep2bit) for ep2bit
    nrf_drv_usbd.o(i.USBD_ISR_SetupData) refers to nrf_drv_usbd.o(i.usbd_ep_data_handler) for usbd_ep_data_handler
    nrf_drv_usbd.o(i.USBD_ISR_SetupData) refers to nrf_drv_usbd.o(.data) for .data
    nrf_drv_usbd.o(i.USBD_ISR_Sof) refers to nrf_drv_usbd.o(i.ep2bit) for ep2bit
    nrf_drv_usbd.o(i.USBD_ISR_Sof) refers to nrf_drv_usbd.o(.data) for .data
    nrf_drv_usbd.o(i.USBD_ISR_Started) refers to nrf_drv_usbd.o(i.bit2ep) for bit2ep
    nrf_drv_usbd.o(i.USBD_ISR_Usbreset) refers to nrf_drv_usbd.o(i.usbd_ep_abort_all) for usbd_ep_abort_all
    nrf_drv_usbd.o(i.USBD_ISR_Usbreset) refers to nrf_drv_usbd.o(.data) for .data
    nrf_drv_usbd.o(i.USBD_ISR_Usbreset) refers to nrf_drv_usbd.o(.constdata) for .constdata
    nrf_drv_usbd.o(i.USBD_ISR_dma_epin0) refers to nrf_drv_usbd.o(i.ep_state_access) for ep_state_access
    nrf_drv_usbd.o(i.USBD_ISR_dma_epin0) refers to nrf_drv_usbd.o(i.ep2bit) for ep2bit
    nrf_drv_usbd.o(i.USBD_ISR_dma_epin0) refers to nrf_drv_usbd.o(i.nrf_atomic_u32_and) for nrf_atomic_u32_and
    nrf_drv_usbd.o(i.USBD_ISR_dma_epin0) refers to nrf_drv_usbd.o(.data) for .data
    nrf_drv_usbd.o(i.USBD_ISR_dma_epin1) refers to nrf_drv_usbd.o(i.nrf_usbd_epin_dma_handler) for nrf_usbd_epin_dma_handler
    nrf_drv_usbd.o(i.USBD_ISR_dma_epin2) refers to nrf_drv_usbd.o(i.nrf_usbd_epin_dma_handler) for nrf_usbd_epin_dma_handler
    nrf_drv_usbd.o(i.USBD_ISR_dma_epin3) refers to nrf_drv_usbd.o(i.nrf_usbd_epin_dma_handler) for nrf_usbd_epin_dma_handler
    nrf_drv_usbd.o(i.USBD_ISR_dma_epin4) refers to nrf_drv_usbd.o(i.nrf_usbd_epin_dma_handler) for nrf_usbd_epin_dma_handler
    nrf_drv_usbd.o(i.USBD_ISR_dma_epin5) refers to nrf_drv_usbd.o(i.nrf_usbd_epin_dma_handler) for nrf_usbd_epin_dma_handler
    nrf_drv_usbd.o(i.USBD_ISR_dma_epin6) refers to nrf_drv_usbd.o(i.nrf_usbd_epin_dma_handler) for nrf_usbd_epin_dma_handler
    nrf_drv_usbd.o(i.USBD_ISR_dma_epin7) refers to nrf_drv_usbd.o(i.nrf_usbd_epin_dma_handler) for nrf_usbd_epin_dma_handler
    nrf_drv_usbd.o(i.USBD_ISR_dma_epin8) refers to nrf_drv_usbd.o(i.ep_state_access) for ep_state_access
    nrf_drv_usbd.o(i.USBD_ISR_dma_epin8) refers to nrf_drv_usbd.o(i.ep2bit) for ep2bit
    nrf_drv_usbd.o(i.USBD_ISR_dma_epin8) refers to nrf_drv_usbd.o(i.nrf_atomic_u32_and) for nrf_atomic_u32_and
    nrf_drv_usbd.o(i.USBD_ISR_dma_epin8) refers to nrf_drv_usbd.o(.data) for .data
    nrf_drv_usbd.o(i.USBD_ISR_dma_epin8) refers to nrf_drv_usbd.o(.constdata) for .constdata
    nrf_drv_usbd.o(i.USBD_ISR_dma_epout0) refers to nrf_drv_usbd.o(i.ep_state_access) for ep_state_access
    nrf_drv_usbd.o(i.USBD_ISR_dma_epout0) refers to nrf_drv_usbd.o(i.nrf_drv_usbd_setup_data_clear) for nrf_drv_usbd_setup_data_clear
    nrf_drv_usbd.o(i.USBD_ISR_dma_epout0) refers to nrf_drv_usbd.o(i.ep2bit) for ep2bit
    nrf_drv_usbd.o(i.USBD_ISR_dma_epout0) refers to nrf_drv_usbd.o(i.nrf_atomic_u32_and) for nrf_atomic_u32_and
    nrf_drv_usbd.o(i.USBD_ISR_dma_epout0) refers to nrf_drv_usbd.o(.data) for .data
    nrf_drv_usbd.o(i.USBD_ISR_dma_epout0) refers to nrf_drv_usbd.o(.constdata) for .constdata
    nrf_drv_usbd.o(i.USBD_ISR_dma_epout1) refers to nrf_drv_usbd.o(i.nrf_usbd_epout_dma_handler) for nrf_usbd_epout_dma_handler
    nrf_drv_usbd.o(i.USBD_ISR_dma_epout2) refers to nrf_drv_usbd.o(i.nrf_usbd_epout_dma_handler) for nrf_usbd_epout_dma_handler
    nrf_drv_usbd.o(i.USBD_ISR_dma_epout3) refers to nrf_drv_usbd.o(i.nrf_usbd_epout_dma_handler) for nrf_usbd_epout_dma_handler
    nrf_drv_usbd.o(i.USBD_ISR_dma_epout4) refers to nrf_drv_usbd.o(i.nrf_usbd_epout_dma_handler) for nrf_usbd_epout_dma_handler
    nrf_drv_usbd.o(i.USBD_ISR_dma_epout5) refers to nrf_drv_usbd.o(i.nrf_usbd_epout_dma_handler) for nrf_usbd_epout_dma_handler
    nrf_drv_usbd.o(i.USBD_ISR_dma_epout6) refers to nrf_drv_usbd.o(i.nrf_usbd_epout_dma_handler) for nrf_usbd_epout_dma_handler
    nrf_drv_usbd.o(i.USBD_ISR_dma_epout7) refers to nrf_drv_usbd.o(i.nrf_usbd_epout_dma_handler) for nrf_usbd_epout_dma_handler
    nrf_drv_usbd.o(i.USBD_ISR_dma_epout8) refers to nrf_drv_usbd.o(i.ep_state_access) for ep_state_access
    nrf_drv_usbd.o(i.USBD_ISR_dma_epout8) refers to nrf_drv_usbd.o(i.ep2bit) for ep2bit
    nrf_drv_usbd.o(i.USBD_ISR_dma_epout8) refers to nrf_drv_usbd.o(i.nrf_atomic_u32_and) for nrf_atomic_u32_and
    nrf_drv_usbd.o(i.USBD_ISR_dma_epout8) refers to nrf_drv_usbd.o(.data) for .data
    nrf_drv_usbd.o(i.USBD_ISR_dma_epout8) refers to nrf_drv_usbd.o(.constdata) for .constdata
    nrf_drv_usbd.o(i.ep_state_access) refers to nrf_drv_usbd.o(.bss) for .bss
    nrf_drv_usbd.o(i.nrf_atomic_u32_and) refers to nrf_drv_usbd.o(.emb_text) for __asm___14_nrf_drv_usbd_c_f1d4739e__nrf_atomic_internal_and
    nrf_drv_usbd.o(i.nrf_drv_usbd_disable) refers to nrf_drv_usbd.o(i.nrf_drv_usbd_stop) for nrf_drv_usbd_stop
    nrf_drv_usbd.o(i.nrf_drv_usbd_disable) refers to nrf_drv_usbd.o(.data) for .data
    nrf_drv_usbd.o(i.nrf_drv_usbd_enable) refers to nrf_drv_usbd.o(i.nrf_usbd_eventcause_clear) for nrf_usbd_eventcause_clear
    nrf_drv_usbd.o(i.nrf_drv_usbd_enable) refers to nrf_drv_usbd.o(.data) for .data
    nrf_drv_usbd.o(i.nrf_drv_usbd_ep_disable) refers to nrf_drv_usbd.o(i.nrf_drv_usbd_ep_to_int) for nrf_drv_usbd_ep_to_int
    nrf_drv_usbd.o(i.nrf_drv_usbd_ep_enable) refers to nrf_drv_usbd.o(i.nrf_drv_usbd_ep_to_int) for nrf_drv_usbd_ep_to_int
    nrf_drv_usbd.o(i.nrf_drv_usbd_ep_enable) refers to app_util_platform.o(i.app_util_critical_region_enter) for app_util_critical_region_enter
    nrf_drv_usbd.o(i.nrf_drv_usbd_ep_enable) refers to nrf_drv_usbd.o(i.ep2bit) for ep2bit
    nrf_drv_usbd.o(i.nrf_drv_usbd_ep_enable) refers to nrf_drv_usbd.o(i.ep_state_access) for ep_state_access
    nrf_drv_usbd.o(i.nrf_drv_usbd_ep_enable) refers to nrf_drv_usbd.o(i.nrf_drv_usbd_ep_transfer) for nrf_drv_usbd_ep_transfer
    nrf_drv_usbd.o(i.nrf_drv_usbd_ep_enable) refers to app_util_platform.o(i.app_util_critical_region_exit) for app_util_critical_region_exit
    nrf_drv_usbd.o(i.nrf_drv_usbd_ep_enable) refers to nrf_drv_usbd.o(.data) for .data
    nrf_drv_usbd.o(i.nrf_drv_usbd_ep_handled_transfer) refers to nrf_drv_usbd.o(i.ep2bit) for ep2bit
    nrf_drv_usbd.o(i.nrf_drv_usbd_ep_handled_transfer) refers to app_util_platform.o(i.app_util_critical_region_enter) for app_util_critical_region_enter
    nrf_drv_usbd.o(i.nrf_drv_usbd_ep_handled_transfer) refers to nrf_drv_usbd.o(i.nrf_usbd_ep_is_stall) for nrf_usbd_ep_is_stall
    nrf_drv_usbd.o(i.nrf_drv_usbd_ep_handled_transfer) refers to nrf_drv_usbd.o(i.ep_state_access) for ep_state_access
    nrf_drv_usbd.o(i.nrf_drv_usbd_ep_handled_transfer) refers to nrf_drv_usbd.o(i.usbd_int_rise) for usbd_int_rise
    nrf_drv_usbd.o(i.nrf_drv_usbd_ep_handled_transfer) refers to app_util_platform.o(i.app_util_critical_region_exit) for app_util_critical_region_exit
    nrf_drv_usbd.o(i.nrf_drv_usbd_ep_handled_transfer) refers to nrf_drv_usbd.o(.data) for .data
    nrf_drv_usbd.o(i.nrf_drv_usbd_ep_is_busy) refers to nrf_drv_usbd.o(i.ep2bit) for ep2bit
    nrf_drv_usbd.o(i.nrf_drv_usbd_ep_is_busy) refers to nrf_drv_usbd.o(.data) for .data
    nrf_drv_usbd.o(i.nrf_drv_usbd_ep_max_packet_size_get) refers to nrf_drv_usbd.o(i.ep_state_access) for ep_state_access
    nrf_drv_usbd.o(i.nrf_drv_usbd_ep_max_packet_size_set) refers to nrf_drv_usbd.o(i.ep_state_access) for ep_state_access
    nrf_drv_usbd.o(i.nrf_drv_usbd_ep_stall_check) refers to nrf_drv_usbd.o(i.nrf_usbd_ep_is_stall) for nrf_usbd_ep_is_stall
    nrf_drv_usbd.o(i.nrf_drv_usbd_ep_status_get) refers to nrf_drv_usbd.o(i.ep_state_access) for ep_state_access
    nrf_drv_usbd.o(i.nrf_drv_usbd_ep_status_get) refers to app_util_platform.o(i.app_util_critical_region_enter) for app_util_critical_region_enter
    nrf_drv_usbd.o(i.nrf_drv_usbd_ep_status_get) refers to app_util_platform.o(i.app_util_critical_region_exit) for app_util_critical_region_exit
    nrf_drv_usbd.o(i.nrf_drv_usbd_ep_to_int) refers to nrf_drv_usbd.o(.constdata) for .constdata
    nrf_drv_usbd.o(i.nrf_drv_usbd_ep_transfer) refers to nrf_drv_usbd.o(i.ep2bit) for ep2bit
    nrf_drv_usbd.o(i.nrf_drv_usbd_ep_transfer) refers to app_util_platform.o(i.app_util_critical_region_enter) for app_util_critical_region_enter
    nrf_drv_usbd.o(i.nrf_drv_usbd_ep_transfer) refers to nrf_drv_usbd.o(i.nrf_usbd_ep_is_stall) for nrf_usbd_ep_is_stall
    nrf_drv_usbd.o(i.nrf_drv_usbd_ep_transfer) refers to nrf_drv_usbd.o(i.ep_state_access) for ep_state_access
    nrf_drv_usbd.o(i.nrf_drv_usbd_ep_transfer) refers to nrf_drv_usbd.o(i.usbd_int_rise) for usbd_int_rise
    nrf_drv_usbd.o(i.nrf_drv_usbd_ep_transfer) refers to app_util_platform.o(i.app_util_critical_region_exit) for app_util_critical_region_exit
    nrf_drv_usbd.o(i.nrf_drv_usbd_ep_transfer) refers to nrf_drv_usbd.o(.data) for .data
    nrf_drv_usbd.o(i.nrf_drv_usbd_ep_transfer) refers to nrf_drv_usbd.o(.bss) for .bss
    nrf_drv_usbd.o(i.nrf_drv_usbd_ep_transfer) refers to nrf_drv_usbd.o(i.nrf_drv_usbd_feeder_ram_zlp) for nrf_drv_usbd_feeder_ram_zlp
    nrf_drv_usbd.o(i.nrf_drv_usbd_ep_transfer) refers to nrf_drv_usbd.o(i.nrf_drv_usbd_feeder_flash_zlp) for nrf_drv_usbd_feeder_flash_zlp
    nrf_drv_usbd.o(i.nrf_drv_usbd_ep_transfer) refers to nrf_drv_usbd.o(i.nrf_drv_usbd_feeder_ram) for nrf_drv_usbd_feeder_ram
    nrf_drv_usbd.o(i.nrf_drv_usbd_ep_transfer) refers to nrf_drv_usbd.o(i.nrf_drv_usbd_feeder_flash) for nrf_drv_usbd_feeder_flash
    nrf_drv_usbd.o(i.nrf_drv_usbd_ep_transfer) refers to nrf_drv_usbd.o(i.nrf_drv_usbd_consumer) for nrf_drv_usbd_consumer
    nrf_drv_usbd.o(i.nrf_drv_usbd_feeder_buffer_get) refers to nrf_drv_usbd.o(.bss) for .bss
    nrf_drv_usbd.o(i.nrf_drv_usbd_feeder_flash) refers to memcpya.o(.text) for __aeabi_memcpy
    nrf_drv_usbd.o(i.nrf_drv_usbd_feeder_flash) refers to nrf_drv_usbd.o(.bss) for .bss
    nrf_drv_usbd.o(i.nrf_drv_usbd_feeder_flash_zlp) refers to memcpya.o(.text) for __aeabi_memcpy
    nrf_drv_usbd.o(i.nrf_drv_usbd_feeder_flash_zlp) refers to nrf_drv_usbd.o(.bss) for .bss
    nrf_drv_usbd.o(i.nrf_drv_usbd_init) refers to nrf_drv_systick.o(i.nrf_drv_systick_init) for nrf_drv_systick_init
    nrf_drv_usbd.o(i.nrf_drv_usbd_init) refers to nrf_drv_clock.o(i.nrf_drv_clock_hfclk_request) for nrf_drv_clock_hfclk_request
    nrf_drv_usbd.o(i.nrf_drv_usbd_init) refers to nrf_drv_clock.o(i.nrf_drv_clock_hfclk_is_running) for nrf_drv_clock_hfclk_is_running
    nrf_drv_usbd.o(i.nrf_drv_usbd_init) refers to nrf_drv_usbd.o(i.nrf_drv_usbd_ep_max_packet_size_set) for nrf_drv_usbd_ep_max_packet_size_set
    nrf_drv_usbd.o(i.nrf_drv_usbd_init) refers to nrf_drv_usbd.o(i.ep_state_access) for ep_state_access
    nrf_drv_usbd.o(i.nrf_drv_usbd_init) refers to nrf_drv_usbd.o(.data) for .data
    nrf_drv_usbd.o(i.nrf_drv_usbd_is_enabled) refers to nrf_drv_usbd.o(.data) for .data
    nrf_drv_usbd.o(i.nrf_drv_usbd_is_initialized) refers to nrf_drv_usbd.o(.data) for .data
    nrf_drv_usbd.o(i.nrf_drv_usbd_is_started) refers to nrf_drv_usbd.o(i.nrf_drv_usbd_is_enabled) for nrf_drv_usbd_is_enabled
    nrf_drv_usbd.o(i.nrf_drv_usbd_last_setup_dir_get) refers to nrf_drv_usbd.o(.data) for .data
    nrf_drv_usbd.o(i.nrf_drv_usbd_setup_clear) refers to nrf_drv_usbd.o(i.nrf_usbd_task_trigger) for nrf_usbd_task_trigger
    nrf_drv_usbd.o(i.nrf_drv_usbd_setup_data_clear) refers to nrf_drv_usbd.o(i.nrf_usbd_task_trigger) for nrf_usbd_task_trigger
    nrf_drv_usbd.o(i.nrf_drv_usbd_setup_stall) refers to nrf_drv_usbd.o(i.nrf_usbd_task_trigger) for nrf_usbd_task_trigger
    nrf_drv_usbd.o(i.nrf_drv_usbd_start) refers to nrf_drv_common.o(i.nrf_drv_common_irq_enable) for nrf_drv_common_irq_enable
    nrf_drv_usbd.o(i.nrf_drv_usbd_stop) refers to nrf_drv_usbd.o(i.usbd_ep_abort_all) for usbd_ep_abort_all
    nrf_drv_usbd.o(i.nrf_drv_usbd_transfer_out_drop) refers to nrf_drv_usbd.o(i.ep2bit) for ep2bit
    nrf_drv_usbd.o(i.nrf_drv_usbd_transfer_out_drop) refers to nrf_drv_usbd.o(i.nrf_drv_usbd_ep_transfer) for nrf_drv_usbd_ep_transfer
    nrf_drv_usbd.o(i.nrf_drv_usbd_transfer_out_drop) refers to nrf_drv_usbd.o(.data) for .data
    nrf_drv_usbd.o(i.nrf_drv_usbd_uninit) refers to nrf_drv_clock.o(i.nrf_drv_clock_hfclk_release) for nrf_drv_clock_hfclk_release
    nrf_drv_usbd.o(i.nrf_drv_usbd_uninit) refers to nrf_drv_usbd.o(.data) for .data
    nrf_drv_usbd.o(i.nrf_usbd_epin_dma_handler) refers to nrf_drv_usbd.o(i.ep_state_access) for ep_state_access
    nrf_drv_usbd.o(i.nrf_usbd_epin_dma_handler) refers to nrf_drv_usbd.o(i.ep2bit) for ep2bit
    nrf_drv_usbd.o(i.nrf_usbd_epin_dma_handler) refers to nrf_drv_usbd.o(i.nrf_atomic_u32_and) for nrf_atomic_u32_and
    nrf_drv_usbd.o(i.nrf_usbd_epin_dma_handler) refers to nrf_drv_usbd.o(.data) for .data
    nrf_drv_usbd.o(i.nrf_usbd_epout_dma_handler) refers to nrf_drv_usbd.o(i.ep_state_access) for ep_state_access
    nrf_drv_usbd.o(i.nrf_usbd_epout_dma_handler) refers to nrf_drv_usbd.o(i.ep2bit) for ep2bit
    nrf_drv_usbd.o(i.nrf_usbd_epout_dma_handler) refers to nrf_drv_usbd.o(i.nrf_atomic_u32_and) for nrf_atomic_u32_and
    nrf_drv_usbd.o(i.nrf_usbd_epout_dma_handler) refers to nrf_drv_usbd.o(i.usbd_dmareq_process) for usbd_dmareq_process
    nrf_drv_usbd.o(i.nrf_usbd_epout_dma_handler) refers to nrf_drv_usbd.o(.data) for .data
    nrf_drv_usbd.o(i.nrf_usbd_epout_dma_handler) refers to nrf_drv_usbd.o(.constdata) for .constdata
    nrf_drv_usbd.o(i.usbd_dmareq_process) refers to nrf_drv_usbd.o(i.bit2ep) for bit2ep
    nrf_drv_usbd.o(i.usbd_dmareq_process) refers to nrf_drv_usbd.o(i.ep_state_access) for ep_state_access
    nrf_drv_usbd.o(i.usbd_dmareq_process) refers to nrf_drv_usbd.o(i.nrf_drv_usbd_epout_size_get) for nrf_drv_usbd_epout_size_get
    nrf_drv_usbd.o(i.usbd_dmareq_process) refers to nrf_drv_usbd.o(i.nrf_atomic_u32_and) for nrf_atomic_u32_and
    nrf_drv_usbd.o(i.usbd_dmareq_process) refers to nrf_drv_usbd.o(i.nrf_usbd_event_clear) for nrf_usbd_event_clear
    nrf_drv_usbd.o(i.usbd_dmareq_process) refers to nrf_drv_usbd.o(i.nrf_usbd_task_trigger) for nrf_usbd_task_trigger
    nrf_drv_usbd.o(i.usbd_dmareq_process) refers to nrf_drv_systick.o(i.nrf_drv_systick_delay_us) for nrf_drv_systick_delay_us
    nrf_drv_usbd.o(i.usbd_dmareq_process) refers to nrf_drv_usbd.o(i.nrf_usbd_event_check) for nrf_usbd_event_check
    nrf_drv_usbd.o(i.usbd_dmareq_process) refers to nrf_drv_usbd.o(.data) for .data
    nrf_drv_usbd.o(i.usbd_dmareq_process) refers to nrf_drv_usbd.o(.constdata) for .constdata
    nrf_drv_usbd.o(i.usbd_drv_ep_abort) refers to nrf_drv_usbd.o(i.usbd_ep_abort) for usbd_ep_abort
    nrf_drv_usbd.o(i.usbd_ep_abort) refers to app_util_platform.o(i.app_util_critical_region_enter) for app_util_critical_region_enter
    nrf_drv_usbd.o(i.usbd_ep_abort) refers to nrf_drv_usbd.o(i.ep_state_access) for ep_state_access
    nrf_drv_usbd.o(i.usbd_ep_abort) refers to nrf_drv_usbd.o(i.ep2bit) for ep2bit
    nrf_drv_usbd.o(i.usbd_ep_abort) refers to nrf_drv_usbd.o(i.nrf_drv_usbd_transfer_out_drop) for nrf_drv_usbd_transfer_out_drop
    nrf_drv_usbd.o(i.usbd_ep_abort) refers to app_util_platform.o(i.app_util_critical_region_exit) for app_util_critical_region_exit
    nrf_drv_usbd.o(i.usbd_ep_abort) refers to nrf_drv_usbd.o(.data) for .data
    nrf_drv_usbd.o(i.usbd_ep_abort) refers to nrf_drv_usbd.o(.constdata) for .constdata
    nrf_drv_usbd.o(i.usbd_ep_abort_all) refers to nrf_drv_usbd.o(i.bit2ep) for bit2ep
    nrf_drv_usbd.o(i.usbd_ep_abort_all) refers to nrf_drv_usbd.o(i.usbd_ep_abort) for usbd_ep_abort
    nrf_drv_usbd.o(i.usbd_ep_abort_all) refers to nrf_drv_usbd.o(.data) for .data
    nrf_drv_usbd.o(i.usbd_ep_data_handler) refers to nrf_drv_usbd.o(.data) for .data
    nrf_drv_usbd.o(i.usbd_ep_data_handler) refers to nrf_drv_usbd.o(.constdata) for .constdata
    nrf_drv_usbd.o(.constdata) refers to nrf_drv_usbd.o(i.USBD_ISR_Usbreset) for USBD_ISR_Usbreset
    nrf_drv_usbd.o(.constdata) refers to nrf_drv_usbd.o(i.USBD_ISR_Started) for USBD_ISR_Started
    nrf_drv_usbd.o(.constdata) refers to nrf_drv_usbd.o(i.USBD_ISR_dma_epin0) for USBD_ISR_dma_epin0
    nrf_drv_usbd.o(.constdata) refers to nrf_drv_usbd.o(i.USBD_ISR_dma_epin1) for USBD_ISR_dma_epin1
    nrf_drv_usbd.o(.constdata) refers to nrf_drv_usbd.o(i.USBD_ISR_dma_epin2) for USBD_ISR_dma_epin2
    nrf_drv_usbd.o(.constdata) refers to nrf_drv_usbd.o(i.USBD_ISR_dma_epin3) for USBD_ISR_dma_epin3
    nrf_drv_usbd.o(.constdata) refers to nrf_drv_usbd.o(i.USBD_ISR_dma_epin4) for USBD_ISR_dma_epin4
    nrf_drv_usbd.o(.constdata) refers to nrf_drv_usbd.o(i.USBD_ISR_dma_epin5) for USBD_ISR_dma_epin5
    nrf_drv_usbd.o(.constdata) refers to nrf_drv_usbd.o(i.USBD_ISR_dma_epin6) for USBD_ISR_dma_epin6
    nrf_drv_usbd.o(.constdata) refers to nrf_drv_usbd.o(i.USBD_ISR_dma_epin7) for USBD_ISR_dma_epin7
    nrf_drv_usbd.o(.constdata) refers to nrf_drv_usbd.o(i.USBD_ISR_SetupData) for USBD_ISR_SetupData
    nrf_drv_usbd.o(.constdata) refers to nrf_drv_usbd.o(i.USBD_ISR_dma_epin8) for USBD_ISR_dma_epin8
    nrf_drv_usbd.o(.constdata) refers to nrf_drv_usbd.o(i.USBD_ISR_dma_epout0) for USBD_ISR_dma_epout0
    nrf_drv_usbd.o(.constdata) refers to nrf_drv_usbd.o(i.USBD_ISR_dma_epout1) for USBD_ISR_dma_epout1
    nrf_drv_usbd.o(.constdata) refers to nrf_drv_usbd.o(i.USBD_ISR_dma_epout2) for USBD_ISR_dma_epout2
    nrf_drv_usbd.o(.constdata) refers to nrf_drv_usbd.o(i.USBD_ISR_dma_epout3) for USBD_ISR_dma_epout3
    nrf_drv_usbd.o(.constdata) refers to nrf_drv_usbd.o(i.USBD_ISR_dma_epout4) for USBD_ISR_dma_epout4
    nrf_drv_usbd.o(.constdata) refers to nrf_drv_usbd.o(i.USBD_ISR_dma_epout5) for USBD_ISR_dma_epout5
    nrf_drv_usbd.o(.constdata) refers to nrf_drv_usbd.o(i.USBD_ISR_dma_epout6) for USBD_ISR_dma_epout6
    nrf_drv_usbd.o(.constdata) refers to nrf_drv_usbd.o(i.USBD_ISR_dma_epout7) for USBD_ISR_dma_epout7
    nrf_drv_usbd.o(.constdata) refers to nrf_drv_usbd.o(i.USBD_ISR_dma_epout8) for USBD_ISR_dma_epout8
    nrf_drv_usbd.o(.constdata) refers to nrf_drv_usbd.o(i.USBD_ISR_Sof) for USBD_ISR_Sof
    nrf_drv_usbd.o(.constdata) refers to nrf_drv_usbd.o(i.USBD_ISR_Event) for USBD_ISR_Event
    nrf_drv_usbd.o(.constdata) refers to nrf_drv_usbd.o(i.USBD_ISR_Setup) for USBD_ISR_Setup
    nrf_drv_usbd.o(.constdata) refers to nrf_drv_usbd.o(i.USBD_ISR_EpDataStatus) for USBD_ISR_EpDataStatus
    nrf_drv_usbd.o(.constdata) refers to nrf_drv_usbd.o(i.USBD_ISR_AccessFault) for USBD_ISR_AccessFault
    nrf_nvic.o(i.sd_nvic_critical_region_enter) refers to nrf_nvic.o(.data) for .data
    nrf_nvic.o(i.sd_nvic_critical_region_exit) refers to nrf_nvic.o(.data) for .data
    app_button.o(i.app_button_disable) refers to nrf_drv_gpiote.o(i.nrf_drv_gpiote_in_event_disable) for nrf_drv_gpiote_in_event_disable
    app_button.o(i.app_button_disable) refers to app_timer.o(i.app_timer_stop) for app_timer_stop
    app_button.o(i.app_button_disable) refers to app_button.o(.data) for .data
    app_button.o(i.app_button_disable) refers to app_button.o(.constdata) for .constdata
    app_button.o(i.app_button_enable) refers to nrf_drv_gpiote.o(i.nrf_drv_gpiote_in_event_enable) for nrf_drv_gpiote_in_event_enable
    app_button.o(i.app_button_enable) refers to app_button.o(.data) for .data
    app_button.o(i.app_button_init) refers to nrf_drv_gpiote.o(i.nrf_drv_gpiote_is_init) for nrf_drv_gpiote_is_init
    app_button.o(i.app_button_init) refers to nrf_drv_gpiote.o(i.nrf_drv_gpiote_init) for nrf_drv_gpiote_init
    app_button.o(i.app_button_init) refers to nrf_drv_gpiote.o(i.nrf_drv_gpiote_in_init) for nrf_drv_gpiote_in_init
    app_button.o(i.app_button_init) refers to app_timer.o(i.app_timer_create) for app_timer_create
    app_button.o(i.app_button_init) refers to app_button.o(.data) for .data
    app_button.o(i.app_button_init) refers to app_button.o(.constdata) for .constdata
    app_button.o(i.app_button_init) refers to app_button.o(i.gpiote_event_handler) for gpiote_event_handler
    app_button.o(i.app_button_init) refers to app_button.o(i.detection_delay_timeout_handler) for detection_delay_timeout_handler
    app_button.o(i.app_button_is_pushed) refers to nrf_drv_gpiote.o(i.nrf_drv_gpiote_in_is_set) for nrf_drv_gpiote_in_is_set
    app_button.o(i.app_button_is_pushed) refers to app_button.o(.data) for .data
    app_button.o(i.detection_delay_timeout_handler) refers to nrf_drv_gpiote.o(i.nrf_drv_gpiote_in_is_set) for nrf_drv_gpiote_in_is_set
    app_button.o(i.detection_delay_timeout_handler) refers to app_button.o(.data) for .data
    app_button.o(i.gpiote_event_handler) refers to app_timer.o(i.app_timer_stop) for app_timer_stop
    app_button.o(i.gpiote_event_handler) refers to nrf_drv_gpiote.o(i.nrf_drv_gpiote_in_is_set) for nrf_drv_gpiote_in_is_set
    app_button.o(i.gpiote_event_handler) refers to app_timer.o(i.app_timer_start) for app_timer_start
    app_button.o(i.gpiote_event_handler) refers to app_button.o(.constdata) for .constdata
    app_button.o(i.gpiote_event_handler) refers to app_button.o(.data) for .data
    app_button.o(.constdata) refers to app_button.o(.bss) for m_detection_delay_timer_id_data
    app_error.o(i.app_error_handler) refers to app_error_weak.o(i.app_error_fault_handler) for app_error_fault_handler
    app_error.o(i.app_error_handler_bare) refers to app_error_weak.o(i.app_error_fault_handler) for app_error_fault_handler
    app_error.o(i.app_error_save_and_stop) refers to app_error.o(.bss) for .bss
    app_error_weak.o(i.app_error_fault_handler) refers to nrf_log_frontend.o(i.nrf_log_frontend_std_0) for nrf_log_frontend_std_0
    app_error_weak.o(i.app_error_fault_handler) refers to nrf_log_frontend.o(i.nrf_log_blocking_backend_set) for nrf_log_blocking_backend_set
    app_error_weak.o(i.app_error_fault_handler) refers to nrf_log_frontend.o(i.nrf_log_frontend_dequeue) for nrf_log_frontend_dequeue
    app_fifo.o(i.app_fifo_get) refers to app_fifo.o(i.fifo_get) for fifo_get
    app_fifo.o(i.app_fifo_put) refers to app_fifo.o(i.fifo_put) for fifo_put
    app_fifo.o(i.app_fifo_read) refers to app_fifo.o(i.fifo_get) for fifo_get
    app_fifo.o(i.app_fifo_write) refers to app_fifo.o(i.fifo_put) for fifo_put
    app_scheduler.o(i.app_sched_event_put) refers to app_util_platform.o(i.app_util_critical_region_enter) for app_util_critical_region_enter
    app_scheduler.o(i.app_sched_event_put) refers to app_util_platform.o(i.app_util_critical_region_exit) for app_util_critical_region_exit
    app_scheduler.o(i.app_sched_event_put) refers to memcpya.o(.text) for __aeabi_memcpy
    app_scheduler.o(i.app_sched_event_put) refers to app_scheduler.o(.data) for .data
    app_scheduler.o(i.app_sched_execute) refers to app_scheduler.o(.data) for .data
    app_scheduler.o(i.app_sched_init) refers to app_scheduler.o(.data) for .data
    app_scheduler.o(i.app_sched_queue_space_get) refers to app_scheduler.o(.data) for .data
    app_timer.o(i.RTC1_IRQHandler) refers to app_timer.o(i.timer_timeouts_check) for timer_timeouts_check
    app_timer.o(i.SWI0_EGU0_IRQHandler) refers to app_timer.o(i.timer_list_handler) for timer_list_handler
    app_timer.o(i.app_timer_create) refers to app_timer.o(.bss) for .bss
    app_timer.o(i.app_timer_init) refers to app_timer.o(i.rtc1_stop) for rtc1_stop
    app_timer.o(i.app_timer_init) refers to app_timer.o(i.NVIC_ClearPendingIRQ) for NVIC_ClearPendingIRQ
    app_timer.o(i.app_timer_init) refers to app_timer.o(i.NVIC_SetPriority) for NVIC_SetPriority
    app_timer.o(i.app_timer_init) refers to app_timer.o(i.NVIC_EnableIRQ) for NVIC_EnableIRQ
    app_timer.o(i.app_timer_init) refers to app_timer.o(.bss) for .bss
    app_timer.o(i.app_timer_init) refers to app_timer.o(.data) for .data
    app_timer.o(i.app_timer_start) refers to app_util_platform.o(i.app_util_critical_region_enter) for app_util_critical_region_enter
    app_timer.o(i.app_timer_start) refers to app_timer.o(i.user_op_alloc) for user_op_alloc
    app_timer.o(i.app_timer_start) refers to app_util_platform.o(i.app_util_critical_region_exit) for app_util_critical_region_exit
    app_timer.o(i.app_timer_start) refers to app_timer.o(i.NVIC_SetPendingIRQ) for NVIC_SetPendingIRQ
    app_timer.o(i.app_timer_start) refers to app_timer.o(.bss) for .bss
    app_timer.o(i.app_timer_stop) refers to app_timer.o(i.timer_stop_op_schedule) for timer_stop_op_schedule
    app_timer.o(i.app_timer_stop) refers to app_timer.o(.bss) for .bss
    app_timer.o(i.app_timer_stop_all) refers to app_timer.o(i.timer_stop_op_schedule) for timer_stop_op_schedule
    app_timer.o(i.app_timer_stop_all) refers to app_timer.o(.bss) for .bss
    app_timer.o(i.compare_reg_update) refers to app_timer.o(i.NVIC_ClearPendingIRQ) for NVIC_ClearPendingIRQ
    app_timer.o(i.compare_reg_update) refers to app_timer.o(i.NVIC_EnableIRQ) for NVIC_EnableIRQ
    app_timer.o(i.compare_reg_update) refers to app_timer.o(i.nrf_delay_us) for nrf_delay_us
    app_timer.o(i.compare_reg_update) refers to app_timer.o(i.NVIC_SetPendingIRQ) for NVIC_SetPendingIRQ
    app_timer.o(i.compare_reg_update) refers to app_timer.o(i.rtc1_stop) for rtc1_stop
    app_timer.o(i.compare_reg_update) refers to app_timer.o(.data) for .data
    app_timer.o(i.elapsed_ticks_acquire) refers to app_timer.o(.data) for .data
    app_timer.o(i.list_insertions_handler) refers to app_timer.o(i.timer_list_remove) for timer_list_remove
    app_timer.o(i.list_insertions_handler) refers to app_timer.o(i.timer_list_insert) for timer_list_insert
    app_timer.o(i.list_insertions_handler) refers to app_timer.o(.data) for .data
    app_timer.o(i.list_insertions_handler) refers to app_timer.o(.bss) for .bss
    app_timer.o(i.nrf_delay_us) refers to system_nrf52840.o(.data) for SystemCoreClock
    app_timer.o(i.rtc1_stop) refers to app_timer.o(i.nrf_delay_us) for nrf_delay_us
    app_timer.o(i.rtc1_stop) refers to app_timer.o(.data) for .data
    app_timer.o(i.timer_list_handler) refers to app_timer.o(i.elapsed_ticks_acquire) for elapsed_ticks_acquire
    app_timer.o(i.timer_list_handler) refers to app_timer.o(i.list_insertions_handler) for list_insertions_handler
    app_timer.o(i.timer_list_handler) refers to app_timer.o(i.compare_reg_update) for compare_reg_update
    app_timer.o(i.timer_list_handler) refers to app_timer.o(.data) for .data
    app_timer.o(i.timer_list_insert) refers to app_timer.o(.data) for .data
    app_timer.o(i.timer_list_remove) refers to app_timer.o(i.nrf_delay_us) for nrf_delay_us
    app_timer.o(i.timer_list_remove) refers to app_timer.o(.data) for .data
    app_timer.o(i.timer_stop_op_schedule) refers to app_util_platform.o(i.app_util_critical_region_enter) for app_util_critical_region_enter
    app_timer.o(i.timer_stop_op_schedule) refers to app_timer.o(i.user_op_alloc) for user_op_alloc
    app_timer.o(i.timer_stop_op_schedule) refers to app_util_platform.o(i.app_util_critical_region_exit) for app_util_critical_region_exit
    app_timer.o(i.timer_stop_op_schedule) refers to app_timer.o(i.NVIC_SetPendingIRQ) for NVIC_SetPendingIRQ
    app_timer.o(i.timer_stop_op_schedule) refers to app_timer.o(.bss) for .bss
    app_timer.o(i.timer_timeouts_check) refers to app_timer.o(i.NVIC_SetPendingIRQ) for NVIC_SetPendingIRQ
    app_timer.o(i.timer_timeouts_check) refers to app_timer.o(.data) for .data
    app_timer.o(i.user_op_alloc) refers to app_timer.o(.bss) for .bss
    app_uart_fifo.o(i.app_uart_close) refers to nrf_drv_uart.o(i.nrf_drv_uart_uninit) for nrf_drv_uart_uninit
    app_uart_fifo.o(i.app_uart_close) refers to app_uart_fifo.o(.data) for .data
    app_uart_fifo.o(i.app_uart_flush) refers to app_fifo.o(i.app_fifo_flush) for app_fifo_flush
    app_uart_fifo.o(i.app_uart_flush) refers to app_uart_fifo.o(.bss) for .bss
    app_uart_fifo.o(i.app_uart_get) refers to app_fifo.o(i.app_fifo_get) for app_fifo_get
    app_uart_fifo.o(i.app_uart_get) refers to nrf_drv_uart.o(i.nrf_drv_uart_rx) for nrf_drv_uart_rx
    app_uart_fifo.o(i.app_uart_get) refers to app_error.o(i.app_error_handler_bare) for app_error_handler_bare
    app_uart_fifo.o(i.app_uart_get) refers to app_uart_fifo.o(.data) for .data
    app_uart_fifo.o(i.app_uart_get) refers to app_uart_fifo.o(.bss) for .bss
    app_uart_fifo.o(i.app_uart_init) refers to app_fifo.o(i.app_fifo_init) for app_fifo_init
    app_uart_fifo.o(i.app_uart_init) refers to memcpya.o(.text) for __aeabi_memcpy4
    app_uart_fifo.o(i.app_uart_init) refers to nrf_drv_uart.o(i.nrf_drv_uart_init) for nrf_drv_uart_init
    app_uart_fifo.o(i.app_uart_init) refers to nrf_drv_uart.o(i.nrf_drv_uart_rx_enable) for nrf_drv_uart_rx_enable
    app_uart_fifo.o(i.app_uart_init) refers to nrf_drv_uart.o(i.nrf_drv_uart_rx) for nrf_drv_uart_rx
    app_uart_fifo.o(i.app_uart_init) refers to app_uart_fifo.o(.data) for .data
    app_uart_fifo.o(i.app_uart_init) refers to app_uart_fifo.o(.bss) for .bss
    app_uart_fifo.o(i.app_uart_init) refers to app_uart_fifo.o(.constdata) for .constdata
    app_uart_fifo.o(i.app_uart_init) refers to app_uart_fifo.o(i.uart_event_handler) for uart_event_handler
    app_uart_fifo.o(i.app_uart_put) refers to app_fifo.o(i.app_fifo_put) for app_fifo_put
    app_uart_fifo.o(i.app_uart_put) refers to nrf_drv_uart.o(i.nrf_drv_uart_tx_in_progress) for nrf_drv_uart_tx_in_progress
    app_uart_fifo.o(i.app_uart_put) refers to app_fifo.o(i.app_fifo_get) for app_fifo_get
    app_uart_fifo.o(i.app_uart_put) refers to nrf_drv_uart.o(i.nrf_drv_uart_tx) for nrf_drv_uart_tx
    app_uart_fifo.o(i.app_uart_put) refers to app_uart_fifo.o(.bss) for .bss
    app_uart_fifo.o(i.app_uart_put) refers to app_uart_fifo.o(.data) for .data
    app_uart_fifo.o(i.uart_event_handler) refers to nrf_drv_uart.o(i.nrf_drv_uart_rx) for nrf_drv_uart_rx
    app_uart_fifo.o(i.uart_event_handler) refers to app_fifo.o(i.app_fifo_put) for app_fifo_put
    app_uart_fifo.o(i.uart_event_handler) refers to app_fifo.o(i.app_fifo_get) for app_fifo_get
    app_uart_fifo.o(i.uart_event_handler) refers to nrf_drv_uart.o(i.nrf_drv_uart_tx) for nrf_drv_uart_tx
    app_uart_fifo.o(i.uart_event_handler) refers to app_uart_fifo.o(.data) for .data
    app_uart_fifo.o(i.uart_event_handler) refers to app_uart_fifo.o(.bss) for .bss
    app_usbd_cdc_acm.o(i.app_usbd_cdc_acm_line_state_get) refers to app_util_platform.o(i.app_util_critical_region_enter) for app_util_critical_region_enter
    app_usbd_cdc_acm.o(i.app_usbd_cdc_acm_line_state_get) refers to app_util_platform.o(i.app_util_critical_region_exit) for app_util_critical_region_exit
    app_usbd_cdc_acm.o(i.app_usbd_cdc_acm_read) refers to app_usbd_cdc_acm.o(i.data_ep_out_addr_get) for data_ep_out_addr_get
    app_usbd_cdc_acm.o(i.app_usbd_cdc_acm_read) refers to app_usbd_core.o(i.app_usbd_core_ep_transfer) for app_usbd_core_ep_transfer
    app_usbd_cdc_acm.o(i.app_usbd_cdc_acm_rx_size) refers to app_usbd_cdc_acm.o(i.data_ep_out_addr_get) for data_ep_out_addr_get
    app_usbd_cdc_acm.o(i.app_usbd_cdc_acm_rx_size) refers to nrf_drv_usbd.o(i.nrf_drv_usbd_ep_status_get) for nrf_drv_usbd_ep_status_get
    app_usbd_cdc_acm.o(i.app_usbd_cdc_acm_serial_state_notify) refers to app_util_platform.o(i.app_util_critical_region_enter) for app_util_critical_region_enter
    app_usbd_cdc_acm.o(i.app_usbd_cdc_acm_serial_state_notify) refers to app_util_platform.o(i.app_util_critical_region_exit) for app_util_critical_region_exit
    app_usbd_cdc_acm.o(i.app_usbd_cdc_acm_serial_state_notify) refers to app_usbd_cdc_acm.o(i.comm_ep_in_addr_get) for comm_ep_in_addr_get
    app_usbd_cdc_acm.o(i.app_usbd_cdc_acm_serial_state_notify) refers to app_usbd_core.o(i.app_usbd_core_ep_transfer) for app_usbd_core_ep_transfer
    app_usbd_cdc_acm.o(i.app_usbd_cdc_acm_serial_state_notify) refers to app_usbd_cdc_acm.o(.constdata) for .constdata
    app_usbd_cdc_acm.o(i.app_usbd_cdc_acm_write) refers to app_usbd_cdc_acm.o(i.data_ep_in_addr_get) for data_ep_in_addr_get
    app_usbd_cdc_acm.o(i.app_usbd_cdc_acm_write) refers to app_usbd_core.o(i.app_usbd_core_ep_transfer) for app_usbd_core_ep_transfer
    app_usbd_cdc_acm.o(i.cdc_acm_event_handler) refers to app_usbd_cdc_acm.o(i.setup_event_handler) for setup_event_handler
    app_usbd_cdc_acm.o(i.cdc_acm_event_handler) refers to app_usbd_cdc_acm.o(i.comm_ep_in_addr_get) for comm_ep_in_addr_get
    app_usbd_cdc_acm.o(i.cdc_acm_event_handler) refers to app_usbd_cdc_acm.o(i.user_event_handler) for user_event_handler
    app_usbd_cdc_acm.o(i.cdc_acm_event_handler) refers to app_usbd.o(i.app_usbd_class_sof_register) for app_usbd_class_sof_register
    app_usbd_cdc_acm.o(i.cdc_acm_event_handler) refers to app_usbd.o(i.app_usbd_class_sof_unregister) for app_usbd_class_sof_unregister
    app_usbd_cdc_acm.o(i.comm_ep_in_addr_get) refers to app_usbd_cdc_acm.o(i.app_usbd_class_iface_get) for app_usbd_class_iface_get
    app_usbd_cdc_acm.o(i.comm_ep_in_addr_get) refers to app_usbd_cdc_acm.o(i.app_usbd_class_iface_ep_get) for app_usbd_class_iface_ep_get
    app_usbd_cdc_acm.o(i.data_ep_in_addr_get) refers to app_usbd_cdc_acm.o(i.app_usbd_class_iface_get) for app_usbd_class_iface_get
    app_usbd_cdc_acm.o(i.data_ep_in_addr_get) refers to app_usbd_cdc_acm.o(i.app_usbd_class_iface_ep_get) for app_usbd_class_iface_ep_get
    app_usbd_cdc_acm.o(i.data_ep_out_addr_get) refers to app_usbd_cdc_acm.o(i.app_usbd_class_iface_get) for app_usbd_class_iface_get
    app_usbd_cdc_acm.o(i.data_ep_out_addr_get) refers to app_usbd_cdc_acm.o(i.app_usbd_class_iface_ep_get) for app_usbd_class_iface_ep_get
    app_usbd_cdc_acm.o(i.setup_event_handler) refers to app_usbd.o(i.app_usbd_class_descriptor_find) for app_usbd_class_descriptor_find
    app_usbd_cdc_acm.o(i.setup_event_handler) refers to app_usbd_core.o(i.app_usbd_core_setup_transfer_buff_get) for app_usbd_core_setup_transfer_buff_get
    app_usbd_cdc_acm.o(i.setup_event_handler) refers to app_usbd_core.o(i.app_usbd_core_setup_rsp) for app_usbd_core_setup_rsp
    app_usbd_cdc_acm.o(i.setup_event_handler) refers to app_usbd_cdc_acm.o(i.setup_req_class_out) for setup_req_class_out
    app_usbd_cdc_acm.o(i.setup_req_class_out) refers to app_util_platform.o(i.app_util_critical_region_enter) for app_util_critical_region_enter
    app_usbd_cdc_acm.o(i.setup_req_class_out) refers to app_usbd_core.o(i.app_usbd_core_setup_data_transfer) for app_usbd_core_setup_data_transfer
    app_usbd_cdc_acm.o(i.setup_req_class_out) refers to app_usbd_core.o(i.app_usbd_core_setup_data_handler_set) for app_usbd_core_setup_data_handler_set
    app_usbd_cdc_acm.o(i.setup_req_class_out) refers to app_util_platform.o(i.app_util_critical_region_exit) for app_util_critical_region_exit
    app_usbd_cdc_acm.o(i.setup_req_class_out) refers to app_usbd_cdc_acm.o(i.user_event_handler) for user_event_handler
    app_usbd_cdc_acm.o(i.setup_req_class_out) refers to app_usbd_cdc_acm.o(i.data_ep_in_addr_get) for data_ep_in_addr_get
    app_usbd_cdc_acm.o(i.setup_req_class_out) refers to nrf_drv_usbd.o(i.usbd_drv_ep_abort) for usbd_drv_ep_abort
    app_usbd_cdc_acm.o(i.setup_req_class_out) refers to app_usbd_cdc_acm.o(i.data_ep_out_addr_get) for data_ep_out_addr_get
    app_usbd_cdc_acm.o(i.setup_req_class_out) refers to app_usbd_cdc_acm.o(.constdata) for .constdata
    app_usbd_cdc_acm.o(.constdata) refers to app_usbd_cdc_acm.o(i.cdc_acm_event_handler) for cdc_acm_event_handler
    app_usbd_cdc_acm.o(.constdata) refers to app_usbd_cdc_acm.o(i.cdc_acm_get_descriptors) for cdc_acm_get_descriptors
    app_usbd_cdc_acm.o(.constdata) refers to app_usbd_cdc_acm.o(i.cdc_acm_req_out_data_cb) for cdc_acm_req_out_data_cb
    app_util_platform.o(i.app_util_critical_region_enter) refers to app_util_platform.o(i.app_util_disable_irq) for app_util_disable_irq
    app_util_platform.o(i.app_util_critical_region_exit) refers to app_util_platform.o(i.app_util_enable_irq) for app_util_enable_irq
    app_util_platform.o(i.app_util_disable_irq) refers to app_util_platform.o(.data) for .data
    app_util_platform.o(i.app_util_enable_irq) refers to app_util_platform.o(.data) for .data
    hardfault_handler_keil.o(.emb_text) refers to hardfault_implementation.o(i.HardFault_c_handler) for HardFault_c_handler
    hardfault_implementation.o(i.HardFault_c_handler) refers to nrf_log_frontend.o(i.nrf_log_frontend_std_1) for nrf_log_frontend_std_1
    hardfault_implementation.o(i.HardFault_c_handler) refers to nrf_log_frontend.o(i.nrf_log_blocking_backend_set) for nrf_log_blocking_backend_set
    hardfault_implementation.o(i.HardFault_c_handler) refers to nrf_log_frontend.o(i.nrf_log_frontend_dequeue) for nrf_log_frontend_dequeue
    hardfault_implementation.o(i.HardFault_c_handler) refers to hardfault_implementation.o(i.HardFault_process) for HardFault_process
    nrf_assert.o(i.assert_nrf_callback) refers to app_error_weak.o(i.app_error_fault_handler) for app_error_fault_handler
    nrf_strerror.o(i.nrf_strerror_find) refers to nrf_strerror.o(.constdata) for .constdata
    nrf_strerror.o(i.nrf_strerror_get) refers to nrf_strerror.o(i.nrf_strerror_find) for nrf_strerror_find
    nrf_strerror.o(i.nrf_strerror_get) refers to nrf_strerror.o(.constdata) for .constdata
    nrf_strerror.o(.constdata) refers to nrf_strerror.o(.conststring) for .conststring
    nrf_log_backend_serial.o(i.nrf_log_backend_getchar) refers to nrf_drv_uart.o(i.nrf_drv_uart_rx) for nrf_drv_uart_rx
    nrf_log_backend_serial.o(i.nrf_log_backend_getchar) refers to nrf_log_backend_serial.o(.data) for .data
    nrf_log_backend_serial.o(i.nrf_log_backend_hexdump_handler_get) refers to nrf_log_backend_serial.o(i.nrf_log_backend_serial_hexdump_handler) for nrf_log_backend_serial_hexdump_handler
    nrf_log_backend_serial.o(i.nrf_log_backend_init) refers to memcpya.o(.text) for __aeabi_memcpy4
    nrf_log_backend_serial.o(i.nrf_log_backend_init) refers to nrf_drv_uart.o(i.nrf_drv_uart_uninit) for nrf_drv_uart_uninit
    nrf_log_backend_serial.o(i.nrf_log_backend_init) refers to nrf_drv_uart.o(i.nrf_drv_uart_init) for nrf_drv_uart_init
    nrf_log_backend_serial.o(i.nrf_log_backend_init) refers to nrf_log_backend_serial.o(.data) for .data
    nrf_log_backend_serial.o(i.nrf_log_backend_init) refers to nrf_log_backend_serial.o(.constdata) for .constdata
    nrf_log_backend_serial.o(i.nrf_log_backend_init) refers to nrf_log_backend_serial.o(i.uart_event_handler) for uart_event_handler
    nrf_log_backend_serial.o(i.nrf_log_backend_serial_hexdump_handler) refers to nrf_log_backend_serial.o(i.serial_is_busy) for serial_is_busy
    nrf_log_backend_serial.o(i.nrf_log_backend_serial_hexdump_handler) refers to nrf_log_backend_serial.o(i.timestamp_process) for timestamp_process
    nrf_log_backend_serial.o(i.nrf_log_backend_serial_hexdump_handler) refers to strlen.o(.text) for strlen
    nrf_log_backend_serial.o(i.nrf_log_backend_serial_hexdump_handler) refers to memcpya.o(.text) for __aeabi_memcpy
    nrf_log_backend_serial.o(i.nrf_log_backend_serial_hexdump_handler) refers to ctype_o.o(.text) for __rt_ctype_table
    nrf_log_backend_serial.o(i.nrf_log_backend_serial_hexdump_handler) refers to nrf_log_backend_serial.o(i.serial_tx) for serial_tx
    nrf_log_backend_serial.o(i.nrf_log_backend_serial_std_handler) refers to nrf_log_backend_serial.o(i.serial_is_busy) for serial_is_busy
    nrf_log_backend_serial.o(i.nrf_log_backend_serial_std_handler) refers to nrf_log_backend_serial.o(i.timestamp_process) for timestamp_process
    nrf_log_backend_serial.o(i.nrf_log_backend_serial_std_handler) refers to strlen.o(.text) for strlen
    nrf_log_backend_serial.o(i.nrf_log_backend_serial_std_handler) refers to memcpya.o(.text) for __aeabi_memcpy
    nrf_log_backend_serial.o(i.nrf_log_backend_serial_std_handler) refers to printf8.o(i.__0snprintf$8) for __2snprintf
    nrf_log_backend_serial.o(i.nrf_log_backend_serial_std_handler) refers to nrf_log_backend_serial.o(i.buf_len_update) for buf_len_update
    nrf_log_backend_serial.o(i.nrf_log_backend_serial_std_handler) refers to nrf_log_backend_serial.o(i.serial_tx) for serial_tx
    nrf_log_backend_serial.o(i.nrf_log_backend_std_handler_get) refers to nrf_log_backend_serial.o(i.nrf_log_backend_serial_std_handler) for nrf_log_backend_serial_std_handler
    nrf_log_backend_serial.o(i.serial_is_busy) refers to nrf_drv_uart.o(i.nrf_drv_uart_tx_in_progress) for nrf_drv_uart_tx_in_progress
    nrf_log_backend_serial.o(i.serial_is_busy) refers to nrf_log_backend_serial.o(.data) for .data
    nrf_log_backend_serial.o(i.serial_tx) refers to memcpya.o(.text) for __aeabi_memcpy
    nrf_log_backend_serial.o(i.serial_tx) refers to nrf_drv_uart.o(i.nrf_drv_uart_tx) for nrf_drv_uart_tx
    nrf_log_backend_serial.o(i.serial_tx) refers to nrf_log_backend_serial.o(.bss) for .bss
    nrf_log_backend_serial.o(i.serial_tx) refers to nrf_log_backend_serial.o(.data) for .data
    nrf_log_backend_serial.o(i.timestamp_process) refers to printf8.o(i.__0snprintf$8) for __2snprintf
    nrf_log_backend_serial.o(i.timestamp_process) refers to nrf_log_backend_serial.o(i.buf_len_update) for buf_len_update
    nrf_log_backend_serial.o(i.uart_event_handler) refers to nrf_log_backend_serial.o(.data) for .data
    nrf_log_frontend.o(i.buf_prealloc) refers to app_util_platform.o(i.app_util_critical_region_enter) for app_util_critical_region_enter
    nrf_log_frontend.o(i.buf_prealloc) refers to app_util_platform.o(i.app_util_critical_region_exit) for app_util_critical_region_exit
    nrf_log_frontend.o(i.buf_prealloc) refers to nrf_log_frontend.o(.bss) for .bss
    nrf_log_frontend.o(i.buf_prealloc) refers to nrf_log_frontend.o(.constdata) for .constdata
    nrf_log_frontend.o(i.buf_prealloc) refers to nrf_log_frontend.o(.data) for .data
    nrf_log_frontend.o(i.buffer_is_empty) refers to nrf_log_frontend.o(.bss) for .bss
    nrf_log_frontend.o(i.cont_buf_prealloc) refers to app_util_platform.o(i.app_util_critical_region_enter) for app_util_critical_region_enter
    nrf_log_frontend.o(i.cont_buf_prealloc) refers to app_util_platform.o(i.app_util_critical_region_exit) for app_util_critical_region_exit
    nrf_log_frontend.o(i.cont_buf_prealloc) refers to nrf_log_frontend.o(.bss) for .bss
    nrf_log_frontend.o(i.nrf_log_blocking_backend_set) refers to nrf_log_backend_serial.o(i.nrf_log_backend_init) for nrf_log_backend_init
    nrf_log_frontend.o(i.nrf_log_frontend_dequeue) refers to nrf_log_frontend.o(i.buffer_is_empty) for buffer_is_empty
    nrf_log_frontend.o(i.nrf_log_frontend_dequeue) refers to nrf_log_frontend.o(.bss) for .bss
    nrf_log_frontend.o(i.nrf_log_frontend_hexdump) refers to nrf_log_frontend.o(i.buf_prealloc) for buf_prealloc
    nrf_log_frontend.o(i.nrf_log_frontend_hexdump) refers to memcpya.o(.text) for __aeabi_memcpy
    nrf_log_frontend.o(i.nrf_log_frontend_hexdump) refers to nrf_log_frontend.o(.bss) for .bss
    nrf_log_frontend.o(i.nrf_log_frontend_hexdump) refers to nrf_log_frontend.o(.constdata) for .constdata
    nrf_log_frontend.o(i.nrf_log_frontend_init) refers to nrf_log_frontend.o(i.nrf_log_handlers_set) for nrf_log_handlers_set
    nrf_log_frontend.o(i.nrf_log_frontend_init) refers to nrf_log_frontend.o(.bss) for .bss
    nrf_log_frontend.o(i.nrf_log_frontend_std_0) refers to nrf_log_frontend.o(i.buf_prealloc) for buf_prealloc
    nrf_log_frontend.o(i.nrf_log_frontend_std_0) refers to nrf_log_frontend.o(.bss) for .bss
    nrf_log_frontend.o(i.nrf_log_frontend_std_0) refers to nrf_log_frontend.o(.constdata) for .constdata
    nrf_log_frontend.o(i.nrf_log_frontend_std_1) refers to nrf_log_frontend.o(i.buf_prealloc) for buf_prealloc
    nrf_log_frontend.o(i.nrf_log_frontend_std_1) refers to nrf_log_frontend.o(.bss) for .bss
    nrf_log_frontend.o(i.nrf_log_frontend_std_1) refers to nrf_log_frontend.o(.constdata) for .constdata
    nrf_log_frontend.o(i.nrf_log_frontend_std_2) refers to nrf_log_frontend.o(i.buf_prealloc) for buf_prealloc
    nrf_log_frontend.o(i.nrf_log_frontend_std_2) refers to nrf_log_frontend.o(.bss) for .bss
    nrf_log_frontend.o(i.nrf_log_frontend_std_2) refers to nrf_log_frontend.o(.constdata) for .constdata
    nrf_log_frontend.o(i.nrf_log_frontend_std_3) refers to nrf_log_frontend.o(i.buf_prealloc) for buf_prealloc
    nrf_log_frontend.o(i.nrf_log_frontend_std_3) refers to nrf_log_frontend.o(.bss) for .bss
    nrf_log_frontend.o(i.nrf_log_frontend_std_3) refers to nrf_log_frontend.o(.constdata) for .constdata
    nrf_log_frontend.o(i.nrf_log_frontend_std_4) refers to nrf_log_frontend.o(i.buf_prealloc) for buf_prealloc
    nrf_log_frontend.o(i.nrf_log_frontend_std_4) refers to nrf_log_frontend.o(.bss) for .bss
    nrf_log_frontend.o(i.nrf_log_frontend_std_4) refers to nrf_log_frontend.o(.constdata) for .constdata
    nrf_log_frontend.o(i.nrf_log_frontend_std_5) refers to nrf_log_frontend.o(i.buf_prealloc) for buf_prealloc
    nrf_log_frontend.o(i.nrf_log_frontend_std_5) refers to nrf_log_frontend.o(.bss) for .bss
    nrf_log_frontend.o(i.nrf_log_frontend_std_5) refers to nrf_log_frontend.o(.constdata) for .constdata
    nrf_log_frontend.o(i.nrf_log_frontend_std_6) refers to nrf_log_frontend.o(i.buf_prealloc) for buf_prealloc
    nrf_log_frontend.o(i.nrf_log_frontend_std_6) refers to nrf_log_frontend.o(.bss) for .bss
    nrf_log_frontend.o(i.nrf_log_frontend_std_6) refers to nrf_log_frontend.o(.constdata) for .constdata
    nrf_log_frontend.o(i.nrf_log_getchar) refers to nrf_log_backend_serial.o(i.nrf_log_backend_getchar) for nrf_log_backend_getchar
    nrf_log_frontend.o(i.nrf_log_handlers_set) refers to nrf_log_frontend.o(.bss) for .bss
    nrf_log_frontend.o(i.nrf_log_init) refers to nrf_log_backend_serial.o(i.nrf_log_backend_init) for nrf_log_backend_init
    nrf_log_frontend.o(i.nrf_log_init) refers to nrf_log_backend_serial.o(i.nrf_log_backend_hexdump_handler_get) for nrf_log_backend_hexdump_handler_get
    nrf_log_frontend.o(i.nrf_log_init) refers to nrf_log_backend_serial.o(i.nrf_log_backend_std_handler_get) for nrf_log_backend_std_handler_get
    nrf_log_frontend.o(i.nrf_log_init) refers to nrf_log_frontend.o(i.nrf_log_frontend_init) for nrf_log_frontend_init
    nrf_log_frontend.o(i.nrf_log_push) refers to strlen.o(.text) for strlen
    nrf_log_frontend.o(i.nrf_log_push) refers to nrf_log_frontend.o(i.cont_buf_prealloc) for cont_buf_prealloc
    nrf_log_frontend.o(i.nrf_log_push) refers to memcpya.o(.text) for __aeabi_memcpy
    nrf_log_frontend.o(i.nrf_log_push) refers to nrf_log_frontend.o(.bss) for .bss
    nrf_log_frontend.o(.data) refers to nrf_log_frontend.o(.conststring) for .conststring
    segger_rtt.o(i.SEGGER_RTT_ConfigDownBuffer) refers to segger_rtt.o(i._DoInit) for _DoInit
    segger_rtt.o(i.SEGGER_RTT_ConfigDownBuffer) refers to app_util_platform.o(i.app_util_critical_region_enter) for app_util_critical_region_enter
    segger_rtt.o(i.SEGGER_RTT_ConfigDownBuffer) refers to app_util_platform.o(i.app_util_critical_region_exit) for app_util_critical_region_exit
    segger_rtt.o(i.SEGGER_RTT_ConfigDownBuffer) refers to segger_rtt.o(.bss) for .bss
    segger_rtt.o(i.SEGGER_RTT_ConfigUpBuffer) refers to segger_rtt.o(i._DoInit) for _DoInit
    segger_rtt.o(i.SEGGER_RTT_ConfigUpBuffer) refers to app_util_platform.o(i.app_util_critical_region_enter) for app_util_critical_region_enter
    segger_rtt.o(i.SEGGER_RTT_ConfigUpBuffer) refers to app_util_platform.o(i.app_util_critical_region_exit) for app_util_critical_region_exit
    segger_rtt.o(i.SEGGER_RTT_ConfigUpBuffer) refers to segger_rtt.o(.bss) for .bss
    segger_rtt.o(i.SEGGER_RTT_GetKey) refers to segger_rtt.o(i.SEGGER_RTT_Read) for SEGGER_RTT_Read
    segger_rtt.o(i.SEGGER_RTT_HasData) refers to segger_rtt.o(.bss) for .bss
    segger_rtt.o(i.SEGGER_RTT_HasKey) refers to segger_rtt.o(i._DoInit) for _DoInit
    segger_rtt.o(i.SEGGER_RTT_HasKey) refers to segger_rtt.o(.bss) for .bss
    segger_rtt.o(i.SEGGER_RTT_Init) refers to segger_rtt.o(i._DoInit) for _DoInit
    segger_rtt.o(i.SEGGER_RTT_Init) refers to segger_rtt.o(.bss) for .bss
    segger_rtt.o(i.SEGGER_RTT_Read) refers to app_util_platform.o(i.app_util_critical_region_enter) for app_util_critical_region_enter
    segger_rtt.o(i.SEGGER_RTT_Read) refers to segger_rtt.o(i.SEGGER_RTT_ReadNoLock) for SEGGER_RTT_ReadNoLock
    segger_rtt.o(i.SEGGER_RTT_Read) refers to app_util_platform.o(i.app_util_critical_region_exit) for app_util_critical_region_exit
    segger_rtt.o(i.SEGGER_RTT_ReadNoLock) refers to segger_rtt.o(i._DoInit) for _DoInit
    segger_rtt.o(i.SEGGER_RTT_ReadNoLock) refers to memcpya.o(.text) for __aeabi_memcpy
    segger_rtt.o(i.SEGGER_RTT_ReadNoLock) refers to segger_rtt.o(.bss) for .bss
    segger_rtt.o(i.SEGGER_RTT_SetNameDownBuffer) refers to segger_rtt.o(i._DoInit) for _DoInit
    segger_rtt.o(i.SEGGER_RTT_SetNameDownBuffer) refers to app_util_platform.o(i.app_util_critical_region_enter) for app_util_critical_region_enter
    segger_rtt.o(i.SEGGER_RTT_SetNameDownBuffer) refers to app_util_platform.o(i.app_util_critical_region_exit) for app_util_critical_region_exit
    segger_rtt.o(i.SEGGER_RTT_SetNameDownBuffer) refers to segger_rtt.o(.bss) for .bss
    segger_rtt.o(i.SEGGER_RTT_SetNameUpBuffer) refers to segger_rtt.o(i._DoInit) for _DoInit
    segger_rtt.o(i.SEGGER_RTT_SetNameUpBuffer) refers to app_util_platform.o(i.app_util_critical_region_enter) for app_util_critical_region_enter
    segger_rtt.o(i.SEGGER_RTT_SetNameUpBuffer) refers to app_util_platform.o(i.app_util_critical_region_exit) for app_util_critical_region_exit
    segger_rtt.o(i.SEGGER_RTT_SetNameUpBuffer) refers to segger_rtt.o(.bss) for .bss
    segger_rtt.o(i.SEGGER_RTT_SetTerminal) refers to segger_rtt.o(i._DoInit) for _DoInit
    segger_rtt.o(i.SEGGER_RTT_SetTerminal) refers to app_util_platform.o(i.app_util_critical_region_enter) for app_util_critical_region_enter
    segger_rtt.o(i.SEGGER_RTT_SetTerminal) refers to segger_rtt.o(i._GetAvailWriteSpace) for _GetAvailWriteSpace
    segger_rtt.o(i.SEGGER_RTT_SetTerminal) refers to segger_rtt.o(i._WriteNoCheck) for _WriteNoCheck
    segger_rtt.o(i.SEGGER_RTT_SetTerminal) refers to segger_rtt.o(i._WriteBlocking) for _WriteBlocking
    segger_rtt.o(i.SEGGER_RTT_SetTerminal) refers to app_util_platform.o(i.app_util_critical_region_exit) for app_util_critical_region_exit
    segger_rtt.o(i.SEGGER_RTT_SetTerminal) refers to segger_rtt.o(.bss) for .bss
    segger_rtt.o(i.SEGGER_RTT_SetTerminal) refers to segger_rtt.o(.data) for .data
    segger_rtt.o(i.SEGGER_RTT_TerminalOut) refers to segger_rtt.o(i._DoInit) for _DoInit
    segger_rtt.o(i.SEGGER_RTT_TerminalOut) refers to strlen.o(.text) for strlen
    segger_rtt.o(i.SEGGER_RTT_TerminalOut) refers to app_util_platform.o(i.app_util_critical_region_enter) for app_util_critical_region_enter
    segger_rtt.o(i.SEGGER_RTT_TerminalOut) refers to segger_rtt.o(i._GetAvailWriteSpace) for _GetAvailWriteSpace
    segger_rtt.o(i.SEGGER_RTT_TerminalOut) refers to segger_rtt.o(i._PostTerminalSwitch) for _PostTerminalSwitch
    segger_rtt.o(i.SEGGER_RTT_TerminalOut) refers to segger_rtt.o(i._WriteBlocking) for _WriteBlocking
    segger_rtt.o(i.SEGGER_RTT_TerminalOut) refers to app_util_platform.o(i.app_util_critical_region_exit) for app_util_critical_region_exit
    segger_rtt.o(i.SEGGER_RTT_TerminalOut) refers to segger_rtt.o(.bss) for .bss
    segger_rtt.o(i.SEGGER_RTT_TerminalOut) refers to segger_rtt.o(.data) for .data
    segger_rtt.o(i.SEGGER_RTT_WaitKey) refers to segger_rtt.o(i.SEGGER_RTT_GetKey) for SEGGER_RTT_GetKey
    segger_rtt.o(i.SEGGER_RTT_Write) refers to segger_rtt.o(i._DoInit) for _DoInit
    segger_rtt.o(i.SEGGER_RTT_Write) refers to app_util_platform.o(i.app_util_critical_region_enter) for app_util_critical_region_enter
    segger_rtt.o(i.SEGGER_RTT_Write) refers to segger_rtt.o(i.SEGGER_RTT_WriteNoLock) for SEGGER_RTT_WriteNoLock
    segger_rtt.o(i.SEGGER_RTT_Write) refers to app_util_platform.o(i.app_util_critical_region_exit) for app_util_critical_region_exit
    segger_rtt.o(i.SEGGER_RTT_Write) refers to segger_rtt.o(.bss) for .bss
    segger_rtt.o(i.SEGGER_RTT_WriteNoLock) refers to segger_rtt.o(i._GetAvailWriteSpace) for _GetAvailWriteSpace
    segger_rtt.o(i.SEGGER_RTT_WriteNoLock) refers to segger_rtt.o(i._WriteNoCheck) for _WriteNoCheck
    segger_rtt.o(i.SEGGER_RTT_WriteNoLock) refers to segger_rtt.o(i._WriteBlocking) for _WriteBlocking
    segger_rtt.o(i.SEGGER_RTT_WriteNoLock) refers to segger_rtt.o(.bss) for .bss
    segger_rtt.o(i.SEGGER_RTT_WriteSkipNoLock) refers to memcpya.o(.text) for __aeabi_memcpy
    segger_rtt.o(i.SEGGER_RTT_WriteSkipNoLock) refers to segger_rtt.o(.bss) for .bss
    segger_rtt.o(i.SEGGER_RTT_WriteString) refers to strlen.o(.text) for strlen
    segger_rtt.o(i.SEGGER_RTT_WriteString) refers to segger_rtt.o(i.SEGGER_RTT_Write) for SEGGER_RTT_Write
    segger_rtt.o(i._DoInit) refers to strcpy.o(.text) for strcpy
    segger_rtt.o(i._DoInit) refers to segger_rtt.o(.bss) for .bss
    segger_rtt.o(i._PostTerminalSwitch) refers to segger_rtt.o(i._WriteBlocking) for _WriteBlocking
    segger_rtt.o(i._PostTerminalSwitch) refers to segger_rtt.o(.data) for .data
    segger_rtt.o(i._WriteBlocking) refers to memcpya.o(.text) for __aeabi_memcpy
    segger_rtt.o(i._WriteNoCheck) refers to memcpya.o(.text) for __aeabi_memcpy
    arm_startup_nrf52840.o(RESET) refers to arm_startup_nrf52840.o(STACK) for __initial_sp
    arm_startup_nrf52840.o(RESET) refers to arm_startup_nrf52840.o(.text) for Reset_Handler
    arm_startup_nrf52840.o(RESET) refers to hardfault_handler_keil.o(.emb_text) for HardFault_Handler
    arm_startup_nrf52840.o(RESET) refers to nrf_drv_common.o(i.POWER_CLOCK_IRQHandler) for POWER_CLOCK_IRQHandler
    arm_startup_nrf52840.o(RESET) refers to nrf_drv_uart.o(i.UARTE0_UART0_IRQHandler) for UARTE0_UART0_IRQHandler
    arm_startup_nrf52840.o(RESET) refers to nrf_drv_gpiote.o(i.GPIOTE_IRQHandler) for GPIOTE_IRQHandler
    arm_startup_nrf52840.o(RESET) refers to app_timer.o(i.RTC1_IRQHandler) for RTC1_IRQHandler
    arm_startup_nrf52840.o(RESET) refers to app_timer.o(i.SWI0_EGU0_IRQHandler) for SWI0_EGU0_IRQHandler
    arm_startup_nrf52840.o(RESET) refers to nrf_drv_usbd.o(i.USBD_IRQHandler) for USBD_IRQHandler
    arm_startup_nrf52840.o(.text) refers to system_nrf52840.o(i.SystemInit) for SystemInit
    arm_startup_nrf52840.o(.text) refers to entry.o(.ARM.Collect$$$$00000000) for __main
    system_nrf52840.o(i.SystemCoreClockUpdate) refers to system_nrf52840.o(.data) for .data
    system_nrf52840.o(i.SystemInit) refers to system_nrf52840.o(.data) for .data
    entry.o(.ARM.Collect$$$$00000000) refers (Special) to entry10a.o(.ARM.Collect$$$$0000000D) for __rt_final_cpp
    entry.o(.ARM.Collect$$$$00000000) refers (Special) to entry11a.o(.ARM.Collect$$$$0000000F) for __rt_final_exit
    entry.o(.ARM.Collect$$$$00000000) refers (Special) to entry7b.o(.ARM.Collect$$$$00000008) for _main_clock
    entry.o(.ARM.Collect$$$$00000000) refers (Special) to entry8b.o(.ARM.Collect$$$$0000000A) for _main_cpp_init
    entry.o(.ARM.Collect$$$$00000000) refers (Special) to entry9a.o(.ARM.Collect$$$$0000000B) for _main_init
    entry.o(.ARM.Collect$$$$00000000) refers (Special) to entry5.o(.ARM.Collect$$$$00000004) for _main_scatterload
    entry.o(.ARM.Collect$$$$00000000) refers (Special) to entry2.o(.ARM.Collect$$$$00000001) for _main_stk
    uldiv.o(.text) refers to llushr.o(.text) for __aeabi_llsr
    uldiv.o(.text) refers to llshl.o(.text) for __aeabi_llsl
    ctype_o.o(.text) refers to ctype_o.o(.constdata) for .constdata
    ctype_o.o(.constdata) refers to ctype_o.o(.constdata) for __ctype_table
    isalnum_o.o(.text) refers to ctype_o.o(.text) for __rt_ctype_table
    isalpha_o.o(.text) refers to ctype_o.o(.text) for __rt_ctype_table
    isblank_o.o(.text) refers to ctype_o.o(.constdata) for __ctype_table
    iscntrl_o.o(.text) refers to ctype_o.o(.text) for __rt_ctype_table
    isdigit_o.o(.text) refers to ctype_o.o(.text) for __rt_ctype_table
    isgraph_o.o(.text) refers to ctype_o.o(.text) for __rt_ctype_table
    islower_o.o(.text) refers to ctype_o.o(.text) for __rt_ctype_table
    isprint_o.o(.text) refers to ctype_o.o(.text) for __rt_ctype_table
    ispunct_o.o(.text) refers to ctype_o.o(.text) for __rt_ctype_table
    isspace_o.o(.text) refers to ctype_o.o(.text) for __rt_ctype_table
    isupper_o.o(.text) refers to ctype_o.o(.text) for __rt_ctype_table
    isxdigit_o.o(.text) refers to ctype_o.o(.text) for __rt_ctype_table
    printfb.o(i.__0fprintf$bare) refers to printfb.o(i._printf_core) for _printf_core
    printfb.o(i.__0fprintf$bare) refers to fputc.o(i.fputc) for fputc
    printfb.o(i.__0printf$bare) refers to printfb.o(i._printf_core) for _printf_core
    printfb.o(i.__0printf$bare) refers to fputc.o(i.fputc) for fputc
    printfb.o(i.__0printf$bare) refers to stdout.o(.data) for __stdout
    printfb.o(i.__0snprintf$bare) refers to printfb.o(i._printf_core) for _printf_core
    printfb.o(i.__0snprintf$bare) refers to printfb.o(i._snputc) for _snputc
    printfb.o(i.__0sprintf$bare) refers to printfb.o(i._printf_core) for _printf_core
    printfb.o(i.__0sprintf$bare) refers to printfb.o(i._sputc) for _sputc
    printfb.o(i.__0vfprintf$bare) refers to printfb.o(i._printf_core) for _printf_core
    printfb.o(i.__0vfprintf$bare) refers to fputc.o(i.fputc) for fputc
    printfb.o(i.__0vprintf$bare) refers to printfb.o(i._printf_core) for _printf_core
    printfb.o(i.__0vprintf$bare) refers to fputc.o(i.fputc) for fputc
    printfb.o(i.__0vprintf$bare) refers to stdout.o(.data) for __stdout
    printfb.o(i.__0vsnprintf$bare) refers to printfb.o(i._printf_core) for _printf_core
    printfb.o(i.__0vsnprintf$bare) refers to printfb.o(i._snputc) for _snputc
    printfb.o(i.__0vsprintf$bare) refers to printfb.o(i._printf_core) for _printf_core
    printfb.o(i.__0vsprintf$bare) refers to printfb.o(i._sputc) for _sputc
    printf0.o(i.__0fprintf$0) refers to printf0.o(i._printf_core) for _printf_core
    printf0.o(i.__0fprintf$0) refers to fputc.o(i.fputc) for fputc
    printf0.o(i.__0printf$0) refers to printf0.o(i._printf_core) for _printf_core
    printf0.o(i.__0printf$0) refers to fputc.o(i.fputc) for fputc
    printf0.o(i.__0printf$0) refers to stdout.o(.data) for __stdout
    printf0.o(i.__0snprintf$0) refers to printf0.o(i._printf_core) for _printf_core
    printf0.o(i.__0snprintf$0) refers to printf0.o(i._snputc) for _snputc
    printf0.o(i.__0sprintf$0) refers to printf0.o(i._printf_core) for _printf_core
    printf0.o(i.__0sprintf$0) refers to printf0.o(i._sputc) for _sputc
    printf0.o(i.__0vfprintf$0) refers to printf0.o(i._printf_core) for _printf_core
    printf0.o(i.__0vfprintf$0) refers to fputc.o(i.fputc) for fputc
    printf0.o(i.__0vprintf$0) refers to printf0.o(i._printf_core) for _printf_core
    printf0.o(i.__0vprintf$0) refers to fputc.o(i.fputc) for fputc
    printf0.o(i.__0vprintf$0) refers to stdout.o(.data) for __stdout
    printf0.o(i.__0vsnprintf$0) refers to printf0.o(i._printf_core) for _printf_core
    printf0.o(i.__0vsnprintf$0) refers to printf0.o(i._snputc) for _snputc
    printf0.o(i.__0vsprintf$0) refers to printf0.o(i._printf_core) for _printf_core
    printf0.o(i.__0vsprintf$0) refers to printf0.o(i._sputc) for _sputc
    printf1.o(i.__0fprintf$1) refers to printf1.o(i._printf_core) for _printf_core
    printf1.o(i.__0fprintf$1) refers to fputc.o(i.fputc) for fputc
    printf1.o(i.__0printf$1) refers to printf1.o(i._printf_core) for _printf_core
    printf1.o(i.__0printf$1) refers to fputc.o(i.fputc) for fputc
    printf1.o(i.__0printf$1) refers to stdout.o(.data) for __stdout
    printf1.o(i.__0snprintf$1) refers to printf1.o(i._printf_core) for _printf_core
    printf1.o(i.__0snprintf$1) refers to printf1.o(i._snputc) for _snputc
    printf1.o(i.__0sprintf$1) refers to printf1.o(i._printf_core) for _printf_core
    printf1.o(i.__0sprintf$1) refers to printf1.o(i._sputc) for _sputc
    printf1.o(i.__0vfprintf$1) refers to printf1.o(i._printf_core) for _printf_core
    printf1.o(i.__0vfprintf$1) refers to fputc.o(i.fputc) for fputc
    printf1.o(i.__0vprintf$1) refers to printf1.o(i._printf_core) for _printf_core
    printf1.o(i.__0vprintf$1) refers to fputc.o(i.fputc) for fputc
    printf1.o(i.__0vprintf$1) refers to stdout.o(.data) for __stdout
    printf1.o(i.__0vsnprintf$1) refers to printf1.o(i._printf_core) for _printf_core
    printf1.o(i.__0vsnprintf$1) refers to printf1.o(i._snputc) for _snputc
    printf1.o(i.__0vsprintf$1) refers to printf1.o(i._printf_core) for _printf_core
    printf1.o(i.__0vsprintf$1) refers to printf1.o(i._sputc) for _sputc
    printf1.o(i._printf_core) refers to uidiv.o(.text) for __aeabi_uidivmod
    printf2.o(i.__0fprintf$2) refers to printf2.o(i._printf_core) for _printf_core
    printf2.o(i.__0fprintf$2) refers to fputc.o(i.fputc) for fputc
    printf2.o(i.__0printf$2) refers to printf2.o(i._printf_core) for _printf_core
    printf2.o(i.__0printf$2) refers to fputc.o(i.fputc) for fputc
    printf2.o(i.__0printf$2) refers to stdout.o(.data) for __stdout
    printf2.o(i.__0snprintf$2) refers to printf2.o(i._printf_core) for _printf_core
    printf2.o(i.__0snprintf$2) refers to printf2.o(i._snputc) for _snputc
    printf2.o(i.__0sprintf$2) refers to printf2.o(i._printf_core) for _printf_core
    printf2.o(i.__0sprintf$2) refers to printf2.o(i._sputc) for _sputc
    printf2.o(i.__0vfprintf$2) refers to printf2.o(i._printf_core) for _printf_core
    printf2.o(i.__0vfprintf$2) refers to fputc.o(i.fputc) for fputc
    printf2.o(i.__0vprintf$2) refers to printf2.o(i._printf_core) for _printf_core
    printf2.o(i.__0vprintf$2) refers to fputc.o(i.fputc) for fputc
    printf2.o(i.__0vprintf$2) refers to stdout.o(.data) for __stdout
    printf2.o(i.__0vsnprintf$2) refers to printf2.o(i._printf_core) for _printf_core
    printf2.o(i.__0vsnprintf$2) refers to printf2.o(i._snputc) for _snputc
    printf2.o(i.__0vsprintf$2) refers to printf2.o(i._printf_core) for _printf_core
    printf2.o(i.__0vsprintf$2) refers to printf2.o(i._sputc) for _sputc
    printf3.o(i.__0fprintf$3) refers to printf3.o(i._printf_core) for _printf_core
    printf3.o(i.__0fprintf$3) refers to fputc.o(i.fputc) for fputc
    printf3.o(i.__0printf$3) refers to printf3.o(i._printf_core) for _printf_core
    printf3.o(i.__0printf$3) refers to fputc.o(i.fputc) for fputc
    printf3.o(i.__0printf$3) refers to stdout.o(.data) for __stdout
    printf3.o(i.__0snprintf$3) refers to printf3.o(i._printf_core) for _printf_core
    printf3.o(i.__0snprintf$3) refers to printf3.o(i._snputc) for _snputc
    printf3.o(i.__0sprintf$3) refers to printf3.o(i._printf_core) for _printf_core
    printf3.o(i.__0sprintf$3) refers to printf3.o(i._sputc) for _sputc
    printf3.o(i.__0vfprintf$3) refers to printf3.o(i._printf_core) for _printf_core
    printf3.o(i.__0vfprintf$3) refers to fputc.o(i.fputc) for fputc
    printf3.o(i.__0vprintf$3) refers to printf3.o(i._printf_core) for _printf_core
    printf3.o(i.__0vprintf$3) refers to fputc.o(i.fputc) for fputc
    printf3.o(i.__0vprintf$3) refers to stdout.o(.data) for __stdout
    printf3.o(i.__0vsnprintf$3) refers to printf3.o(i._printf_core) for _printf_core
    printf3.o(i.__0vsnprintf$3) refers to printf3.o(i._snputc) for _snputc
    printf3.o(i.__0vsprintf$3) refers to printf3.o(i._printf_core) for _printf_core
    printf3.o(i.__0vsprintf$3) refers to printf3.o(i._sputc) for _sputc
    printf3.o(i._printf_core) refers to uidiv.o(.text) for __aeabi_uidivmod
    printf4.o(i.__0fprintf$4) refers to printf4.o(i._printf_core) for _printf_core
    printf4.o(i.__0fprintf$4) refers to fputc.o(i.fputc) for fputc
    printf4.o(i.__0printf$4) refers to printf4.o(i._printf_core) for _printf_core
    printf4.o(i.__0printf$4) refers to fputc.o(i.fputc) for fputc
    printf4.o(i.__0printf$4) refers to stdout.o(.data) for __stdout
    printf4.o(i.__0snprintf$4) refers to printf4.o(i._printf_core) for _printf_core
    printf4.o(i.__0snprintf$4) refers to printf4.o(i._snputc) for _snputc
    printf4.o(i.__0sprintf$4) refers to printf4.o(i._printf_core) for _printf_core
    printf4.o(i.__0sprintf$4) refers to printf4.o(i._sputc) for _sputc
    printf4.o(i.__0vfprintf$4) refers to printf4.o(i._printf_core) for _printf_core
    printf4.o(i.__0vfprintf$4) refers to fputc.o(i.fputc) for fputc
    printf4.o(i.__0vprintf$4) refers to printf4.o(i._printf_core) for _printf_core
    printf4.o(i.__0vprintf$4) refers to fputc.o(i.fputc) for fputc
    printf4.o(i.__0vprintf$4) refers to stdout.o(.data) for __stdout
    printf4.o(i.__0vsnprintf$4) refers to printf4.o(i._printf_core) for _printf_core
    printf4.o(i.__0vsnprintf$4) refers to printf4.o(i._snputc) for _snputc
    printf4.o(i.__0vsprintf$4) refers to printf4.o(i._printf_core) for _printf_core
    printf4.o(i.__0vsprintf$4) refers to printf4.o(i._sputc) for _sputc
    printf4.o(i._printf_core) refers to uldiv.o(.text) for __aeabi_uldivmod
    printf5.o(i.__0fprintf$5) refers to printf5.o(i._printf_core) for _printf_core
    printf5.o(i.__0fprintf$5) refers to fputc.o(i.fputc) for fputc
    printf5.o(i.__0printf$5) refers to printf5.o(i._printf_core) for _printf_core
    printf5.o(i.__0printf$5) refers to fputc.o(i.fputc) for fputc
    printf5.o(i.__0printf$5) refers to stdout.o(.data) for __stdout
    printf5.o(i.__0snprintf$5) refers to printf5.o(i._printf_core) for _printf_core
    printf5.o(i.__0snprintf$5) refers to printf5.o(i._snputc) for _snputc
    printf5.o(i.__0sprintf$5) refers to printf5.o(i._printf_core) for _printf_core
    printf5.o(i.__0sprintf$5) refers to printf5.o(i._sputc) for _sputc
    printf5.o(i.__0vfprintf$5) refers to printf5.o(i._printf_core) for _printf_core
    printf5.o(i.__0vfprintf$5) refers to fputc.o(i.fputc) for fputc
    printf5.o(i.__0vprintf$5) refers to printf5.o(i._printf_core) for _printf_core
    printf5.o(i.__0vprintf$5) refers to fputc.o(i.fputc) for fputc
    printf5.o(i.__0vprintf$5) refers to stdout.o(.data) for __stdout
    printf5.o(i.__0vsnprintf$5) refers to printf5.o(i._printf_core) for _printf_core
    printf5.o(i.__0vsnprintf$5) refers to printf5.o(i._snputc) for _snputc
    printf5.o(i.__0vsprintf$5) refers to printf5.o(i._printf_core) for _printf_core
    printf5.o(i.__0vsprintf$5) refers to printf5.o(i._sputc) for _sputc
    printf5.o(i._printf_core) refers to uldiv.o(.text) for __aeabi_uldivmod
    printf6.o(i.__0fprintf$6) refers to printf6.o(i._printf_core) for _printf_core
    printf6.o(i.__0fprintf$6) refers to fputc.o(i.fputc) for fputc
    printf6.o(i.__0printf$6) refers to printf6.o(i._printf_core) for _printf_core
    printf6.o(i.__0printf$6) refers to fputc.o(i.fputc) for fputc
    printf6.o(i.__0printf$6) refers to stdout.o(.data) for __stdout
    printf6.o(i.__0snprintf$6) refers to printf6.o(i._printf_core) for _printf_core
    printf6.o(i.__0snprintf$6) refers to printf6.o(i._snputc) for _snputc
    printf6.o(i.__0sprintf$6) refers to printf6.o(i._printf_core) for _printf_core
    printf6.o(i.__0sprintf$6) refers to printf6.o(i._sputc) for _sputc
    printf6.o(i.__0vfprintf$6) refers to printf6.o(i._printf_core) for _printf_core
    printf6.o(i.__0vfprintf$6) refers to fputc.o(i.fputc) for fputc
    printf6.o(i.__0vprintf$6) refers to printf6.o(i._printf_core) for _printf_core
    printf6.o(i.__0vprintf$6) refers to fputc.o(i.fputc) for fputc
    printf6.o(i.__0vprintf$6) refers to stdout.o(.data) for __stdout
    printf6.o(i.__0vsnprintf$6) refers to printf6.o(i._printf_core) for _printf_core
    printf6.o(i.__0vsnprintf$6) refers to printf6.o(i._snputc) for _snputc
    printf6.o(i.__0vsprintf$6) refers to printf6.o(i._printf_core) for _printf_core
    printf6.o(i.__0vsprintf$6) refers to printf6.o(i._sputc) for _sputc
    printf6.o(i._printf_core) refers to printf6.o(i._printf_pre_padding) for _printf_pre_padding
    printf6.o(i._printf_core) refers to uidiv.o(.text) for __aeabi_uidivmod
    printf6.o(i._printf_core) refers to printf6.o(i._printf_post_padding) for _printf_post_padding
    printf7.o(i.__0fprintf$7) refers to printf7.o(i._printf_core) for _printf_core
    printf7.o(i.__0fprintf$7) refers to fputc.o(i.fputc) for fputc
    printf7.o(i.__0printf$7) refers to printf7.o(i._printf_core) for _printf_core
    printf7.o(i.__0printf$7) refers to fputc.o(i.fputc) for fputc
    printf7.o(i.__0printf$7) refers to stdout.o(.data) for __stdout
    printf7.o(i.__0snprintf$7) refers to printf7.o(i._printf_core) for _printf_core
    printf7.o(i.__0snprintf$7) refers to printf7.o(i._snputc) for _snputc
    printf7.o(i.__0sprintf$7) refers to printf7.o(i._printf_core) for _printf_core
    printf7.o(i.__0sprintf$7) refers to printf7.o(i._sputc) for _sputc
    printf7.o(i.__0vfprintf$7) refers to printf7.o(i._printf_core) for _printf_core
    printf7.o(i.__0vfprintf$7) refers to fputc.o(i.fputc) for fputc
    printf7.o(i.__0vprintf$7) refers to printf7.o(i._printf_core) for _printf_core
    printf7.o(i.__0vprintf$7) refers to fputc.o(i.fputc) for fputc
    printf7.o(i.__0vprintf$7) refers to stdout.o(.data) for __stdout
    printf7.o(i.__0vsnprintf$7) refers to printf7.o(i._printf_core) for _printf_core
    printf7.o(i.__0vsnprintf$7) refers to printf7.o(i._snputc) for _snputc
    printf7.o(i.__0vsprintf$7) refers to printf7.o(i._printf_core) for _printf_core
    printf7.o(i.__0vsprintf$7) refers to printf7.o(i._sputc) for _sputc
    printf7.o(i._printf_core) refers to printf7.o(i._printf_pre_padding) for _printf_pre_padding
    printf7.o(i._printf_core) refers to uldiv.o(.text) for __aeabi_uldivmod
    printf7.o(i._printf_core) refers to printf7.o(i._printf_post_padding) for _printf_post_padding
    printf8.o(i.__0fprintf$8) refers to printf8.o(i._printf_core) for _printf_core
    printf8.o(i.__0fprintf$8) refers to fputc.o(i.fputc) for fputc
    printf8.o(i.__0printf$8) refers to printf8.o(i._printf_core) for _printf_core
    printf8.o(i.__0printf$8) refers to fputc.o(i.fputc) for fputc
    printf8.o(i.__0printf$8) refers to stdout.o(.data) for __stdout
    printf8.o(i.__0snprintf$8) refers to printf8.o(i._printf_core) for _printf_core
    printf8.o(i.__0snprintf$8) refers to printf8.o(i._snputc) for _snputc
    printf8.o(i.__0sprintf$8) refers to printf8.o(i._printf_core) for _printf_core
    printf8.o(i.__0sprintf$8) refers to printf8.o(i._sputc) for _sputc
    printf8.o(i.__0vfprintf$8) refers to printf8.o(i._printf_core) for _printf_core
    printf8.o(i.__0vfprintf$8) refers to fputc.o(i.fputc) for fputc
    printf8.o(i.__0vprintf$8) refers to printf8.o(i._printf_core) for _printf_core
    printf8.o(i.__0vprintf$8) refers to fputc.o(i.fputc) for fputc
    printf8.o(i.__0vprintf$8) refers to stdout.o(.data) for __stdout
    printf8.o(i.__0vsnprintf$8) refers to printf8.o(i._printf_core) for _printf_core
    printf8.o(i.__0vsnprintf$8) refers to printf8.o(i._snputc) for _snputc
    printf8.o(i.__0vsprintf$8) refers to printf8.o(i._printf_core) for _printf_core
    printf8.o(i.__0vsprintf$8) refers to printf8.o(i._sputc) for _sputc
    printf8.o(i._printf_core) refers to printf8.o(i._printf_pre_padding) for _printf_pre_padding
    printf8.o(i._printf_core) refers to uldiv.o(.text) for __aeabi_uldivmod
    printf8.o(i._printf_core) refers to printf8.o(i._printf_post_padding) for _printf_post_padding
    printfa.o(i.__0fprintf) refers (Special) to iusefp.o(.text) for __I$use$fp
    printfa.o(i.__0fprintf) refers to printfa.o(i._printf_core) for _printf_core
    printfa.o(i.__0fprintf) refers to fputc.o(i.fputc) for fputc
    printfa.o(i.__0printf) refers (Special) to iusefp.o(.text) for __I$use$fp
    printfa.o(i.__0printf) refers to printfa.o(i._printf_core) for _printf_core
    printfa.o(i.__0printf) refers to fputc.o(i.fputc) for fputc
    printfa.o(i.__0printf) refers to stdout.o(.data) for __stdout
    printfa.o(i.__0snprintf) refers (Special) to iusefp.o(.text) for __I$use$fp
    printfa.o(i.__0snprintf) refers to printfa.o(i._printf_core) for _printf_core
    printfa.o(i.__0snprintf) refers to printfa.o(i._snputc) for _snputc
    printfa.o(i.__0sprintf) refers (Special) to iusefp.o(.text) for __I$use$fp
    printfa.o(i.__0sprintf) refers to printfa.o(i._printf_core) for _printf_core
    printfa.o(i.__0sprintf) refers to printfa.o(i._sputc) for _sputc
    printfa.o(i.__0vfprintf) refers (Special) to iusefp.o(.text) for __I$use$fp
    printfa.o(i.__0vfprintf) refers to printfa.o(i._printf_core) for _printf_core
    printfa.o(i.__0vfprintf) refers to fputc.o(i.fputc) for fputc
    printfa.o(i.__0vprintf) refers (Special) to iusefp.o(.text) for __I$use$fp
    printfa.o(i.__0vprintf) refers to printfa.o(i._printf_core) for _printf_core
    printfa.o(i.__0vprintf) refers to fputc.o(i.fputc) for fputc
    printfa.o(i.__0vprintf) refers to stdout.o(.data) for __stdout
    printfa.o(i.__0vsnprintf) refers (Special) to iusefp.o(.text) for __I$use$fp
    printfa.o(i.__0vsnprintf) refers to printfa.o(i._printf_core) for _printf_core
    printfa.o(i.__0vsnprintf) refers to printfa.o(i._snputc) for _snputc
    printfa.o(i.__0vsprintf) refers (Special) to iusefp.o(.text) for __I$use$fp
    printfa.o(i.__0vsprintf) refers to printfa.o(i._printf_core) for _printf_core
    printfa.o(i.__0vsprintf) refers to printfa.o(i._sputc) for _sputc
    printfa.o(i._fp_digits) refers (Special) to iusefp.o(.text) for __I$use$fp
    printfa.o(i._fp_digits) refers to dmul.o(.text) for __aeabi_dmul
    printfa.o(i._fp_digits) refers to ddiv.o(.text) for __aeabi_ddiv
    printfa.o(i._fp_digits) refers to cdrcmple.o(.text) for __aeabi_cdrcmple
    printfa.o(i._fp_digits) refers to dadd.o(.text) for __aeabi_dadd
    printfa.o(i._fp_digits) refers to dfixul.o(.text) for __aeabi_d2ulz
    printfa.o(i._fp_digits) refers to uldiv.o(.text) for __aeabi_uldivmod
    printfa.o(i._printf_core) refers (Special) to iusefp.o(.text) for __I$use$fp
    printfa.o(i._printf_core) refers to printfa.o(i._printf_pre_padding) for _printf_pre_padding
    printfa.o(i._printf_core) refers to uldiv.o(.text) for __aeabi_uldivmod
    printfa.o(i._printf_core) refers to printfa.o(i._printf_post_padding) for _printf_post_padding
    printfa.o(i._printf_core) refers to printfa.o(i._fp_digits) for _fp_digits
    printfa.o(i._printf_core) refers to uidiv.o(.text) for __aeabi_uidivmod
    printfa.o(i._printf_post_padding) refers (Special) to iusefp.o(.text) for __I$use$fp
    printfa.o(i._printf_pre_padding) refers (Special) to iusefp.o(.text) for __I$use$fp
    printfa.o(i._snputc) refers (Special) to iusefp.o(.text) for __I$use$fp
    printfa.o(i._sputc) refers (Special) to iusefp.o(.text) for __I$use$fp
    entry2.o(.ARM.Collect$$$$00000001) refers to entry2.o(.ARM.Collect$$$$00002712) for __lit__00000000
    entry2.o(.ARM.Collect$$$$00002712) refers to arm_startup_nrf52840.o(STACK) for __initial_sp
    entry2.o(__vectab_stack_and_reset_area) refers to arm_startup_nrf52840.o(STACK) for __initial_sp
    entry2.o(__vectab_stack_and_reset_area) refers to entry.o(.ARM.Collect$$$$00000000) for __main
    entry5.o(.ARM.Collect$$$$00000004) refers to init.o(.text) for __scatterload
    entry9a.o(.ARM.Collect$$$$0000000B) refers to main.o(i.main) for main
    entry9b.o(.ARM.Collect$$$$0000000C) refers to main.o(i.main) for main
    fputc.o(i.fputc) refers (Special) to iusesemip.o(.text) for __I$use$semihosting$fputc
    fputc.o(i.fputc) refers (Special) to semi.o(.text) for __semihosting_library_function
    dadd.o(.text) refers to llshl.o(.text) for __aeabi_llsl
    dadd.o(.text) refers to llsshr.o(.text) for __aeabi_lasr
    dadd.o(.text) refers to depilogue.o(.text) for _double_epilogue
    dmul.o(.text) refers to depilogue.o(.text) for _double_epilogue
    ddiv.o(.text) refers to depilogue.o(.text) for _double_round
    dfixul.o(.text) refers to llushr.o(.text) for __aeabi_llsr
    dfixul.o(.text) refers to llshl.o(.text) for __aeabi_llsl
    init.o(.text) refers to entry5.o(.ARM.Collect$$$$00000004) for __main_after_scatterload
    depilogue.o(.text) refers to llshl.o(.text) for __aeabi_llsl
    depilogue.o(.text) refers to llushr.o(.text) for __aeabi_llsr


==============================================================================

Removing Unused input sections from the image.

    Removing main.o(.rev16_text), (4 bytes).
    Removing main.o(.revsh_text), (4 bytes).
    Removing main.o(.rrx_text), (6 bytes).
    Removing boards.o(.rev16_text), (4 bytes).
    Removing boards.o(.revsh_text), (4 bytes).
    Removing boards.o(.rrx_text), (6 bytes).
    Removing boards.o(i.bsp_board_button_idx_to_pin), (12 bytes).
    Removing boards.o(i.bsp_board_led_idx_to_pin), (12 bytes).
    Removing boards.o(i.bsp_board_led_state_get), (40 bytes).
    Removing boards.o(i.bsp_board_leds_on), (18 bytes).
    Removing boards.o(i.bsp_board_pin_to_button_idx), (36 bytes).
    Removing boards.o(i.bsp_board_pin_to_led_idx), (36 bytes).
    Removing bsp.o(.rev16_text), (4 bytes).
    Removing bsp.o(.revsh_text), (4 bytes).
    Removing bsp.o(.rrx_text), (6 bytes).
    Removing bsp.o(i.alert_timer_handler), (6 bytes).
    Removing bsp.o(i.bsp_button_event_handler), (144 bytes).
    Removing bsp.o(i.bsp_button_is_pressed), (4 bytes).
    Removing bsp.o(i.bsp_buttons_disable), (4 bytes).
    Removing bsp.o(i.bsp_buttons_enable), (4 bytes).
    Removing bsp.o(i.bsp_event_to_button_action_assign), (68 bytes).
    Removing bsp.o(i.bsp_indication_set), (24 bytes).
    Removing bsp.o(i.bsp_init), (148 bytes).
    Removing bsp.o(i.bsp_led_indication), (440 bytes).
    Removing bsp.o(i.bsp_wakeup_button_disable), (16 bytes).
    Removing bsp.o(i.bsp_wakeup_button_enable), (16 bytes).
    Removing bsp.o(i.button_timer_handler), (8 bytes).
    Removing bsp.o(i.leds_off), (48 bytes).
    Removing bsp.o(i.leds_timer_handler), (20 bytes).
    Removing bsp.o(i.nrf_gpio_cfg_sense_set), (52 bytes).
    Removing bsp.o(.bss), (32 bytes).
    Removing bsp.o(.bss), (32 bytes).
    Removing bsp.o(.bss), (12 bytes).
    Removing bsp.o(.bss), (32 bytes).
    Removing bsp.o(.constdata), (44 bytes).
    Removing bsp.o(.data), (16 bytes).
    Removing bsp_nfc.o(.rev16_text), (4 bytes).
    Removing bsp_nfc.o(.revsh_text), (4 bytes).
    Removing bsp_nfc.o(.rrx_text), (6 bytes).
    Removing bsp_nfc.o(i.bsp_nfc_btn_deinit), (8 bytes).
    Removing bsp_nfc.o(i.bsp_nfc_btn_init), (8 bytes).
    Removing bsp_nfc.o(i.bsp_nfc_sleep_mode_prepare), (40 bytes).
    Removing app_usbd.o(.rev16_text), (4 bytes).
    Removing app_usbd.o(.revsh_text), (4 bytes).
    Removing app_usbd.o(.rrx_text), (6 bytes).
    Removing app_usbd.o(i.app_usbd_class_remove), (128 bytes).
    Removing app_usbd.o(i.app_usbd_class_remove_all), (32 bytes).
    Removing app_usbd.o(i.app_usbd_class_sof_first_get), (12 bytes).
    Removing app_usbd.o(i.app_usbd_ep_handler_set), (34 bytes).
    Removing app_usbd.o(i.app_usbd_req_std_set_interface), (110 bytes).
    Removing app_usbd.o(i.app_usbd_uninit), (80 bytes).
    Removing app_usbd_core.o(.rev16_text), (4 bytes).
    Removing app_usbd_core.o(.revsh_text), (4 bytes).
    Removing app_usbd_core.o(.rrx_text), (6 bytes).
    Removing app_usbd_core.o(i.app_usbd_core_class_rwu_pend), (60 bytes).
    Removing app_usbd_core.o(i.app_usbd_core_class_rwu_register), (16 bytes).
    Removing app_usbd_core.o(i.app_usbd_core_class_rwu_unregister), (16 bytes).
    Removing app_usbd_core.o(i.app_usbd_core_state_get), (12 bytes).
    Removing app_usbd_core.o(i.app_usbd_ep_handled_transfer), (24 bytes).
    Removing app_usbd_string_desc.o(.rev16_text), (4 bytes).
    Removing app_usbd_string_desc.o(.revsh_text), (4 bytes).
    Removing app_usbd_string_desc.o(.rrx_text), (6 bytes).
    Removing app_usbd_string_desc.o(.constdata), (2 bytes).
    Removing nrf_drv_clock.o(.rev16_text), (4 bytes).
    Removing nrf_drv_clock.o(.revsh_text), (4 bytes).
    Removing nrf_drv_clock.o(.rrx_text), (6 bytes).
    Removing nrf_drv_clock.o(i.hfclk_stop), (32 bytes).
    Removing nrf_drv_clock.o(i.lfclk_stop), (40 bytes).
    Removing nrf_drv_clock.o(i.nrf_drv_clock_calibration_abort), (4 bytes).
    Removing nrf_drv_clock.o(i.nrf_drv_clock_calibration_start), (4 bytes).
    Removing nrf_drv_clock.o(i.nrf_drv_clock_hfclk_release), (40 bytes).
    Removing nrf_drv_clock.o(i.nrf_drv_clock_init_check), (12 bytes).
    Removing nrf_drv_clock.o(i.nrf_drv_clock_is_calibrating), (4 bytes).
    Removing nrf_drv_clock.o(i.nrf_drv_clock_lfclk_is_running), (16 bytes).
    Removing nrf_drv_clock.o(i.nrf_drv_clock_lfclk_release), (40 bytes).
    Removing nrf_drv_clock.o(i.nrf_drv_clock_lfclk_request), (96 bytes).
    Removing nrf_drv_clock.o(i.nrf_drv_clock_uninit), (40 bytes).
    Removing nrf_drv_clock.o(.constdata), (19 bytes).
    Removing nrf_drv_clock.o(.constdata), (32 bytes).
    Removing nrf_drv_clock.o(.constdata), (32 bytes).
    Removing nrf_drv_clock.o(.constdata), (29 bytes).
    Removing nrf_drv_common.o(.rev16_text), (4 bytes).
    Removing nrf_drv_common.o(.revsh_text), (4 bytes).
    Removing nrf_drv_common.o(.rrx_text), (6 bytes).
    Removing nrf_drv_common.o(i.nrf_drv_common_clock_irq_disable), (20 bytes).
    Removing nrf_drv_common.o(i.nrf_drv_common_irq_disable), (22 bytes).
    Removing nrf_drv_common.o(i.nrf_drv_common_power_irq_disable), (20 bytes).
    Removing nrf_drv_gpiote.o(.rev16_text), (4 bytes).
    Removing nrf_drv_gpiote.o(.revsh_text), (4 bytes).
    Removing nrf_drv_gpiote.o(.rrx_text), (6 bytes).
    Removing nrf_drv_gpiote.o(i.channel_free), (28 bytes).
    Removing nrf_drv_gpiote.o(i.channel_port_alloc), (72 bytes).
    Removing nrf_drv_gpiote.o(i.nrf_drv_gpiote_clr_task_addr_get), (24 bytes).
    Removing nrf_drv_gpiote.o(i.nrf_drv_gpiote_clr_task_trigger), (28 bytes).
    Removing nrf_drv_gpiote.o(i.nrf_drv_gpiote_in_event_addr_get), (40 bytes).
    Removing nrf_drv_gpiote.o(i.nrf_drv_gpiote_in_event_disable), (72 bytes).
    Removing nrf_drv_gpiote.o(i.nrf_drv_gpiote_in_event_enable), (152 bytes).
    Removing nrf_drv_gpiote.o(i.nrf_drv_gpiote_in_init), (192 bytes).
    Removing nrf_drv_gpiote.o(i.nrf_drv_gpiote_in_is_set), (14 bytes).
    Removing nrf_drv_gpiote.o(i.nrf_drv_gpiote_in_uninit), (72 bytes).
    Removing nrf_drv_gpiote.o(i.nrf_drv_gpiote_init), (92 bytes).
    Removing nrf_drv_gpiote.o(i.nrf_drv_gpiote_is_init), (20 bytes).
    Removing nrf_drv_gpiote.o(i.nrf_drv_gpiote_out_clear), (4 bytes).
    Removing nrf_drv_gpiote.o(i.nrf_drv_gpiote_out_init), (176 bytes).
    Removing nrf_drv_gpiote.o(i.nrf_drv_gpiote_out_set), (4 bytes).
    Removing nrf_drv_gpiote.o(i.nrf_drv_gpiote_out_task_addr_get), (20 bytes).
    Removing nrf_drv_gpiote.o(i.nrf_drv_gpiote_out_task_disable), (36 bytes).
    Removing nrf_drv_gpiote.o(i.nrf_drv_gpiote_out_task_enable), (36 bytes).
    Removing nrf_drv_gpiote.o(i.nrf_drv_gpiote_out_task_force), (40 bytes).
    Removing nrf_drv_gpiote.o(i.nrf_drv_gpiote_out_task_trigger), (24 bytes).
    Removing nrf_drv_gpiote.o(i.nrf_drv_gpiote_out_toggle), (36 bytes).
    Removing nrf_drv_gpiote.o(i.nrf_drv_gpiote_out_uninit), (68 bytes).
    Removing nrf_drv_gpiote.o(i.nrf_drv_gpiote_set_task_addr_get), (24 bytes).
    Removing nrf_drv_gpiote.o(i.nrf_drv_gpiote_set_task_trigger), (28 bytes).
    Removing nrf_drv_gpiote.o(i.nrf_drv_gpiote_uninit), (56 bytes).
    Removing nrf_drv_gpiote.o(i.nrf_gpio_cfg), (50 bytes).
    Removing nrf_drv_gpiote.o(i.nrf_gpio_cfg_default), (18 bytes).
    Removing nrf_drv_gpiote.o(i.nrf_gpio_pin_clear), (20 bytes).
    Removing nrf_drv_gpiote.o(i.nrf_gpio_pin_read), (22 bytes).
    Removing nrf_drv_gpiote.o(i.nrf_gpio_pin_set), (20 bytes).
    Removing nrf_drv_gpiote.o(i.pin_in_use_by_port), (24 bytes).
    Removing nrf_drv_gpiote.o(i.pin_in_use_by_te), (24 bytes).
    Removing nrf_drv_gpiote.o(.constdata), (20 bytes).
    Removing nrf_drv_gpiote.o(.constdata), (24 bytes).
    Removing nrf_drv_gpiote.o(.constdata), (23 bytes).
    Removing nrf_drv_power.o(.rev16_text), (4 bytes).
    Removing nrf_drv_power.o(.revsh_text), (4 bytes).
    Removing nrf_drv_power.o(.rrx_text), (6 bytes).
    Removing nrf_drv_power.o(i.nrf_drv_power_init_check), (12 bytes).
    Removing nrf_drv_power.o(i.nrf_drv_power_pof_init), (72 bytes).
    Removing nrf_drv_power.o(i.nrf_drv_power_pof_uninit), (20 bytes).
    Removing nrf_drv_power.o(i.nrf_drv_power_sleepevt_init), (68 bytes).
    Removing nrf_drv_power.o(i.nrf_drv_power_sleepevt_uninit), (24 bytes).
    Removing nrf_drv_power.o(i.nrf_drv_power_uninit), (28 bytes).
    Removing nrf_drv_systick.o(.rev16_text), (4 bytes).
    Removing nrf_drv_systick.o(.revsh_text), (4 bytes).
    Removing nrf_drv_systick.o(.rrx_text), (6 bytes).
    Removing nrf_drv_systick.o(i.nrf_drv_systick_delay_ms), (38 bytes).
    Removing nrf_drv_systick.o(i.nrf_drv_systick_get), (10 bytes).
    Removing nrf_drv_systick.o(i.nrf_drv_systick_ms_tick), (20 bytes).
    Removing nrf_drv_systick.o(i.nrf_drv_systick_test), (48 bytes).
    Removing nrf_drv_uart.o(.rev16_text), (4 bytes).
    Removing nrf_drv_uart.o(.revsh_text), (4 bytes).
    Removing nrf_drv_uart.o(.rrx_text), (6 bytes).
    Removing nrf_drv_uart.o(i.nrf_drv_uart_errorsrc_get), (48 bytes).
    Removing nrf_drv_uart.o(i.nrf_drv_uart_rx), (176 bytes).
    Removing nrf_drv_uart.o(i.nrf_drv_uart_rx_abort), (40 bytes).
    Removing nrf_drv_uart.o(i.nrf_drv_uart_rx_disable), (36 bytes).
    Removing nrf_drv_uart.o(i.nrf_drv_uart_rx_enable), (48 bytes).
    Removing nrf_drv_uart.o(i.nrf_drv_uart_rx_for_uart), (168 bytes).
    Removing nrf_drv_uart.o(i.nrf_drv_uart_rx_for_uarte), (176 bytes).
    Removing nrf_drv_uart.o(i.nrf_drv_uart_rx_ready), (36 bytes).
    Removing nrf_drv_uart.o(i.nrf_drv_uart_tx_abort), (88 bytes).
    Removing nrf_drv_uart.o(i.rx_enable), (32 bytes).
    Removing nrf_drv_uart.o(.constdata), (18 bytes).
    Removing nrf_drv_uart.o(.constdata), (25 bytes).
    Removing nrf_drv_uart.o(.constdata), (26 bytes).
    Removing nrf_drv_uart.o(.constdata), (16 bytes).
    Removing nrf_drv_uart.o(.constdata), (25 bytes).
    Removing nrf_drv_uart.o(.constdata), (26 bytes).
    Removing nrf_drv_uart.o(.constdata), (16 bytes).
    Removing nrf_drv_usbd.o(.rev16_text), (4 bytes).
    Removing nrf_drv_usbd.o(.revsh_text), (4 bytes).
    Removing nrf_drv_usbd.o(.rrx_text), (6 bytes).
    Removing nrf_drv_usbd.o(i.nrf_drv_usbd_ep_disable), (60 bytes).
    Removing nrf_drv_usbd.o(i.nrf_drv_usbd_ep_enable_check), (40 bytes).
    Removing nrf_drv_usbd.o(i.nrf_drv_usbd_ep_is_busy), (32 bytes).
    Removing nrf_drv_usbd.o(i.nrf_drv_usbd_is_initialized), (16 bytes).
    Removing nrf_drv_usbd.o(i.nrf_drv_usbd_uninit), (32 bytes).
    Removing nrf_nvic.o(.rev16_text), (4 bytes).
    Removing nrf_nvic.o(.revsh_text), (4 bytes).
    Removing nrf_nvic.o(.rrx_text), (6 bytes).
    Removing nrf_nvic.o(i.sd_nvic_ClearPendingIRQ), (24 bytes).
    Removing nrf_nvic.o(i.sd_nvic_DisableIRQ), (24 bytes).
    Removing nrf_nvic.o(i.sd_nvic_EnableIRQ), (24 bytes).
    Removing nrf_nvic.o(i.sd_nvic_GetPendingIRQ), (42 bytes).
    Removing nrf_nvic.o(i.sd_nvic_GetPriority), (40 bytes).
    Removing nrf_nvic.o(i.sd_nvic_SetPendingIRQ), (24 bytes).
    Removing nrf_nvic.o(i.sd_nvic_SetPriority), (34 bytes).
    Removing nrf_nvic.o(i.sd_nvic_SystemReset), (36 bytes).
    Removing nrf_nvic.o(i.sd_nvic_critical_region_enter), (28 bytes).
    Removing nrf_nvic.o(i.sd_nvic_critical_region_exit), (24 bytes).
    Removing nrf_nvic.o(.data), (1 bytes).
    Removing nrf_soc.o(.rev16_text), (4 bytes).
    Removing nrf_soc.o(.revsh_text), (4 bytes).
    Removing nrf_soc.o(.rrx_text), (6 bytes).
    Removing nrf_soc.o(i.sd_app_evt_wait), (6 bytes).
    Removing app_button.o(.rev16_text), (4 bytes).
    Removing app_button.o(.revsh_text), (4 bytes).
    Removing app_button.o(.rrx_text), (6 bytes).
    Removing app_button.o(i.app_button_disable), (48 bytes).
    Removing app_button.o(i.app_button_enable), (36 bytes).
    Removing app_button.o(i.app_button_init), (112 bytes).
    Removing app_button.o(i.app_button_is_pushed), (36 bytes).
    Removing app_button.o(i.detection_delay_timeout_handler), (96 bytes).
    Removing app_button.o(i.gpiote_event_handler), (88 bytes).
    Removing app_button.o(.bss), (32 bytes).
    Removing app_button.o(.constdata), (8 bytes).
    Removing app_button.o(.data), (20 bytes).
    Removing app_error.o(.rev16_text), (4 bytes).
    Removing app_error.o(.revsh_text), (4 bytes).
    Removing app_error.o(.rrx_text), (6 bytes).
    Removing app_error.o(i.app_error_handler), (24 bytes).
    Removing app_error.o(i.app_error_save_and_stop), (100 bytes).
    Removing app_error.o(.bss), (32 bytes).
    Removing app_error_weak.o(.rev16_text), (4 bytes).
    Removing app_error_weak.o(.revsh_text), (4 bytes).
    Removing app_error_weak.o(.rrx_text), (6 bytes).
    Removing app_fifo.o(.rev16_text), (4 bytes).
    Removing app_fifo.o(.revsh_text), (4 bytes).
    Removing app_fifo.o(.rrx_text), (6 bytes).
    Removing app_fifo.o(i.app_fifo_flush), (8 bytes).
    Removing app_fifo.o(i.app_fifo_get), (22 bytes).
    Removing app_fifo.o(i.app_fifo_init), (32 bytes).
    Removing app_fifo.o(i.app_fifo_peek), (34 bytes).
    Removing app_fifo.o(i.app_fifo_put), (26 bytes).
    Removing app_fifo.o(i.app_fifo_read), (74 bytes).
    Removing app_fifo.o(i.app_fifo_write), (82 bytes).
    Removing app_fifo.o(i.fifo_get), (20 bytes).
    Removing app_fifo.o(i.fifo_put), (18 bytes).
    Removing app_scheduler.o(.rev16_text), (4 bytes).
    Removing app_scheduler.o(.revsh_text), (4 bytes).
    Removing app_scheduler.o(.rrx_text), (6 bytes).
    Removing app_scheduler.o(i.app_sched_event_put), (156 bytes).
    Removing app_scheduler.o(i.app_sched_execute), (64 bytes).
    Removing app_scheduler.o(i.app_sched_init), (44 bytes).
    Removing app_scheduler.o(i.app_sched_queue_space_get), (36 bytes).
    Removing app_scheduler.o(.data), (16 bytes).
    Removing app_timer.o(.rev16_text), (4 bytes).
    Removing app_timer.o(.revsh_text), (4 bytes).
    Removing app_timer.o(.rrx_text), (6 bytes).
    Removing app_timer.o(i.NVIC_SetPriority), (32 bytes).
    Removing app_timer.o(i.app_timer_cnt_diff_compute), (8 bytes).
    Removing app_timer.o(i.app_timer_cnt_get), (12 bytes).
    Removing app_timer.o(i.app_timer_create), (36 bytes).
    Removing app_timer.o(i.app_timer_init), (84 bytes).
    Removing app_timer.o(i.app_timer_pause), (12 bytes).
    Removing app_timer.o(i.app_timer_resume), (12 bytes).
    Removing app_timer.o(i.app_timer_start), (128 bytes).
    Removing app_timer.o(i.app_timer_stop), (32 bytes).
    Removing app_timer.o(i.app_timer_stop_all), (24 bytes).
    Removing app_timer.o(i.timer_stop_op_schedule), (64 bytes).
    Removing app_timer.o(i.user_op_alloc), (48 bytes).
    Removing app_uart_fifo.o(.rev16_text), (4 bytes).
    Removing app_uart_fifo.o(.revsh_text), (4 bytes).
    Removing app_uart_fifo.o(.rrx_text), (6 bytes).
    Removing app_uart_fifo.o(i.app_uart_close), (16 bytes).
    Removing app_uart_fifo.o(i.app_uart_flush), (32 bytes).
    Removing app_uart_fifo.o(i.app_uart_get), (52 bytes).
    Removing app_uart_fifo.o(i.app_uart_init), (180 bytes).
    Removing app_uart_fifo.o(i.app_uart_put), (60 bytes).
    Removing app_uart_fifo.o(i.uart_event_handler), (160 bytes).
    Removing app_uart_fifo.o(.bss), (32 bytes).
    Removing app_uart_fifo.o(.constdata), (32 bytes).
    Removing app_uart_fifo.o(.data), (16 bytes).
    Removing app_usbd_cdc_acm.o(.rev16_text), (4 bytes).
    Removing app_usbd_cdc_acm.o(.revsh_text), (4 bytes).
    Removing app_usbd_cdc_acm.o(.rrx_text), (6 bytes).
    Removing app_usbd_cdc_acm.o(i.app_usbd_cdc_acm_line_state_get), (54 bytes).
    Removing app_usbd_cdc_acm.o(i.app_usbd_cdc_acm_serial_state_notify), (136 bytes).
    Removing app_util_platform.o(.rev16_text), (4 bytes).
    Removing app_util_platform.o(.revsh_text), (4 bytes).
    Removing app_util_platform.o(.rrx_text), (6 bytes).
    Removing app_util_platform.o(i.current_int_priority_get), (48 bytes).
    Removing app_util_platform.o(i.privilege_level_get), (26 bytes).
    Removing hardfault_handler_keil.o(.rev16_text), (4 bytes).
    Removing hardfault_handler_keil.o(.revsh_text), (4 bytes).
    Removing hardfault_handler_keil.o(.rrx_text), (6 bytes).
    Removing hardfault_implementation.o(.rev16_text), (4 bytes).
    Removing hardfault_implementation.o(.revsh_text), (4 bytes).
    Removing hardfault_implementation.o(.rrx_text), (6 bytes).
    Removing nrf_assert.o(.rev16_text), (4 bytes).
    Removing nrf_assert.o(.revsh_text), (4 bytes).
    Removing nrf_assert.o(.rrx_text), (6 bytes).
    Removing nrf_strerror.o(.rev16_text), (4 bytes).
    Removing nrf_strerror.o(.revsh_text), (4 bytes).
    Removing nrf_strerror.o(.rrx_text), (6 bytes).
    Removing nrf_strerror.o(i.nrf_strerror_find), (56 bytes).
    Removing nrf_strerror.o(i.nrf_strerror_get), (20 bytes).
    Removing nrf_strerror.o(.constdata), (260 bytes).
    Removing nrf_strerror.o(.conststring), (776 bytes).
    Removing nrf_log_backend_serial.o(.rev16_text), (4 bytes).
    Removing nrf_log_backend_serial.o(.revsh_text), (4 bytes).
    Removing nrf_log_backend_serial.o(.rrx_text), (6 bytes).
    Removing nrf_log_backend_serial.o(i.nrf_log_backend_getchar), (52 bytes).
    Removing nrf_log_backend_serial.o(.constdata), (5 bytes).
    Removing nrf_log_frontend.o(.rev16_text), (4 bytes).
    Removing nrf_log_frontend.o(.revsh_text), (4 bytes).
    Removing nrf_log_frontend.o(.rrx_text), (6 bytes).
    Removing nrf_log_frontend.o(i.cont_buf_prealloc), (116 bytes).
    Removing nrf_log_frontend.o(i.nrf_log_frontend_hexdump), (144 bytes).
    Removing nrf_log_frontend.o(i.nrf_log_frontend_std_3), (124 bytes).
    Removing nrf_log_frontend.o(i.nrf_log_frontend_std_4), (136 bytes).
    Removing nrf_log_frontend.o(i.nrf_log_frontend_std_5), (152 bytes).
    Removing nrf_log_frontend.o(i.nrf_log_frontend_std_6), (164 bytes).
    Removing nrf_log_frontend.o(i.nrf_log_getchar), (4 bytes).
    Removing nrf_log_frontend.o(i.nrf_log_push), (96 bytes).
    Removing segger_rtt.o(.rev16_text), (4 bytes).
    Removing segger_rtt.o(.revsh_text), (4 bytes).
    Removing segger_rtt.o(.rrx_text), (6 bytes).
    Removing segger_rtt.o(i.SEGGER_RTT_ConfigDownBuffer), (92 bytes).
    Removing segger_rtt.o(i.SEGGER_RTT_ConfigUpBuffer), (92 bytes).
    Removing segger_rtt.o(i.SEGGER_RTT_GetKey), (28 bytes).
    Removing segger_rtt.o(i.SEGGER_RTT_HasData), (24 bytes).
    Removing segger_rtt.o(i.SEGGER_RTT_HasKey), (32 bytes).
    Removing segger_rtt.o(i.SEGGER_RTT_Init), (20 bytes).
    Removing segger_rtt.o(i.SEGGER_RTT_Read), (38 bytes).
    Removing segger_rtt.o(i.SEGGER_RTT_ReadNoLock), (124 bytes).
    Removing segger_rtt.o(i.SEGGER_RTT_SetNameDownBuffer), (60 bytes).
    Removing segger_rtt.o(i.SEGGER_RTT_SetNameUpBuffer), (60 bytes).
    Removing segger_rtt.o(i.SEGGER_RTT_SetTerminal), (132 bytes).
    Removing segger_rtt.o(i.SEGGER_RTT_TerminalOut), (172 bytes).
    Removing segger_rtt.o(i.SEGGER_RTT_WaitKey), (14 bytes).
    Removing segger_rtt.o(i.SEGGER_RTT_Write), (52 bytes).
    Removing segger_rtt.o(i.SEGGER_RTT_WriteNoLock), (92 bytes).
    Removing segger_rtt.o(i.SEGGER_RTT_WriteSkipNoLock), (116 bytes).
    Removing segger_rtt.o(i.SEGGER_RTT_WriteString), (26 bytes).
    Removing segger_rtt.o(i._DoInit), (104 bytes).
    Removing segger_rtt.o(i._GetAvailWriteSpace), (22 bytes).
    Removing segger_rtt.o(i._PostTerminalSwitch), (32 bytes).
    Removing segger_rtt.o(i._WriteBlocking), (90 bytes).
    Removing segger_rtt.o(i._WriteNoCheck), (62 bytes).
    Removing segger_rtt.o(.bss), (200 bytes).
    Removing segger_rtt.o(.data), (17 bytes).
    Removing arm_startup_nrf52840.o(HEAP), (8192 bytes).
    Removing system_nrf52840.o(.rev16_text), (4 bytes).
    Removing system_nrf52840.o(.revsh_text), (4 bytes).
    Removing system_nrf52840.o(.rrx_text), (6 bytes).
    Removing system_nrf52840.o(i.SystemCoreClockUpdate), (16 bytes).
    Removing dadd.o(.text), (334 bytes).
    Removing dmul.o(.text), (228 bytes).
    Removing ddiv.o(.text), (222 bytes).
    Removing dfixul.o(.text), (48 bytes).
    Removing cdrcmple.o(.text), (48 bytes).
    Removing depilogue.o(.text), (186 bytes).

335 unused section(s) (total 21980 bytes) removed from the image.

==============================================================================

Image Symbol Table

    Local Symbols

    Symbol Name                              Value     Ov Type        Size  Object(Section)

    RESET                                    0x00000000   Section      512  arm_startup_nrf52840.o(RESET)
    ../clib/microlib/ctype/ctype.c           0x00000000   Number         0  ctype_o.o ABSOLUTE
    ../clib/microlib/ctype/ctype.c           0x00000000   Number         0  isxdigit_o.o ABSOLUTE
    ../clib/microlib/ctype/ctype.c           0x00000000   Number         0  isalnum_o.o ABSOLUTE
    ../clib/microlib/ctype/ctype.c           0x00000000   Number         0  isalpha_o.o ABSOLUTE
    ../clib/microlib/ctype/ctype.c           0x00000000   Number         0  iscntrl_o.o ABSOLUTE
    ../clib/microlib/ctype/ctype.c           0x00000000   Number         0  isdigit_o.o ABSOLUTE
    ../clib/microlib/ctype/ctype.c           0x00000000   Number         0  isgraph_o.o ABSOLUTE
    ../clib/microlib/ctype/ctype.c           0x00000000   Number         0  islower_o.o ABSOLUTE
    ../clib/microlib/ctype/ctype.c           0x00000000   Number         0  isprint_o.o ABSOLUTE
    ../clib/microlib/ctype/ctype.c           0x00000000   Number         0  ispunct_o.o ABSOLUTE
    ../clib/microlib/ctype/ctype.c           0x00000000   Number         0  isspace_o.o ABSOLUTE
    ../clib/microlib/ctype/ctype.c           0x00000000   Number         0  isupper_o.o ABSOLUTE
    ../clib/microlib/ctype/ctype.c           0x00000000   Number         0  isblank_o.o ABSOLUTE
    ../clib/microlib/division.c              0x00000000   Number         0  uidiv.o ABSOLUTE
    ../clib/microlib/division.c              0x00000000   Number         0  uldiv.o ABSOLUTE
    ../clib/microlib/init/entry.s            0x00000000   Number         0  entry9a.o ABSOLUTE
    ../clib/microlib/init/entry.s            0x00000000   Number         0  entry8a.o ABSOLUTE
    ../clib/microlib/init/entry.s            0x00000000   Number         0  entry8b.o ABSOLUTE
    ../clib/microlib/init/entry.s            0x00000000   Number         0  entry9b.o ABSOLUTE
    ../clib/microlib/init/entry.s            0x00000000   Number         0  entry10a.o ABSOLUTE
    ../clib/microlib/init/entry.s            0x00000000   Number         0  entry11b.o ABSOLUTE
    ../clib/microlib/init/entry.s            0x00000000   Number         0  entry7b.o ABSOLUTE
    ../clib/microlib/init/entry.s            0x00000000   Number         0  entry11a.o ABSOLUTE
    ../clib/microlib/init/entry.s            0x00000000   Number         0  entry2.o ABSOLUTE
    ../clib/microlib/init/entry.s            0x00000000   Number         0  entry10b.o ABSOLUTE
    ../clib/microlib/init/entry.s            0x00000000   Number         0  entry.o ABSOLUTE
    ../clib/microlib/init/entry.s            0x00000000   Number         0  entry5.o ABSOLUTE
    ../clib/microlib/init/entry.s            0x00000000   Number         0  entry7a.o ABSOLUTE
    ../clib/microlib/longlong.c              0x00000000   Number         0  llshl.o ABSOLUTE
    ../clib/microlib/longlong.c              0x00000000   Number         0  llsshr.o ABSOLUTE
    ../clib/microlib/longlong.c              0x00000000   Number         0  llushr.o ABSOLUTE
    ../clib/microlib/printf/printf.c         0x00000000   Number         0  printf7.o ABSOLUTE
    ../clib/microlib/printf/printf.c         0x00000000   Number         0  printf6.o ABSOLUTE
    ../clib/microlib/printf/printf.c         0x00000000   Number         0  printfa.o ABSOLUTE
    ../clib/microlib/printf/printf.c         0x00000000   Number         0  printf4.o ABSOLUTE
    ../clib/microlib/printf/printf.c         0x00000000   Number         0  printf3.o ABSOLUTE
    ../clib/microlib/printf/printf.c         0x00000000   Number         0  printf2.o ABSOLUTE
    ../clib/microlib/printf/printf.c         0x00000000   Number         0  printf1.o ABSOLUTE
    ../clib/microlib/printf/printf.c         0x00000000   Number         0  printf0.o ABSOLUTE
    ../clib/microlib/printf/printf.c         0x00000000   Number         0  printfb.o ABSOLUTE
    ../clib/microlib/printf/printf.c         0x00000000   Number         0  printf8.o ABSOLUTE
    ../clib/microlib/printf/printf.c         0x00000000   Number         0  printf5.o ABSOLUTE
    ../clib/microlib/printf/stubs.s          0x00000000   Number         0  stubs.o ABSOLUTE
    ../clib/microlib/stdio/fputc.c           0x00000000   Number         0  fputc.o ABSOLUTE
    ../clib/microlib/stdio/semi.s            0x00000000   Number         0  semi.o ABSOLUTE
    ../clib/microlib/stdio/streams.c         0x00000000   Number         0  stdout.o ABSOLUTE
    ../clib/microlib/string/memcpy.c         0x00000000   Number         0  memcpya.o ABSOLUTE
    ../clib/microlib/string/memcpy.c         0x00000000   Number         0  memcpyb.o ABSOLUTE
    ../clib/microlib/string/memset.c         0x00000000   Number         0  memseta.o ABSOLUTE
    ../clib/microlib/string/strcpy.c         0x00000000   Number         0  strcpy.o ABSOLUTE
    ../clib/microlib/string/strlen.c         0x00000000   Number         0  strlen.o ABSOLUTE
    ../clib/microlib/stubs.s                 0x00000000   Number         0  iusesemip.o ABSOLUTE
    ../clib/microlib/stubs.s                 0x00000000   Number         0  iusefp.o ABSOLUTE
    ../fplib/microlib/fpadd.c                0x00000000   Number         0  dadd.o ABSOLUTE
    ../fplib/microlib/fpdiv.c                0x00000000   Number         0  ddiv.o ABSOLUTE
    ../fplib/microlib/fpepilogue.c           0x00000000   Number         0  depilogue.o ABSOLUTE
    ../fplib/microlib/fpfix.c                0x00000000   Number         0  dfixul.o ABSOLUTE
    ../fplib/microlib/fpmul.c                0x00000000   Number         0  dmul.o ABSOLUTE
    ..\..\..\..\..\..\components\boards\boards.c 0x00000000   Number         0  boards.o ABSOLUTE
    ..\..\..\..\..\..\components\drivers_nrf\clock\nrf_drv_clock.c 0x00000000   Number         0  nrf_drv_clock.o ABSOLUTE
    ..\..\..\..\..\..\components\drivers_nrf\common\nrf_drv_common.c 0x00000000   Number         0  nrf_drv_common.o ABSOLUTE
    ..\..\..\..\..\..\components\drivers_nrf\gpiote\nrf_drv_gpiote.c 0x00000000   Number         0  nrf_drv_gpiote.o ABSOLUTE
    ..\..\..\..\..\..\components\drivers_nrf\nrf_soc_nosd\nrf_nvic.c 0x00000000   Number         0  nrf_nvic.o ABSOLUTE
    ..\..\..\..\..\..\components\drivers_nrf\nrf_soc_nosd\nrf_soc.c 0x00000000   Number         0  nrf_soc.o ABSOLUTE
    ..\..\..\..\..\..\components\drivers_nrf\power\nrf_drv_power.c 0x00000000   Number         0  nrf_drv_power.o ABSOLUTE
    ..\..\..\..\..\..\components\drivers_nrf\systick\nrf_drv_systick.c 0x00000000   Number         0  nrf_drv_systick.o ABSOLUTE
    ..\..\..\..\..\..\components\drivers_nrf\uart\nrf_drv_uart.c 0x00000000   Number         0  nrf_drv_uart.o ABSOLUTE
    ..\..\..\..\..\..\components\drivers_nrf\usbd\nrf_drv_usbd.c 0x00000000   Number         0  nrf_drv_usbd.o ABSOLUTE
    ..\..\..\..\..\..\components\libraries\bsp\bsp.c 0x00000000   Number         0  bsp.o ABSOLUTE
    ..\..\..\..\..\..\components\libraries\bsp\bsp_nfc.c 0x00000000   Number         0  bsp_nfc.o ABSOLUTE
    ..\..\..\..\..\..\components\libraries\button\app_button.c 0x00000000   Number         0  app_button.o ABSOLUTE
    ..\..\..\..\..\..\components\libraries\fifo\app_fifo.c 0x00000000   Number         0  app_fifo.o ABSOLUTE
    ..\..\..\..\..\..\components\libraries\hardfault\hardfault_implementation.c 0x00000000   Number         0  hardfault_implementation.o ABSOLUTE
    ..\..\..\..\..\..\components\libraries\hardfault\nrf52\handler\hardfault_handler_keil.c 0x00000000   Number         0  hardfault_handler_keil.o ABSOLUTE
    ..\..\..\..\..\..\components\libraries\log\src\nrf_log_backend_serial.c 0x00000000   Number         0  nrf_log_backend_serial.o ABSOLUTE
    ..\..\..\..\..\..\components\libraries\log\src\nrf_log_frontend.c 0x00000000   Number         0  nrf_log_frontend.o ABSOLUTE
    ..\..\..\..\..\..\components\libraries\scheduler\app_scheduler.c 0x00000000   Number         0  app_scheduler.o ABSOLUTE
    ..\..\..\..\..\..\components\libraries\strerror\nrf_strerror.c 0x00000000   Number         0  nrf_strerror.o ABSOLUTE
    ..\..\..\..\..\..\components\libraries\timer\app_timer.c 0x00000000   Number         0  app_timer.o ABSOLUTE
    ..\..\..\..\..\..\components\libraries\uart\app_uart_fifo.c 0x00000000   Number         0  app_uart_fifo.o ABSOLUTE
    ..\..\..\..\..\..\components\libraries\usbd\app_usbd.c 0x00000000   Number         0  app_usbd.o ABSOLUTE
    ..\..\..\..\..\..\components\libraries\usbd\app_usbd_core.c 0x00000000   Number         0  app_usbd_core.o ABSOLUTE
    ..\..\..\..\..\..\components\libraries\usbd\app_usbd_string_desc.c 0x00000000   Number         0  app_usbd_string_desc.o ABSOLUTE
    ..\..\..\..\..\..\components\libraries\usbd\class\cdc\acm\app_usbd_cdc_acm.c 0x00000000   Number         0  app_usbd_cdc_acm.o ABSOLUTE
    ..\..\..\..\..\..\components\libraries\util\app_error.c 0x00000000   Number         0  app_error.o ABSOLUTE
    ..\..\..\..\..\..\components\libraries\util\app_error_weak.c 0x00000000   Number         0  app_error_weak.o ABSOLUTE
    ..\..\..\..\..\..\components\libraries\util\app_util_platform.c 0x00000000   Number         0  app_util_platform.o ABSOLUTE
    ..\..\..\..\..\..\components\libraries\util\nrf_assert.c 0x00000000   Number         0  nrf_assert.o ABSOLUTE
    ..\..\..\..\..\..\external\segger_rtt\RTT_Syscalls_KEIL.c 0x00000000   Number         0  rtt_syscalls_keil.o ABSOLUTE
    ..\..\..\..\..\..\external\segger_rtt\SEGGER_RTT.c 0x00000000   Number         0  segger_rtt.o ABSOLUTE
    ..\..\..\..\..\..\external\segger_rtt\SEGGER_RTT_printf.c 0x00000000   Number         0  segger_rtt_printf.o ABSOLUTE
    ..\..\..\main.c                          0x00000000   Number         0  main.o ABSOLUTE
    ..\\..\\..\\..\\..\\..\\components\\boards\\boards.c 0x00000000   Number         0  boards.o ABSOLUTE
    ..\\..\\..\\..\\..\\..\\components\\drivers_nrf\\clock\\nrf_drv_clock.c 0x00000000   Number         0  nrf_drv_clock.o ABSOLUTE
    ..\\..\\..\\..\\..\\..\\components\\drivers_nrf\\common\\nrf_drv_common.c 0x00000000   Number         0  nrf_drv_common.o ABSOLUTE
    ..\\..\\..\\..\\..\\..\\components\\drivers_nrf\\gpiote\\nrf_drv_gpiote.c 0x00000000   Number         0  nrf_drv_gpiote.o ABSOLUTE
    ..\\..\\..\\..\\..\\..\\components\\drivers_nrf\\nrf_soc_nosd\\nrf_nvic.c 0x00000000   Number         0  nrf_nvic.o ABSOLUTE
    ..\\..\\..\\..\\..\\..\\components\\drivers_nrf\\nrf_soc_nosd\\nrf_soc.c 0x00000000   Number         0  nrf_soc.o ABSOLUTE
    ..\\..\\..\\..\\..\\..\\components\\drivers_nrf\\power\\nrf_drv_power.c 0x00000000   Number         0  nrf_drv_power.o ABSOLUTE
    ..\\..\\..\\..\\..\\..\\components\\drivers_nrf\\systick\\nrf_drv_systick.c 0x00000000   Number         0  nrf_drv_systick.o ABSOLUTE
    ..\\..\\..\\..\\..\\..\\components\\drivers_nrf\\uart\\nrf_drv_uart.c 0x00000000   Number         0  nrf_drv_uart.o ABSOLUTE
    ..\\..\\..\\..\\..\\..\\components\\drivers_nrf\\usbd\\nrf_drv_usbd.c 0x00000000   Number         0  nrf_drv_usbd.o ABSOLUTE
    ..\\..\\..\\..\\..\\..\\components\\libraries\\bsp\\bsp.c 0x00000000   Number         0  bsp.o ABSOLUTE
    ..\\..\\..\\..\\..\\..\\components\\libraries\\bsp\\bsp_nfc.c 0x00000000   Number         0  bsp_nfc.o ABSOLUTE
    ..\\..\\..\\..\\..\\..\\components\\libraries\\button\\app_button.c 0x00000000   Number         0  app_button.o ABSOLUTE
    ..\\..\\..\\..\\..\\..\\components\\libraries\\fifo\\app_fifo.c 0x00000000   Number         0  app_fifo.o ABSOLUTE
    ..\\..\\..\\..\\..\\..\\components\\libraries\\hardfault\\hardfault_implementation.c 0x00000000   Number         0  hardfault_implementation.o ABSOLUTE
    ..\\..\\..\\..\\..\\..\\components\\libraries\\hardfault\\nrf52\\handler\\hardfault_handler_keil.c 0x00000000   Number         0  hardfault_handler_keil.o ABSOLUTE
    ..\\..\\..\\..\\..\\..\\components\\libraries\\log\\src\\nrf_log_backend_serial.c 0x00000000   Number         0  nrf_log_backend_serial.o ABSOLUTE
    ..\\..\\..\\..\\..\\..\\components\\libraries\\log\\src\\nrf_log_frontend.c 0x00000000   Number         0  nrf_log_frontend.o ABSOLUTE
    ..\\..\\..\\..\\..\\..\\components\\libraries\\scheduler\\app_scheduler.c 0x00000000   Number         0  app_scheduler.o ABSOLUTE
    ..\\..\\..\\..\\..\\..\\components\\libraries\\strerror\\nrf_strerror.c 0x00000000   Number         0  nrf_strerror.o ABSOLUTE
    ..\\..\\..\\..\\..\\..\\components\\libraries\\timer\\app_timer.c 0x00000000   Number         0  app_timer.o ABSOLUTE
    ..\\..\\..\\..\\..\\..\\components\\libraries\\uart\\app_uart_fifo.c 0x00000000   Number         0  app_uart_fifo.o ABSOLUTE
    ..\\..\\..\\..\\..\\..\\components\\libraries\\usbd\\app_usbd.c 0x00000000   Number         0  app_usbd.o ABSOLUTE
    ..\\..\\..\\..\\..\\..\\components\\libraries\\usbd\\app_usbd_core.c 0x00000000   Number         0  app_usbd_core.o ABSOLUTE
    ..\\..\\..\\..\\..\\..\\components\\libraries\\usbd\\app_usbd_string_desc.c 0x00000000   Number         0  app_usbd_string_desc.o ABSOLUTE
    ..\\..\\..\\..\\..\\..\\components\\libraries\\usbd\\class\\cdc\\acm\\app_usbd_cdc_acm.c 0x00000000   Number         0  app_usbd_cdc_acm.o ABSOLUTE
    ..\\..\\..\\..\\..\\..\\components\\libraries\\util\\app_error.c 0x00000000   Number         0  app_error.o ABSOLUTE
    ..\\..\\..\\..\\..\\..\\components\\libraries\\util\\app_error_weak.c 0x00000000   Number         0  app_error_weak.o ABSOLUTE
    ..\\..\\..\\..\\..\\..\\components\\libraries\\util\\app_util_platform.c 0x00000000   Number         0  app_util_platform.o ABSOLUTE
    ..\\..\\..\\..\\..\\..\\components\\libraries\\util\\nrf_assert.c 0x00000000   Number         0  nrf_assert.o ABSOLUTE
    ..\\..\\..\\..\\..\\..\\external\\segger_rtt\\SEGGER_RTT.c 0x00000000   Number         0  segger_rtt.o ABSOLUTE
    ..\\..\\..\\main.c                       0x00000000   Number         0  main.o ABSOLUTE
    RTE\Device\nRF52840_xxAA\arm_startup_nrf52840.s 0x00000000   Number         0  arm_startup_nrf52840.o ABSOLUTE
    RTE\Device\nRF52840_xxAA\system_nrf52840.c 0x00000000   Number         0  system_nrf52840.o ABSOLUTE
    RTE\\Device\\nRF52840_xxAA\\system_nrf52840.c 0x00000000   Number         0  system_nrf52840.o ABSOLUTE
    cdrcmple.s                               0x00000000   Number         0  cdrcmple.o ABSOLUTE
    dc.s                                     0x00000000   Number         0  dc.o ABSOLUTE
    handlers.s                               0x00000000   Number         0  handlers.o ABSOLUTE
    init.s                                   0x00000000   Number         0  init.o ABSOLUTE
    .ARM.Collect$$$$00000000                 0x00000200   Section        0  entry.o(.ARM.Collect$$$$00000000)
    .ARM.Collect$$$$00000001                 0x00000200   Section        4  entry2.o(.ARM.Collect$$$$00000001)
    .ARM.Collect$$$$00000004                 0x00000204   Section        4  entry5.o(.ARM.Collect$$$$00000004)
    .ARM.Collect$$$$00000008                 0x00000208   Section        0  entry7b.o(.ARM.Collect$$$$00000008)
    .ARM.Collect$$$$0000000A                 0x00000208   Section        0  entry8b.o(.ARM.Collect$$$$0000000A)
    .ARM.Collect$$$$0000000B                 0x00000208   Section        8  entry9a.o(.ARM.Collect$$$$0000000B)
    .ARM.Collect$$$$0000000D                 0x00000210   Section        0  entry10a.o(.ARM.Collect$$$$0000000D)
    .ARM.Collect$$$$0000000F                 0x00000210   Section        0  entry11a.o(.ARM.Collect$$$$0000000F)
    .ARM.Collect$$$$00002712                 0x00000210   Section        4  entry2.o(.ARM.Collect$$$$00002712)
    __lit__00000000                          0x00000210   Data           4  entry2.o(.ARM.Collect$$$$00002712)
    .emb_text                                0x00000214   Section      154  app_usbd_core.o(.emb_text)
    $v0                                      0x00000214   Number         0  app_usbd_core.o(.emb_text)
    .emb_text                                0x000002b0   Section      154  nrf_drv_usbd.o(.emb_text)
    $v0                                      0x000002b0   Number         0  nrf_drv_usbd.o(.emb_text)
    .emb_text                                0x0000034c   Section       52  hardfault_handler_keil.o(.emb_text)
    $v0                                      0x0000034c   Number         0  hardfault_handler_keil.o(.emb_text)
    .text                                    0x00000380   Section       36  arm_startup_nrf52840.o(.text)
    $v0                                      0x00000380   Number         0  arm_startup_nrf52840.o(.text)
    .text                                    0x000003a4   Section        0  uldiv.o(.text)
    .text                                    0x00000408   Section        0  ctype_o.o(.text)
    .text                                    0x00000410   Section        0  memcpya.o(.text)
    .text                                    0x00000434   Section        0  memseta.o(.text)
    .text                                    0x00000458   Section        0  strlen.o(.text)
    .text                                    0x00000466   Section        0  llshl.o(.text)
    .text                                    0x00000484   Section        0  llushr.o(.text)
    .text                                    0x000004a4   Section       36  init.o(.text)
    i.GPIOTE_IRQHandler                      0x000004c8   Section        0  nrf_drv_gpiote.o(i.GPIOTE_IRQHandler)
    i.HardFault_c_handler                    0x0000068c   Section        0  hardfault_implementation.o(i.HardFault_c_handler)
    i.HardFault_process                      0x000006d0   Section        0  hardfault_implementation.o(i.HardFault_process)
    i.NVIC_ClearPendingIRQ                   0x000006f4   Section        0  app_timer.o(i.NVIC_ClearPendingIRQ)
    NVIC_ClearPendingIRQ                     0x000006f5   Thumb Code    22  app_timer.o(i.NVIC_ClearPendingIRQ)
    i.NVIC_EnableIRQ                         0x0000070a   Section        0  app_timer.o(i.NVIC_EnableIRQ)
    NVIC_EnableIRQ                           0x0000070b   Thumb Code    22  app_timer.o(i.NVIC_EnableIRQ)
    i.NVIC_SetPendingIRQ                     0x00000720   Section        0  app_timer.o(i.NVIC_SetPendingIRQ)
    NVIC_SetPendingIRQ                       0x00000721   Thumb Code    22  app_timer.o(i.NVIC_SetPendingIRQ)
    i.POWER_CLOCK_IRQHandler                 0x00000736   Section        0  nrf_drv_common.o(i.POWER_CLOCK_IRQHandler)
    i.RTC1_IRQHandler                        0x00000744   Section        0  app_timer.o(i.RTC1_IRQHandler)
    i.SWI0_EGU0_IRQHandler                   0x00000768   Section        0  app_timer.o(i.SWI0_EGU0_IRQHandler)
    i.SystemInit                             0x0000076c   Section        0  system_nrf52840.o(i.SystemInit)
    i.UARTE0_UART0_IRQHandler                0x00000954   Section        0  nrf_drv_uart.o(i.UARTE0_UART0_IRQHandler)
    i.USBD_IRQHandler                        0x00000970   Section        0  nrf_drv_usbd.o(i.USBD_IRQHandler)
    i.USBD_ISR_AccessFault                   0x00000ad0   Section        0  nrf_drv_usbd.o(i.USBD_ISR_AccessFault)
    USBD_ISR_AccessFault                     0x00000ad1   Thumb Code     2  nrf_drv_usbd.o(i.USBD_ISR_AccessFault)
    i.USBD_ISR_EpDataStatus                  0x00000ad4   Section        0  nrf_drv_usbd.o(i.USBD_ISR_EpDataStatus)
    USBD_ISR_EpDataStatus                    0x00000ad5   Thumb Code    82  nrf_drv_usbd.o(i.USBD_ISR_EpDataStatus)
    i.USBD_ISR_Event                         0x00000b30   Section        0  nrf_drv_usbd.o(i.USBD_ISR_Event)
    USBD_ISR_Event                           0x00000b31   Thumb Code    54  nrf_drv_usbd.o(i.USBD_ISR_Event)
    i.USBD_ISR_Setup                         0x00000b74   Section        0  nrf_drv_usbd.o(i.USBD_ISR_Setup)
    USBD_ISR_Setup                           0x00000b75   Thumb Code   122  nrf_drv_usbd.o(i.USBD_ISR_Setup)
    i.USBD_ISR_SetupData                     0x00000c00   Section        0  nrf_drv_usbd.o(i.USBD_ISR_SetupData)
    USBD_ISR_SetupData                       0x00000c01   Thumb Code    22  nrf_drv_usbd.o(i.USBD_ISR_SetupData)
    i.USBD_ISR_Sof                           0x00000c1c   Section        0  nrf_drv_usbd.o(i.USBD_ISR_Sof)
    USBD_ISR_Sof                             0x00000c1d   Thumb Code    52  nrf_drv_usbd.o(i.USBD_ISR_Sof)
    i.USBD_ISR_Started                       0x00000c58   Section        0  nrf_drv_usbd.o(i.USBD_ISR_Started)
    USBD_ISR_Started                         0x00000c59   Thumb Code    46  nrf_drv_usbd.o(i.USBD_ISR_Started)
    i.USBD_ISR_Usbreset                      0x00000c8c   Section        0  nrf_drv_usbd.o(i.USBD_ISR_Usbreset)
    USBD_ISR_Usbreset                        0x00000c8d   Thumb Code    26  nrf_drv_usbd.o(i.USBD_ISR_Usbreset)
    i.USBD_ISR_dma_epin0                     0x00000cb0   Section        0  nrf_drv_usbd.o(i.USBD_ISR_dma_epin0)
    USBD_ISR_dma_epin0                       0x00000cb1   Thumb Code    52  nrf_drv_usbd.o(i.USBD_ISR_dma_epin0)
    i.USBD_ISR_dma_epin1                     0x00000ce8   Section        0  nrf_drv_usbd.o(i.USBD_ISR_dma_epin1)
    USBD_ISR_dma_epin1                       0x00000ce9   Thumb Code     6  nrf_drv_usbd.o(i.USBD_ISR_dma_epin1)
    i.USBD_ISR_dma_epin2                     0x00000cee   Section        0  nrf_drv_usbd.o(i.USBD_ISR_dma_epin2)
    USBD_ISR_dma_epin2                       0x00000cef   Thumb Code     6  nrf_drv_usbd.o(i.USBD_ISR_dma_epin2)
    i.USBD_ISR_dma_epin3                     0x00000cf4   Section        0  nrf_drv_usbd.o(i.USBD_ISR_dma_epin3)
    USBD_ISR_dma_epin3                       0x00000cf5   Thumb Code     6  nrf_drv_usbd.o(i.USBD_ISR_dma_epin3)
    i.USBD_ISR_dma_epin4                     0x00000cfa   Section        0  nrf_drv_usbd.o(i.USBD_ISR_dma_epin4)
    USBD_ISR_dma_epin4                       0x00000cfb   Thumb Code     6  nrf_drv_usbd.o(i.USBD_ISR_dma_epin4)
    i.USBD_ISR_dma_epin5                     0x00000d00   Section        0  nrf_drv_usbd.o(i.USBD_ISR_dma_epin5)
    USBD_ISR_dma_epin5                       0x00000d01   Thumb Code     6  nrf_drv_usbd.o(i.USBD_ISR_dma_epin5)
    i.USBD_ISR_dma_epin6                     0x00000d06   Section        0  nrf_drv_usbd.o(i.USBD_ISR_dma_epin6)
    USBD_ISR_dma_epin6                       0x00000d07   Thumb Code     6  nrf_drv_usbd.o(i.USBD_ISR_dma_epin6)
    i.USBD_ISR_dma_epin7                     0x00000d0c   Section        0  nrf_drv_usbd.o(i.USBD_ISR_dma_epin7)
    USBD_ISR_dma_epin7                       0x00000d0d   Thumb Code     6  nrf_drv_usbd.o(i.USBD_ISR_dma_epin7)
    i.USBD_ISR_dma_epin8                     0x00000d14   Section        0  nrf_drv_usbd.o(i.USBD_ISR_dma_epin8)
    USBD_ISR_dma_epin8                       0x00000d15   Thumb Code    66  nrf_drv_usbd.o(i.USBD_ISR_dma_epin8)
    i.USBD_ISR_dma_epout0                    0x00000d60   Section        0  nrf_drv_usbd.o(i.USBD_ISR_dma_epout0)
    USBD_ISR_dma_epout0                      0x00000d61   Thumb Code    64  nrf_drv_usbd.o(i.USBD_ISR_dma_epout0)
    i.USBD_ISR_dma_epout1                    0x00000da8   Section        0  nrf_drv_usbd.o(i.USBD_ISR_dma_epout1)
    USBD_ISR_dma_epout1                      0x00000da9   Thumb Code     6  nrf_drv_usbd.o(i.USBD_ISR_dma_epout1)
    i.USBD_ISR_dma_epout2                    0x00000dae   Section        0  nrf_drv_usbd.o(i.USBD_ISR_dma_epout2)
    USBD_ISR_dma_epout2                      0x00000daf   Thumb Code     6  nrf_drv_usbd.o(i.USBD_ISR_dma_epout2)
    i.USBD_ISR_dma_epout3                    0x00000db4   Section        0  nrf_drv_usbd.o(i.USBD_ISR_dma_epout3)
    USBD_ISR_dma_epout3                      0x00000db5   Thumb Code     6  nrf_drv_usbd.o(i.USBD_ISR_dma_epout3)
    i.USBD_ISR_dma_epout4                    0x00000dba   Section        0  nrf_drv_usbd.o(i.USBD_ISR_dma_epout4)
    USBD_ISR_dma_epout4                      0x00000dbb   Thumb Code     6  nrf_drv_usbd.o(i.USBD_ISR_dma_epout4)
    i.USBD_ISR_dma_epout5                    0x00000dc0   Section        0  nrf_drv_usbd.o(i.USBD_ISR_dma_epout5)
    USBD_ISR_dma_epout5                      0x00000dc1   Thumb Code     6  nrf_drv_usbd.o(i.USBD_ISR_dma_epout5)
    i.USBD_ISR_dma_epout6                    0x00000dc6   Section        0  nrf_drv_usbd.o(i.USBD_ISR_dma_epout6)
    USBD_ISR_dma_epout6                      0x00000dc7   Thumb Code     6  nrf_drv_usbd.o(i.USBD_ISR_dma_epout6)
    i.USBD_ISR_dma_epout7                    0x00000dcc   Section        0  nrf_drv_usbd.o(i.USBD_ISR_dma_epout7)
    USBD_ISR_dma_epout7                      0x00000dcd   Thumb Code     6  nrf_drv_usbd.o(i.USBD_ISR_dma_epout7)
    i.USBD_ISR_dma_epout8                    0x00000dd4   Section        0  nrf_drv_usbd.o(i.USBD_ISR_dma_epout8)
    USBD_ISR_dma_epout8                      0x00000dd5   Thumb Code    66  nrf_drv_usbd.o(i.USBD_ISR_dma_epout8)
    i.__0snprintf$8                          0x00000e20   Section        0  printf8.o(i.__0snprintf$8)
    i.__0sprintf$8                           0x00000e48   Section        0  printf8.o(i.__0sprintf$8)
    i.__scatterload_copy                     0x00000e70   Section       14  handlers.o(i.__scatterload_copy)
    i.__scatterload_null                     0x00000e7e   Section        2  handlers.o(i.__scatterload_null)
    i.__scatterload_zeroinit                 0x00000e80   Section       14  handlers.o(i.__scatterload_zeroinit)
    i._printf_core                           0x00000e90   Section        0  printf8.o(i._printf_core)
    _printf_core                             0x00000e91   Thumb Code   996  printf8.o(i._printf_core)
    i._printf_post_padding                   0x000012a0   Section        0  printf8.o(i._printf_post_padding)
    _printf_post_padding                     0x000012a1   Thumb Code    36  printf8.o(i._printf_post_padding)
    i._printf_pre_padding                    0x000012c4   Section        0  printf8.o(i._printf_pre_padding)
    _printf_pre_padding                      0x000012c5   Thumb Code    46  printf8.o(i._printf_pre_padding)
    i._snputc                                0x000012f2   Section        0  printf8.o(i._snputc)
    _snputc                                  0x000012f3   Thumb Code    22  printf8.o(i._snputc)
    i._sputc                                 0x00001308   Section        0  printf8.o(i._sputc)
    _sputc                                   0x00001309   Thumb Code    10  printf8.o(i._sputc)
    i.app_error_fault_handler                0x00001314   Section        0  app_error_weak.o(i.app_error_fault_handler)
    i.app_error_handler_bare                 0x00001380   Section        0  app_error.o(i.app_error_handler_bare)
    i.app_usbd_all_call                      0x00001398   Section        0  app_usbd.o(i.app_usbd_all_call)
    i.app_usbd_all_until_served_call         0x000013b8   Section        0  app_usbd.o(i.app_usbd_all_until_served_call)
    i.app_usbd_cdc_acm_read                  0x000013dc   Section        0  app_usbd_cdc_acm.o(i.app_usbd_cdc_acm_read)
    i.app_usbd_cdc_acm_rx_size               0x00001404   Section        0  app_usbd_cdc_acm.o(i.app_usbd_cdc_acm_rx_size)
    i.app_usbd_cdc_acm_write                 0x0000141a   Section        0  app_usbd_cdc_acm.o(i.app_usbd_cdc_acm_write)
    i.app_usbd_class_append                  0x00001444   Section        0  app_usbd.o(i.app_usbd_class_append)
    i.app_usbd_class_descriptor_find         0x000014d4   Section        0  app_usbd.o(i.app_usbd_class_descriptor_find)
    i.app_usbd_class_first_get               0x00001518   Section        0  app_usbd.o(i.app_usbd_class_first_get)
    i.app_usbd_class_iface_ep_get            0x00001524   Section        0  app_usbd.o(i.app_usbd_class_iface_ep_get)
    app_usbd_class_iface_ep_get              0x00001525   Thumb Code    18  app_usbd.o(i.app_usbd_class_iface_ep_get)
    i.app_usbd_class_iface_ep_get            0x00001536   Section        0  app_usbd_cdc_acm.o(i.app_usbd_class_iface_ep_get)
    app_usbd_class_iface_ep_get              0x00001537   Thumb Code    18  app_usbd_cdc_acm.o(i.app_usbd_class_iface_ep_get)
    i.app_usbd_class_iface_get               0x00001548   Section        0  app_usbd.o(i.app_usbd_class_iface_get)
    app_usbd_class_iface_get                 0x00001549   Thumb Code    20  app_usbd.o(i.app_usbd_class_iface_get)
    i.app_usbd_class_iface_get               0x0000155c   Section        0  app_usbd_cdc_acm.o(i.app_usbd_class_iface_get)
    app_usbd_class_iface_get                 0x0000155d   Thumb Code    20  app_usbd_cdc_acm.o(i.app_usbd_class_iface_get)
    i.app_usbd_class_sof_register            0x00001570   Section        0  app_usbd.o(i.app_usbd_class_sof_register)
    i.app_usbd_class_sof_unregister          0x00001588   Section        0  app_usbd.o(i.app_usbd_class_sof_unregister)
    i.app_usbd_core_ep_transfer              0x000015b4   Section        0  app_usbd_core.o(i.app_usbd_core_ep_transfer)
    i.app_usbd_core_event_handler            0x000015cc   Section        0  app_usbd_core.o(i.app_usbd_core_event_handler)
    app_usbd_core_event_handler              0x000015cd   Thumb Code   188  app_usbd_core.o(i.app_usbd_core_event_handler)
    i.app_usbd_core_handler_call             0x00001690   Section        0  app_usbd.o(i.app_usbd_core_handler_call)
    app_usbd_core_handler_call               0x00001691   Thumb Code    10  app_usbd.o(i.app_usbd_core_handler_call)
    i.app_usbd_core_setup_data_handler_set   0x000016a0   Section        0  app_usbd_core.o(i.app_usbd_core_setup_data_handler_set)
    i.app_usbd_core_setup_data_transfer      0x000016c4   Section        0  app_usbd_core.o(i.app_usbd_core_setup_data_transfer)
    i.app_usbd_core_setup_req_handler        0x000016e4   Section        0  app_usbd_core.o(i.app_usbd_core_setup_req_handler)
    app_usbd_core_setup_req_handler          0x000016e5   Thumb Code   192  app_usbd_core.o(i.app_usbd_core_setup_req_handler)
    i.app_usbd_core_setup_rsp                0x000017a4   Section        0  app_usbd_core.o(i.app_usbd_core_setup_rsp)
    i.app_usbd_core_setup_transfer_buff_get  0x00001804   Section        0  app_usbd_core.o(i.app_usbd_core_setup_transfer_buff_get)
    i.app_usbd_disable                       0x00001814   Section        0  app_usbd.o(i.app_usbd_disable)
    i.app_usbd_enable                        0x00001828   Section        0  app_usbd.o(i.app_usbd_enable)
    i.app_usbd_endpoint_std_req_handle       0x00001840   Section        0  app_usbd.o(i.app_usbd_endpoint_std_req_handle)
    i.app_usbd_ep_call                       0x000018ac   Section        0  app_usbd.o(i.app_usbd_ep_call)
    i.app_usbd_ep_conf_access                0x000018c8   Section        0  app_usbd.o(i.app_usbd_ep_conf_access)
    app_usbd_ep_conf_access                  0x000018c9   Thumb Code    22  app_usbd.o(i.app_usbd_ep_conf_access)
    i.app_usbd_ep_instance_get               0x000018e4   Section        0  app_usbd.o(i.app_usbd_ep_instance_get)
    app_usbd_ep_instance_get                 0x000018e5   Thumb Code    10  app_usbd.o(i.app_usbd_ep_instance_get)
    i.app_usbd_ep_instance_set               0x000018ee   Section        0  app_usbd.o(i.app_usbd_ep_instance_set)
    app_usbd_ep_instance_set                 0x000018ef   Thumb Code    24  app_usbd.o(i.app_usbd_ep_instance_set)
    i.app_usbd_event_handler                 0x00001908   Section        0  app_usbd.o(i.app_usbd_event_handler)
    app_usbd_event_handler                   0x00001909   Thumb Code   116  app_usbd.o(i.app_usbd_event_handler)
    i.app_usbd_iface_call                    0x00001980   Section        0  app_usbd.o(i.app_usbd_iface_call)
    i.app_usbd_init                          0x000019c8   Section        0  app_usbd.o(i.app_usbd_init)
    i.app_usbd_interface_std_req_handle      0x00001a58   Section        0  app_usbd.o(i.app_usbd_interface_std_req_handle)
    i.app_usbd_setup_data_handled_transfer   0x00001a7c   Section        0  app_usbd_core.o(i.app_usbd_setup_data_handled_transfer)
    i.app_usbd_start                         0x00001a9c   Section        0  app_usbd.o(i.app_usbd_start)
    i.app_usbd_stop                          0x00001b04   Section        0  app_usbd.o(i.app_usbd_stop)
    i.app_usbd_string_desc_get               0x00001b28   Section        0  app_usbd_string_desc.o(i.app_usbd_string_desc_get)
    i.app_util_critical_region_enter         0x00001b50   Section        0  app_util_platform.o(i.app_util_critical_region_enter)
    i.app_util_critical_region_exit          0x00001b54   Section        0  app_util_platform.o(i.app_util_critical_region_exit)
    i.app_util_disable_irq                   0x00001b58   Section        0  app_util_platform.o(i.app_util_disable_irq)
    i.app_util_enable_irq                    0x00001b68   Section        0  app_util_platform.o(i.app_util_enable_irq)
    i.apply_config                           0x00001b7c   Section        0  nrf_drv_uart.o(i.apply_config)
    apply_config                             0x00001b7d   Thumb Code   162  nrf_drv_uart.o(i.apply_config)
    i.assert_nrf_callback                    0x00001c24   Section        0  nrf_assert.o(i.assert_nrf_callback)
    i.bit2ep                                 0x00001c3a   Section        0  nrf_drv_usbd.o(i.bit2ep)
    bit2ep                                   0x00001c3b   Thumb Code    16  nrf_drv_usbd.o(i.bit2ep)
    i.bsp_board_button_state_get             0x00001c4c   Section        0  boards.o(i.bsp_board_button_state_get)
    i.bsp_board_buttons_init                 0x00001c74   Section        0  boards.o(i.bsp_board_buttons_init)
    i.bsp_board_led_invert                   0x00001c98   Section        0  boards.o(i.bsp_board_led_invert)
    i.bsp_board_led_off                      0x00001cc4   Section        0  boards.o(i.bsp_board_led_off)
    i.bsp_board_led_on                       0x00001cd4   Section        0  boards.o(i.bsp_board_led_on)
    i.bsp_board_leds_init                    0x00001ce4   Section        0  boards.o(i.bsp_board_leds_init)
    i.bsp_board_leds_off                     0x00001d10   Section        0  boards.o(i.bsp_board_leds_off)
    i.buf_len_update                         0x00001d22   Section        0  nrf_log_backend_serial.o(i.buf_len_update)
    buf_len_update                           0x00001d23   Thumb Code    18  nrf_log_backend_serial.o(i.buf_len_update)
    i.buf_prealloc                           0x00001d34   Section        0  nrf_log_frontend.o(i.buf_prealloc)
    buf_prealloc                             0x00001d35   Thumb Code    84  nrf_log_frontend.o(i.buf_prealloc)
    i.buffer_is_empty                        0x00001d94   Section        0  nrf_log_frontend.o(i.buffer_is_empty)
    i.cdc_acm_event_handler                  0x00001da8   Section        0  app_usbd_cdc_acm.o(i.cdc_acm_event_handler)
    cdc_acm_event_handler                    0x00001da9   Thumb Code   118  app_usbd_cdc_acm.o(i.cdc_acm_event_handler)
    i.cdc_acm_get_descriptors                0x00001e1e   Section        0  app_usbd_cdc_acm.o(i.cdc_acm_get_descriptors)
    cdc_acm_get_descriptors                  0x00001e1f   Thumb Code     8  app_usbd_cdc_acm.o(i.cdc_acm_get_descriptors)
    i.cdc_acm_req_out_data_cb                0x00001e26   Section        0  app_usbd_cdc_acm.o(i.cdc_acm_req_out_data_cb)
    cdc_acm_req_out_data_cb                  0x00001e27   Thumb Code    38  app_usbd_cdc_acm.o(i.cdc_acm_req_out_data_cb)
    i.cdc_acm_user_ev_handler                0x00001e4c   Section        0  main.o(i.cdc_acm_user_ev_handler)
    cdc_acm_user_ev_handler                  0x00001e4d   Thumb Code   122  main.o(i.cdc_acm_user_ev_handler)
    i.channel_port_get                       0x00001ee4   Section        0  nrf_drv_gpiote.o(i.channel_port_get)
    channel_port_get                         0x00001ee5   Thumb Code    10  nrf_drv_gpiote.o(i.channel_port_get)
    i.class_event_handler                    0x00001ef4   Section        0  app_usbd.o(i.class_event_handler)
    class_event_handler                      0x00001ef5   Thumb Code     6  app_usbd.o(i.class_event_handler)
    i.clock_clk_started_notify               0x00001efc   Section        0  nrf_drv_clock.o(i.clock_clk_started_notify)
    clock_clk_started_notify                 0x00001efd   Thumb Code    34  nrf_drv_clock.o(i.clock_clk_started_notify)
    i.comm_ep_in_addr_get                    0x00001f24   Section        0  app_usbd_cdc_acm.o(i.comm_ep_in_addr_get)
    comm_ep_in_addr_get                      0x00001f25   Thumb Code    18  app_usbd_cdc_acm.o(i.comm_ep_in_addr_get)
    i.compare_reg_update                     0x00001f38   Section        0  app_timer.o(i.compare_reg_update)
    compare_reg_update                       0x00001f39   Thumb Code   160  app_timer.o(i.compare_reg_update)
    i.data_ep_in_addr_get                    0x00001fe4   Section        0  app_usbd_cdc_acm.o(i.data_ep_in_addr_get)
    data_ep_in_addr_get                      0x00001fe5   Thumb Code    18  app_usbd_cdc_acm.o(i.data_ep_in_addr_get)
    i.data_ep_out_addr_get                   0x00001ff6   Section        0  app_usbd_cdc_acm.o(i.data_ep_out_addr_get)
    data_ep_out_addr_get                     0x00001ff7   Thumb Code    18  app_usbd_cdc_acm.o(i.data_ep_out_addr_get)
    i.elapsed_ticks_acquire                  0x00002008   Section        0  app_timer.o(i.elapsed_ticks_acquire)
    elapsed_ticks_acquire                    0x00002009   Thumb Code    58  app_timer.o(i.elapsed_ticks_acquire)
    i.ep2bit                                 0x00002048   Section        0  nrf_drv_usbd.o(i.ep2bit)
    ep2bit                                   0x00002049   Thumb Code    12  nrf_drv_usbd.o(i.ep2bit)
    i.ep_state_access                        0x00002054   Section        0  nrf_drv_usbd.o(i.ep_state_access)
    ep_state_access                          0x00002055   Thumb Code    18  nrf_drv_usbd.o(i.ep_state_access)
    i.interrupts_enable                      0x0000206c   Section        0  nrf_drv_uart.o(i.interrupts_enable)
    interrupts_enable                        0x0000206d   Thumb Code   106  nrf_drv_uart.o(i.interrupts_enable)
    i.item_enqueue                           0x000020e4   Section        0  nrf_drv_clock.o(i.item_enqueue)
    item_enqueue                             0x000020e5   Thumb Code    22  nrf_drv_clock.o(i.item_enqueue)
    i.list_insertions_handler                0x000020fc   Section        0  app_timer.o(i.list_insertions_handler)
    list_insertions_handler                  0x000020fd   Thumb Code   234  app_timer.o(i.list_insertions_handler)
    i.main                                   0x000021f4   Section        0  main.o(i.main)
    i.nrf_atomic_u32_and                     0x00002378   Section        0  nrf_drv_usbd.o(i.nrf_atomic_u32_and)
    nrf_atomic_u32_and                       0x00002379   Thumb Code    12  nrf_drv_usbd.o(i.nrf_atomic_u32_and)
    i.nrf_bitmask_bit_is_set                 0x00002384   Section        0  nrf_drv_gpiote.o(i.nrf_bitmask_bit_is_set)
    nrf_bitmask_bit_is_set                   0x00002385   Thumb Code    16  nrf_drv_gpiote.o(i.nrf_bitmask_bit_is_set)
    i.nrf_clock_event_check                  0x00002394   Section        0  nrf_drv_clock.o(i.nrf_clock_event_check)
    nrf_clock_event_check                    0x00002395   Thumb Code    14  nrf_drv_clock.o(i.nrf_clock_event_check)
    i.nrf_clock_event_clear                  0x000023a2   Section        0  nrf_drv_clock.o(i.nrf_clock_event_clear)
    nrf_clock_event_clear                    0x000023a3   Thumb Code    16  nrf_drv_clock.o(i.nrf_clock_event_clear)
    i.nrf_clock_hf_is_running                0x000023b4   Section        0  nrf_drv_clock.o(i.nrf_clock_hf_is_running)
    nrf_clock_hf_is_running                  0x000023b5   Thumb Code    24  nrf_drv_clock.o(i.nrf_clock_hf_is_running)
    i.nrf_delay_us                           0x000023d0   Section        0  main.o(i.nrf_delay_us)
    nrf_delay_us                             0x000023d1   Thumb Code   132  main.o(i.nrf_delay_us)
    i.nrf_delay_us                           0x0000245c   Section        0  app_timer.o(i.nrf_delay_us)
    nrf_delay_us                             0x0000245d   Thumb Code   132  app_timer.o(i.nrf_delay_us)
    i.nrf_drv_clock_hfclk_is_running         0x000024e8   Section        0  nrf_drv_clock.o(i.nrf_drv_clock_hfclk_is_running)
    i.nrf_drv_clock_hfclk_request            0x000024f0   Section        0  nrf_drv_clock.o(i.nrf_drv_clock_hfclk_request)
    i.nrf_drv_clock_init                     0x00002548   Section        0  nrf_drv_clock.o(i.nrf_drv_clock_init)
    i.nrf_drv_clock_onIRQ                    0x0000258c   Section        0  nrf_drv_clock.o(i.nrf_drv_clock_onIRQ)
    i.nrf_drv_common_irq_disable             0x000025e4   Section        0  nrf_drv_uart.o(i.nrf_drv_common_irq_disable)
    nrf_drv_common_irq_disable               0x000025e5   Thumb Code    22  nrf_drv_uart.o(i.nrf_drv_common_irq_disable)
    i.nrf_drv_common_irq_enable              0x000025fa   Section        0  nrf_drv_common.o(i.nrf_drv_common_irq_enable)
    i.nrf_drv_get_IRQn                       0x00002632   Section        0  nrf_drv_uart.o(i.nrf_drv_get_IRQn)
    nrf_drv_get_IRQn                         0x00002633   Thumb Code     6  nrf_drv_uart.o(i.nrf_drv_get_IRQn)
    i.nrf_drv_is_in_RAM                      0x00002638   Section        0  nrf_drv_uart.o(i.nrf_drv_is_in_RAM)
    nrf_drv_is_in_RAM                        0x00002639   Thumb Code    16  nrf_drv_uart.o(i.nrf_drv_is_in_RAM)
    i.nrf_drv_power_init                     0x00002648   Section        0  nrf_drv_power.o(i.nrf_drv_power_init)
    i.nrf_drv_power_onIRQ                    0x00002698   Section        0  nrf_drv_power.o(i.nrf_drv_power_onIRQ)
    i.nrf_drv_power_usbevt_init              0x00002728   Section        0  nrf_drv_power.o(i.nrf_drv_power_usbevt_init)
    i.nrf_drv_power_usbevt_uninit            0x0000274c   Section        0  nrf_drv_power.o(i.nrf_drv_power_usbevt_uninit)
    i.nrf_drv_systick_delay_ticks            0x00002764   Section        0  nrf_drv_systick.o(i.nrf_drv_systick_delay_ticks)
    i.nrf_drv_systick_delay_us               0x00002778   Section        0  nrf_drv_systick.o(i.nrf_drv_systick_delay_us)
    i.nrf_drv_systick_init                   0x00002794   Section        0  nrf_drv_systick.o(i.nrf_drv_systick_init)
    i.nrf_drv_uart_init                      0x000027a4   Section        0  nrf_drv_uart.o(i.nrf_drv_uart_init)
    i.nrf_drv_uart_tx                        0x0000280c   Section        0  nrf_drv_uart.o(i.nrf_drv_uart_tx)
    i.nrf_drv_uart_tx_in_progress            0x00002918   Section        0  nrf_drv_uart.o(i.nrf_drv_uart_tx_in_progress)
    i.nrf_drv_uart_uninit                    0x00002930   Section        0  nrf_drv_uart.o(i.nrf_drv_uart_uninit)
    i.nrf_drv_usbd_consumer                  0x00002984   Section        0  nrf_drv_usbd.o(i.nrf_drv_usbd_consumer)
    i.nrf_drv_usbd_disable                   0x000029b4   Section        0  nrf_drv_usbd.o(i.nrf_drv_usbd_disable)
    i.nrf_drv_usbd_enable                    0x000029e8   Section        0  nrf_drv_usbd.o(i.nrf_drv_usbd_enable)
    i.nrf_drv_usbd_ep_enable                 0x00002a3c   Section        0  nrf_drv_usbd.o(i.nrf_drv_usbd_ep_enable)
    i.nrf_drv_usbd_ep_handled_transfer       0x00002ac8   Section        0  nrf_drv_usbd.o(i.nrf_drv_usbd_ep_handled_transfer)
    i.nrf_drv_usbd_ep_max_packet_size_get    0x00002b40   Section        0  nrf_drv_usbd.o(i.nrf_drv_usbd_ep_max_packet_size_get)
    i.nrf_drv_usbd_ep_max_packet_size_set    0x00002b4a   Section        0  nrf_drv_usbd.o(i.nrf_drv_usbd_ep_max_packet_size_set)
    i.nrf_drv_usbd_ep_stall                  0x00002b58   Section        0  nrf_drv_usbd.o(i.nrf_drv_usbd_ep_stall)
    i.nrf_drv_usbd_ep_stall_check            0x00002b70   Section        0  nrf_drv_usbd.o(i.nrf_drv_usbd_ep_stall_check)
    i.nrf_drv_usbd_ep_stall_clear            0x00002b74   Section        0  nrf_drv_usbd.o(i.nrf_drv_usbd_ep_stall_clear)
    i.nrf_drv_usbd_ep_status_get             0x00002b88   Section        0  nrf_drv_usbd.o(i.nrf_drv_usbd_ep_status_get)
    i.nrf_drv_usbd_ep_to_int                 0x00002bb0   Section        0  nrf_drv_usbd.o(i.nrf_drv_usbd_ep_to_int)
    nrf_drv_usbd_ep_to_int                   0x00002bb1   Thumb Code    24  nrf_drv_usbd.o(i.nrf_drv_usbd_ep_to_int)
    i.nrf_drv_usbd_ep_transfer               0x00002bcc   Section        0  nrf_drv_usbd.o(i.nrf_drv_usbd_ep_transfer)
    i.nrf_drv_usbd_epout_size_get            0x00002ca0   Section        0  nrf_drv_usbd.o(i.nrf_drv_usbd_epout_size_get)
    i.nrf_drv_usbd_feeder_buffer_get         0x00002cc4   Section        0  nrf_drv_usbd.o(i.nrf_drv_usbd_feeder_buffer_get)
    i.nrf_drv_usbd_feeder_flash              0x00002ccc   Section        0  nrf_drv_usbd.o(i.nrf_drv_usbd_feeder_flash)
    i.nrf_drv_usbd_feeder_flash_zlp          0x00002d08   Section        0  nrf_drv_usbd.o(i.nrf_drv_usbd_feeder_flash_zlp)
    i.nrf_drv_usbd_feeder_ram                0x00002d4c   Section        0  nrf_drv_usbd.o(i.nrf_drv_usbd_feeder_ram)
    i.nrf_drv_usbd_feeder_ram_zlp            0x00002d70   Section        0  nrf_drv_usbd.o(i.nrf_drv_usbd_feeder_ram_zlp)
    i.nrf_drv_usbd_init                      0x00002da8   Section        0  nrf_drv_usbd.o(i.nrf_drv_usbd_init)
    i.nrf_drv_usbd_is_enabled                0x00002e40   Section        0  nrf_drv_usbd.o(i.nrf_drv_usbd_is_enabled)
    i.nrf_drv_usbd_is_started                0x00002e54   Section        0  nrf_drv_usbd.o(i.nrf_drv_usbd_is_started)
    i.nrf_drv_usbd_last_setup_dir_get        0x00002e74   Section        0  nrf_drv_usbd.o(i.nrf_drv_usbd_last_setup_dir_get)
    i.nrf_drv_usbd_setup_clear               0x00002e80   Section        0  nrf_drv_usbd.o(i.nrf_drv_usbd_setup_clear)
    i.nrf_drv_usbd_setup_data_clear          0x00002e86   Section        0  nrf_drv_usbd.o(i.nrf_drv_usbd_setup_data_clear)
    i.nrf_drv_usbd_setup_get                 0x00002ea0   Section        0  nrf_drv_usbd.o(i.nrf_drv_usbd_setup_get)
    i.nrf_drv_usbd_setup_stall               0x00002ef0   Section        0  nrf_drv_usbd.o(i.nrf_drv_usbd_setup_stall)
    i.nrf_drv_usbd_start                     0x00002ef8   Section        0  nrf_drv_usbd.o(i.nrf_drv_usbd_start)
    i.nrf_drv_usbd_stop                      0x00002f28   Section        0  nrf_drv_usbd.o(i.nrf_drv_usbd_stop)
    i.nrf_drv_usbd_transfer_out_drop         0x00002f50   Section        0  nrf_drv_usbd.o(i.nrf_drv_usbd_transfer_out_drop)
    i.nrf_gpio_cfg                           0x00002f84   Section        0  boards.o(i.nrf_gpio_cfg)
    nrf_gpio_cfg                             0x00002f85   Thumb Code    50  boards.o(i.nrf_gpio_cfg)
    i.nrf_gpio_cfg                           0x00002fb6   Section        0  nrf_drv_uart.o(i.nrf_gpio_cfg)
    nrf_gpio_cfg                             0x00002fb7   Thumb Code    50  nrf_drv_uart.o(i.nrf_gpio_cfg)
    i.nrf_gpio_cfg_default                   0x00002fe8   Section        0  nrf_drv_uart.o(i.nrf_gpio_cfg_default)
    nrf_gpio_cfg_default                     0x00002fe9   Thumb Code    18  nrf_drv_uart.o(i.nrf_gpio_cfg_default)
    i.nrf_gpio_cfg_input                     0x00002ffa   Section        0  nrf_drv_uart.o(i.nrf_gpio_cfg_input)
    nrf_gpio_cfg_input                       0x00002ffb   Thumb Code    18  nrf_drv_uart.o(i.nrf_gpio_cfg_input)
    i.nrf_gpio_cfg_output                    0x0000300c   Section        0  nrf_drv_uart.o(i.nrf_gpio_cfg_output)
    nrf_gpio_cfg_output                      0x0000300d   Thumb Code    20  nrf_drv_uart.o(i.nrf_gpio_cfg_output)
    i.nrf_gpio_cfg_sense_set                 0x00003020   Section        0  nrf_drv_gpiote.o(i.nrf_gpio_cfg_sense_set)
    nrf_gpio_cfg_sense_set                   0x00003021   Thumb Code    48  nrf_drv_gpiote.o(i.nrf_gpio_cfg_sense_set)
    i.nrf_gpio_pin_port_decode               0x00003050   Section        0  boards.o(i.nrf_gpio_pin_port_decode)
    nrf_gpio_pin_port_decode                 0x00003051   Thumb Code    22  boards.o(i.nrf_gpio_pin_port_decode)
    i.nrf_gpio_pin_port_decode               0x0000306c   Section        0  nrf_drv_gpiote.o(i.nrf_gpio_pin_port_decode)
    nrf_gpio_pin_port_decode                 0x0000306d   Thumb Code    22  nrf_drv_gpiote.o(i.nrf_gpio_pin_port_decode)
    i.nrf_gpio_pin_port_decode               0x00003088   Section        0  nrf_drv_uart.o(i.nrf_gpio_pin_port_decode)
    nrf_gpio_pin_port_decode                 0x00003089   Thumb Code    22  nrf_drv_uart.o(i.nrf_gpio_pin_port_decode)
    i.nrf_gpio_pin_set                       0x000030a4   Section        0  nrf_drv_uart.o(i.nrf_gpio_pin_set)
    nrf_gpio_pin_set                         0x000030a5   Thumb Code    20  nrf_drv_uart.o(i.nrf_gpio_pin_set)
    i.nrf_gpio_pin_write                     0x000030b8   Section        0  boards.o(i.nrf_gpio_pin_write)
    nrf_gpio_pin_write                       0x000030b9   Thumb Code    38  boards.o(i.nrf_gpio_pin_write)
    i.nrf_gpio_ports_read                    0x000030e0   Section        0  nrf_drv_gpiote.o(i.nrf_gpio_ports_read)
    nrf_gpio_ports_read                      0x000030e1   Thumb Code    38  nrf_drv_gpiote.o(i.nrf_gpio_ports_read)
    i.nrf_gpiote_event_clear                 0x0000310c   Section        0  nrf_drv_gpiote.o(i.nrf_gpiote_event_clear)
    nrf_gpiote_event_clear                   0x0000310d   Thumb Code    16  nrf_drv_gpiote.o(i.nrf_gpiote_event_clear)
    i.nrf_gpiote_event_is_set                0x00003120   Section        0  nrf_drv_gpiote.o(i.nrf_gpiote_event_is_set)
    nrf_gpiote_event_is_set                  0x00003121   Thumb Code    12  nrf_drv_gpiote.o(i.nrf_gpiote_event_is_set)
    i.nrf_log_backend_hexdump_handler_get    0x00003130   Section        0  nrf_log_backend_serial.o(i.nrf_log_backend_hexdump_handler_get)
    i.nrf_log_backend_init                   0x00003138   Section        0  nrf_log_backend_serial.o(i.nrf_log_backend_init)
    i.nrf_log_backend_serial_hexdump_handler 0x000031a8   Section        0  nrf_log_backend_serial.o(i.nrf_log_backend_serial_hexdump_handler)
    nrf_log_backend_serial_hexdump_handler   0x000031a9   Thumb Code   302  nrf_log_backend_serial.o(i.nrf_log_backend_serial_hexdump_handler)
    i.nrf_log_backend_serial_std_handler     0x000032d6   Section        0  nrf_log_backend_serial.o(i.nrf_log_backend_serial_std_handler)
    nrf_log_backend_serial_std_handler       0x000032d7   Thumb Code   276  nrf_log_backend_serial.o(i.nrf_log_backend_serial_std_handler)
    i.nrf_log_backend_std_handler_get        0x000033ec   Section        0  nrf_log_backend_serial.o(i.nrf_log_backend_std_handler_get)
    i.nrf_log_blocking_backend_set           0x000033f4   Section        0  nrf_log_frontend.o(i.nrf_log_blocking_backend_set)
    i.nrf_log_frontend_dequeue               0x000033fc   Section        0  nrf_log_frontend.o(i.nrf_log_frontend_dequeue)
    i.nrf_log_frontend_init                  0x0000352c   Section        0  nrf_log_frontend.o(i.nrf_log_frontend_init)
    i.nrf_log_frontend_std_0                 0x00003540   Section        0  nrf_log_frontend.o(i.nrf_log_frontend_std_0)
    i.nrf_log_frontend_std_1                 0x0000358c   Section        0  nrf_log_frontend.o(i.nrf_log_frontend_std_1)
    i.nrf_log_frontend_std_2                 0x000035e4   Section        0  nrf_log_frontend.o(i.nrf_log_frontend_std_2)
    i.nrf_log_handlers_set                   0x0000364c   Section        0  nrf_log_frontend.o(i.nrf_log_handlers_set)
    i.nrf_log_init                           0x0000365c   Section        0  nrf_log_frontend.o(i.nrf_log_init)
    i.nrf_power_event_get_and_clear          0x00003680   Section        0  nrf_drv_power.o(i.nrf_power_event_get_and_clear)
    nrf_power_event_get_and_clear            0x00003681   Thumb Code    20  nrf_drv_power.o(i.nrf_power_event_get_and_clear)
    i.nrf_uart_event_check                   0x00003694   Section        0  nrf_drv_uart.o(i.nrf_uart_event_check)
    nrf_uart_event_check                     0x00003695   Thumb Code    10  nrf_drv_uart.o(i.nrf_uart_event_check)
    i.nrf_uart_event_clear                   0x0000369e   Section        0  nrf_drv_uart.o(i.nrf_uart_event_clear)
    nrf_uart_event_clear                     0x0000369f   Thumb Code    12  nrf_drv_uart.o(i.nrf_uart_event_clear)
    i.nrf_uart_int_enable_check              0x000036aa   Section        0  nrf_drv_uart.o(i.nrf_uart_int_enable_check)
    nrf_uart_int_enable_check                0x000036ab   Thumb Code    12  nrf_drv_uart.o(i.nrf_uart_int_enable_check)
    i.nrf_uarte_event_check                  0x000036b6   Section        0  nrf_drv_uart.o(i.nrf_uarte_event_check)
    nrf_uarte_event_check                    0x000036b7   Thumb Code    10  nrf_drv_uart.o(i.nrf_uarte_event_check)
    i.nrf_uarte_event_clear                  0x000036c0   Section        0  nrf_drv_uart.o(i.nrf_uarte_event_clear)
    nrf_uarte_event_clear                    0x000036c1   Thumb Code    12  nrf_drv_uart.o(i.nrf_uarte_event_clear)
    i.nrf_usbd_dtoggle_get                   0x000036cc   Section        0  app_usbd.o(i.nrf_usbd_dtoggle_get)
    nrf_usbd_dtoggle_get                     0x000036cd   Thumb Code    18  app_usbd.o(i.nrf_usbd_dtoggle_get)
    i.nrf_usbd_dtoggle_set                   0x000036e4   Section        0  app_usbd.o(i.nrf_usbd_dtoggle_set)
    nrf_usbd_dtoggle_set                     0x000036e5   Thumb Code    18  app_usbd.o(i.nrf_usbd_dtoggle_set)
    i.nrf_usbd_dtoggle_set                   0x000036fc   Section        0  app_usbd_core.o(i.nrf_usbd_dtoggle_set)
    nrf_usbd_dtoggle_set                     0x000036fd   Thumb Code    18  app_usbd_core.o(i.nrf_usbd_dtoggle_set)
    i.nrf_usbd_ep_is_stall                   0x00003714   Section        0  nrf_drv_usbd.o(i.nrf_usbd_ep_is_stall)
    nrf_usbd_ep_is_stall                     0x00003715   Thumb Code    40  nrf_drv_usbd.o(i.nrf_usbd_ep_is_stall)
    i.nrf_usbd_epin_dma_handler              0x00003740   Section        0  nrf_drv_usbd.o(i.nrf_usbd_epin_dma_handler)
    nrf_usbd_epin_dma_handler                0x00003741   Thumb Code    54  nrf_drv_usbd.o(i.nrf_usbd_epin_dma_handler)
    i.nrf_usbd_epout_dma_handler             0x0000377c   Section        0  nrf_drv_usbd.o(i.nrf_usbd_epout_dma_handler)
    nrf_usbd_epout_dma_handler               0x0000377d   Thumb Code    90  nrf_drv_usbd.o(i.nrf_usbd_epout_dma_handler)
    i.nrf_usbd_event_check                   0x000037e4   Section        0  nrf_drv_usbd.o(i.nrf_usbd_event_check)
    nrf_usbd_event_check                     0x000037e5   Thumb Code    12  nrf_drv_usbd.o(i.nrf_usbd_event_check)
    i.nrf_usbd_event_clear                   0x000037f4   Section        0  nrf_drv_usbd.o(i.nrf_usbd_event_clear)
    nrf_usbd_event_clear                     0x000037f5   Thumb Code    18  nrf_drv_usbd.o(i.nrf_usbd_event_clear)
    i.nrf_usbd_eventcause_clear              0x0000380c   Section        0  nrf_drv_usbd.o(i.nrf_usbd_eventcause_clear)
    nrf_usbd_eventcause_clear                0x0000380d   Thumb Code    14  nrf_drv_usbd.o(i.nrf_usbd_eventcause_clear)
    i.nrf_usbd_task_trigger                  0x00003820   Section        0  app_usbd_core.o(i.nrf_usbd_task_trigger)
    nrf_usbd_task_trigger                    0x00003821   Thumb Code    18  app_usbd_core.o(i.nrf_usbd_task_trigger)
    i.nrf_usbd_task_trigger                  0x00003838   Section        0  nrf_drv_usbd.o(i.nrf_usbd_task_trigger)
    nrf_usbd_task_trigger                    0x00003839   Thumb Code    18  nrf_drv_usbd.o(i.nrf_usbd_task_trigger)
    i.pins_to_default                        0x00003850   Section        0  nrf_drv_uart.o(i.pins_to_default)
    pins_to_default                          0x00003851   Thumb Code   114  nrf_drv_uart.o(i.pins_to_default)
    i.power_usb_event_handler                0x000038c8   Section        0  main.o(i.power_usb_event_handler)
    power_usb_event_handler                  0x000038c9   Thumb Code    78  main.o(i.power_usb_event_handler)
    i.requestTx                              0x00003984   Section        0  main.o(i.requestTx)
    i.rtc1_stop                              0x000039f0   Section        0  app_timer.o(i.rtc1_stop)
    rtc1_stop                                0x000039f1   Thumb Code    52  app_timer.o(i.rtc1_stop)
    i.rx_byte                                0x00003a2c   Section        0  nrf_drv_uart.o(i.rx_byte)
    rx_byte                                  0x00003a2d   Thumb Code    50  nrf_drv_uart.o(i.rx_byte)
    i.rx_done_event                          0x00003a5e   Section        0  nrf_drv_uart.o(i.rx_done_event)
    rx_done_event                            0x00003a5f   Thumb Code    24  nrf_drv_uart.o(i.rx_done_event)
    i.serial_is_busy                         0x00003a78   Section        0  nrf_log_backend_serial.o(i.serial_is_busy)
    serial_is_busy                           0x00003a79   Thumb Code     6  nrf_log_backend_serial.o(i.serial_is_busy)
    i.serial_tx                              0x00003a84   Section        0  nrf_log_backend_serial.o(i.serial_tx)
    serial_tx                                0x00003a85   Thumb Code    34  nrf_log_backend_serial.o(i.serial_tx)
    i.setup_data_handler_empty               0x00003ab0   Section        0  app_usbd_core.o(i.setup_data_handler_empty)
    setup_data_handler_empty                 0x00003ab1   Thumb Code     4  app_usbd_core.o(i.setup_data_handler_empty)
    i.setup_event_handler                    0x00003ab4   Section        0  app_usbd_cdc_acm.o(i.setup_event_handler)
    setup_event_handler                      0x00003ab5   Thumb Code   140  app_usbd_cdc_acm.o(i.setup_event_handler)
    i.setup_req_class_out                    0x00003b40   Section        0  app_usbd_cdc_acm.o(i.setup_req_class_out)
    setup_req_class_out                      0x00003b41   Thumb Code   168  app_usbd_cdc_acm.o(i.setup_req_class_out)
    i.setup_req_get_descriptor               0x00003bec   Section        0  app_usbd_core.o(i.setup_req_get_descriptor)
    setup_req_get_descriptor                 0x00003bed   Thumb Code   210  app_usbd_core.o(i.setup_req_get_descriptor)
    i.setup_req_std_in                       0x00003ccc   Section        0  app_usbd_core.o(i.setup_req_std_in)
    setup_req_std_in                         0x00003ccd   Thumb Code   112  app_usbd_core.o(i.setup_req_std_in)
    i.setup_req_std_out                      0x00003d40   Section        0  app_usbd_core.o(i.setup_req_std_out)
    setup_req_std_out                        0x00003d41   Thumb Code    94  app_usbd_core.o(i.setup_req_std_out)
    i.setup_req_std_set_configuration        0x00003da4   Section        0  app_usbd_core.o(i.setup_req_std_set_configuration)
    setup_req_std_set_configuration          0x00003da5   Thumb Code   194  app_usbd_core.o(i.setup_req_std_set_configuration)
    i.timer_list_handler                     0x00003e70   Section        0  app_timer.o(i.timer_list_handler)
    timer_list_handler                       0x00003e71   Thumb Code   122  app_timer.o(i.timer_list_handler)
    i.timer_list_insert                      0x00003ef0   Section        0  app_timer.o(i.timer_list_insert)
    timer_list_insert                        0x00003ef1   Thumb Code    56  app_timer.o(i.timer_list_insert)
    i.timer_list_remove                      0x00003f2c   Section        0  app_timer.o(i.timer_list_remove)
    timer_list_remove                        0x00003f2d   Thumb Code    88  app_timer.o(i.timer_list_remove)
    i.timer_timeouts_check                   0x00003f8c   Section        0  app_timer.o(i.timer_timeouts_check)
    timer_timeouts_check                     0x00003f8d   Thumb Code   106  app_timer.o(i.timer_timeouts_check)
    i.timestamp_process                      0x00004000   Section        0  nrf_log_backend_serial.o(i.timestamp_process)
    timestamp_process                        0x00004001   Thumb Code    44  nrf_log_backend_serial.o(i.timestamp_process)
    i.tx_byte                                0x00004034   Section        0  nrf_drv_uart.o(i.tx_byte)
    tx_byte                                  0x00004035   Thumb Code    32  nrf_drv_uart.o(i.tx_byte)
    i.tx_done_event                          0x00004054   Section        0  nrf_drv_uart.o(i.tx_done_event)
    tx_done_event                            0x00004055   Thumb Code    28  nrf_drv_uart.o(i.tx_done_event)
    i.uart_event_handler                     0x00004070   Section        0  nrf_log_backend_serial.o(i.uart_event_handler)
    uart_event_handler                       0x00004071   Thumb Code    12  nrf_log_backend_serial.o(i.uart_event_handler)
    i.uart_irq_handler                       0x00004080   Section        0  nrf_drv_uart.o(i.uart_irq_handler)
    uart_irq_handler                         0x00004081   Thumb Code   286  nrf_drv_uart.o(i.uart_irq_handler)
    i.uarte_irq_handler                      0x0000419e   Section        0  nrf_drv_uart.o(i.uarte_irq_handler)
    uarte_irq_handler                        0x0000419f   Thumb Code   240  nrf_drv_uart.o(i.uarte_irq_handler)
    i.usb_core_ep0_handler_check             0x00004290   Section        0  app_usbd_core.o(i.usb_core_ep0_handler_check)
    usb_core_ep0_handler_check               0x00004291   Thumb Code    12  app_usbd_core.o(i.usb_core_ep0_handler_check)
    i.usbd_descriptor_conf_feeder            0x000042a0   Section        0  app_usbd_core.o(i.usbd_descriptor_conf_feeder)
    usbd_descriptor_conf_feeder              0x000042a1   Thumb Code   182  app_usbd_core.o(i.usbd_descriptor_conf_feeder)
    i.usbd_dmareq_process                    0x00004358   Section        0  nrf_drv_usbd.o(i.usbd_dmareq_process)
    usbd_dmareq_process                      0x00004359   Thumb Code   368  nrf_drv_usbd.o(i.usbd_dmareq_process)
    i.usbd_drv_ep_abort                      0x000044e0   Section        0  nrf_drv_usbd.o(i.usbd_drv_ep_abort)
    i.usbd_ep_abort                          0x000044e4   Section        0  nrf_drv_usbd.o(i.usbd_ep_abort)
    usbd_ep_abort                            0x000044e5   Thumb Code   186  nrf_drv_usbd.o(i.usbd_ep_abort)
    i.usbd_ep_abort_all                      0x000045a8   Section        0  nrf_drv_usbd.o(i.usbd_ep_abort_all)
    usbd_ep_abort_all                        0x000045a9   Thumb Code    58  nrf_drv_usbd.o(i.usbd_ep_abort_all)
    i.usbd_ep_data_handler                   0x000045e8   Section        0  nrf_drv_usbd.o(i.usbd_ep_data_handler)
    usbd_ep_data_handler                     0x000045e9   Thumb Code    56  nrf_drv_usbd.o(i.usbd_ep_data_handler)
    i.usbd_int_rise                          0x00004628   Section        0  nrf_drv_usbd.o(i.usbd_int_rise)
    usbd_int_rise                            0x00004629   Thumb Code    10  nrf_drv_usbd.o(i.usbd_int_rise)
    i.usbd_user_ev_handler                   0x00004638   Section        0  main.o(i.usbd_user_ev_handler)
    usbd_user_ev_handler                     0x00004639   Thumb Code    34  main.o(i.usbd_user_ev_handler)
    i.user_event_handler                     0x0000465c   Section        0  app_usbd.o(i.user_event_handler)
    user_event_handler                       0x0000465d   Thumb Code    12  app_usbd.o(i.user_event_handler)
    i.user_event_handler                     0x0000466c   Section        0  app_usbd_cdc_acm.o(i.user_event_handler)
    user_event_handler                       0x0000466d   Thumb Code    10  app_usbd_cdc_acm.o(i.user_event_handler)
    .constdata                               0x00004676   Section       66  main.o(.constdata)
    m_cdc_acm_class_descriptors              0x00004676   Data          66  main.o(.constdata)
    .constdata                               0x000046b8   Section       40  main.o(.constdata)
    m_usbd_config                            0x000046b8   Data           4  main.o(.constdata)
    config                                   0x000046bc   Data           4  main.o(.constdata)
    .constdata                               0x000046e0   Section        8  boards.o(.constdata)
    m_board_led_list                         0x000046e0   Data           4  boards.o(.constdata)
    m_board_btn_list                         0x000046e4   Data           4  boards.o(.constdata)
    .constdata                               0x000046e8   Section       24  app_usbd.o(.constdata)
    m_default_conf                           0x000046fc   Data           4  app_usbd.o(.constdata)
    .constdata                               0x00004700   Section       43  app_usbd_core.o(.constdata)
    m_setup_data_handler_empty_desc          0x00004700   Data           8  app_usbd_core.o(.constdata)
    usbd_descriptor_feeder_desc              0x00004708   Data           8  app_usbd_core.o(.constdata)
    m_device_dsc                             0x00004710   Data          18  app_usbd_core.o(.constdata)
    m_configuration_dsc                      0x00004722   Data           9  app_usbd_core.o(.constdata)
    .constdata                               0x0000472c   Section        8  app_usbd_core.o(.constdata)
    m_core_methods                           0x0000472c   Data           8  app_usbd_core.o(.constdata)
    .constdata                               0x00004734   Section       16  app_usbd_core.o(.constdata)
    .constdata                               0x00004744   Section        4  app_usbd_string_desc.o(.constdata)
    <Data2>                                  0x00004744   Data           4  app_usbd_string_desc.o(.constdata)
    .constdata                               0x00004748   Section       42  app_usbd_string_desc.o(.constdata)
    <Data4>                                  0x00004748   Data          42  app_usbd_string_desc.o(.constdata)
    .constdata                               0x00004772   Section       38  app_usbd_string_desc.o(.constdata)
    <Data6>                                  0x00004772   Data          38  app_usbd_string_desc.o(.constdata)
    .constdata                               0x00004798   Section       14  app_usbd_string_desc.o(.constdata)
    <Data8>                                  0x00004798   Data          14  app_usbd_string_desc.o(.constdata)
    .constdata                               0x000047a6   Section        5  app_usbd_string_desc.o(.constdata)
    m_string_translation                     0x000047a6   Data           5  app_usbd_string_desc.o(.constdata)
    .constdata                               0x000047ac   Section        8  nrf_drv_gpiote.o(.constdata)
    .constdata                               0x000047b4   Section        1  nrf_drv_power.o(.constdata)
    m_drv_power_config_default               0x000047b4   Data           1  nrf_drv_power.o(.constdata)
    .constdata                               0x000047b8   Section      206  nrf_drv_usbd.o(.constdata)
    m_isr                                    0x000047e8   Data         104  nrf_drv_usbd.o(.constdata)
    epin_endev                               0x00004850   Data          18  nrf_drv_usbd.o(.constdata)
    epout_endev                              0x00004862   Data          18  nrf_drv_usbd.o(.constdata)
    epin_bitpos                              0x00004874   Data           9  nrf_drv_usbd.o(.constdata)
    epout_bitpos                             0x0000487d   Data           9  nrf_drv_usbd.o(.constdata)
    .constdata                               0x00004888   Section        8  app_usbd_cdc_acm.o(.constdata)
    .constdata                               0x00004890   Section       20  app_usbd_cdc_acm.o(.constdata)
    .constdata                               0x000048a4   Section       32  nrf_log_backend_serial.o(.constdata)
    .constdata                               0x000048c4   Section       36  nrf_log_frontend.o(.constdata)
    .constdata                               0x000048e8   Section      129  ctype_o.o(.constdata)
    .constdata                               0x0000496c   Section        4  ctype_o.o(.constdata)
    table                                    0x0000496c   Data           4  ctype_o.o(.constdata)
    .conststring                             0x00004970   Section       11  nrf_log_frontend.o(.conststring)
    .data                                    0x20000000   Section       20  main.o(.data)
    m_usb_connected                          0x20000000   Data           1  main.o(.data)
    .data                                    0x20000014   Section       12  app_usbd.o(.data)
    m_p_first_cinst                          0x20000014   Data           4  app_usbd.o(.data)
    m_p_first_sof_cinst                      0x20000018   Data           4  app_usbd.o(.data)
    m_current_conf                           0x2000001c   Data           4  app_usbd.o(.data)
    .data                                    0x20000020   Section       16  app_usbd_core.o(.data)
    app_usbd_state                           0x20000020   Data           1  app_usbd_core.o(.data)
    m_device_features_state                  0x20000021   Data           1  app_usbd_core.o(.data)
    m_rwu_counter                            0x20000022   Data           1  app_usbd_core.o(.data)
    m_rwu_pending                            0x20000024   Data           4  app_usbd_core.o(.data)
    m_ep0_handler_desc                       0x20000028   Data           8  app_usbd_core.o(.data)
    .data                                    0x20000030   Section        8  app_usbd_core.o(.data)
    app_usbd_core_inst_data                  0x20000030   Data           8  app_usbd_core.o(.data)
    .data                                    0x20000038   Section       20  app_usbd_string_desc.o(.data)
    m_string_dsc                             0x20000038   Data          20  app_usbd_string_desc.o(.data)
    .data                                    0x2000004c   Section       16  nrf_drv_power.o(.data)
    m_initialized                            0x2000004c   Data           1  nrf_drv_power.o(.data)
    m_pofwarn_handler                        0x20000050   Data           4  nrf_drv_power.o(.data)
    m_sleepevt_handler                       0x20000054   Data           4  nrf_drv_power.o(.data)
    m_usbevt_handler                         0x20000058   Data           4  nrf_drv_power.o(.data)
    .data                                    0x2000005c   Section       20  nrf_drv_usbd.o(.data)
    m_drv_state                              0x2000005c   Data           1  nrf_drv_usbd.o(.data)
    m_last_setup_dir                         0x2000005d   Data           1  nrf_drv_usbd.o(.data)
    m_dma_pending                            0x2000005e   Data           1  nrf_drv_usbd.o(.data)
    m_event_handler                          0x20000060   Data           4  nrf_drv_usbd.o(.data)
    m_ep_ready                               0x20000064   Data           4  nrf_drv_usbd.o(.data)
    m_ep_dma_waiting                         0x20000068   Data           4  nrf_drv_usbd.o(.data)
    m_simulated_dataepstatus                 0x2000006c   Data           4  nrf_drv_usbd.o(.data)
    .data                                    0x20000070   Section       20  app_timer.o(.data)
    m_ticks_elapsed_q_read_ind               0x20000070   Data           1  app_timer.o(.data)
    m_ticks_elapsed_q_write_ind              0x20000071   Data           1  app_timer.o(.data)
    m_rtc1_running                           0x20000072   Data           1  app_timer.o(.data)
    m_rtc1_reset                             0x20000073   Data           1  app_timer.o(.data)
    mp_timer_id_head                         0x20000074   Data           4  app_timer.o(.data)
    m_ticks_latest                           0x20000078   Data           4  app_timer.o(.data)
    m_ticks_elapsed                          0x2000007c   Data           8  app_timer.o(.data)
    .data                                    0x20000084   Section        4  app_util_platform.o(.data)
    m_in_critical_region                     0x20000084   Data           4  app_util_platform.o(.data)
    .data                                    0x20000088   Section       12  nrf_log_backend_serial.o(.data)
    m_initialized                            0x20000088   Data           1  nrf_log_backend_serial.o(.data)
    m_blocking_mode                          0x20000089   Data           1  nrf_log_backend_serial.o(.data)
    m_rx_done                                0x2000008a   Data           1  nrf_log_backend_serial.o(.data)
    m_uart                                   0x2000008c   Data           8  nrf_log_backend_serial.o(.data)
    .data                                    0x20000094   Section        4  nrf_log_frontend.o(.data)
    m_overflow_info                          0x20000094   Data           4  nrf_log_frontend.o(.data)
    .data                                    0x20000098   Section        4  system_nrf52840.o(.data)
    __tagsym$$used                           0x20000098   Number         0  system_nrf52840.o(.data)
    .bss                                     0x2000009c   Section       32  main.o(.bss)
    m_app_cdc_acm_data                       0x2000009c   Data          32  main.o(.bss)
    .bss                                     0x200000bc   Section     2082  main.o(.bss)
    m_rx_buffer                              0x200000bc   Data        1024  main.o(.bss)
    m_tx_buffer                              0x200004bc   Data        1024  main.o(.bss)
    .bss                                     0x200008e0   Section      144  app_usbd.o(.bss)
    m_epin_conf                              0x200008e0   Data          72  app_usbd.o(.bss)
    m_epout_conf                             0x20000928   Data          72  app_usbd.o(.bss)
    .bss                                     0x20000970   Section       80  app_usbd_core.o(.bss)
    m_setup_transfer_buff                    0x20000970   Data          64  app_usbd_core.o(.bss)
    m_descriptor_conf_feed_data              0x200009b0   Data          16  app_usbd_core.o(.bss)
    .bss                                     0x200009c0   Section       20  nrf_drv_clock.o(.bss)
    m_clock_cb                               0x200009c0   Data          20  nrf_drv_clock.o(.bss)
    .bss                                     0x200009d4   Section      104  nrf_drv_gpiote.o(.bss)
    m_cb                                     0x200009d4   Data         104  nrf_drv_gpiote.o(.bss)
    .bss                                     0x20000a3c   Section       32  nrf_drv_uart.o(.bss)
    m_cb                                     0x20000a3c   Data          32  nrf_drv_uart.o(.bss)
    .bss                                     0x20000a5c   Section      568  nrf_drv_usbd.o(.bss)
    m_ep_state                               0x20000a5c   Data         288  nrf_drv_usbd.o(.bss)
    m_tx_buffer                              0x20000c54   Data          64  nrf_drv_usbd.o(.bss)
    .bss                                     0x20000c94   Section      268  app_timer.o(.bss)
    m_op_queue                               0x20000c94   Data         268  app_timer.o(.bss)
    .bss                                     0x20000da0   Section      256  nrf_log_backend_serial.o(.bss)
    m_uart_buffer                            0x20000da0   Data         256  nrf_log_backend_serial.o(.bss)
    .bss                                     0x20000ea0   Section     1048  nrf_log_frontend.o(.bss)
    m_log_data                               0x20000ea0   Data        1048  nrf_log_frontend.o(.bss)
    STACK                                    0x200012b8   Section     8192  arm_startup_nrf52840.o(STACK)

    Global Symbols

    Symbol Name                              Value     Ov Type        Size  Object(Section)

    BuildAttributes$$THM_ISAv4$E$P$D$K$B$S$7EM$VFPi3$EXTD16$VFPS$VFMA$PE$A:L22UL41UL21$X:L11$S22US41US21$IEEE1$IW$USESV6$~STKCKD$USESV7$~SHL$OSPACE$ROPI$EBA8$MICROLIB$REQ8$PRES8$EABIv2 0x00000000   Number         0  anon$$obj.o ABSOLUTE
    __ARM_use_no_argv                        0x00000000   Number         0  main.o ABSOLUTE
    __Vectors                                0x00000000   Data           4  arm_startup_nrf52840.o(RESET)
    _printf_a                                0x00000000   Number         0  stubs.o ABSOLUTE
    _printf_c                                0x00000000   Number         0  stubs.o ABSOLUTE
    _printf_charcount                        0x00000000   Number         0  stubs.o ABSOLUTE
    _printf_d                                0x00000000   Number         0  stubs.o ABSOLUTE
    _printf_e                                0x00000000   Number         0  stubs.o ABSOLUTE
    _printf_f                                0x00000000   Number         0  stubs.o ABSOLUTE
    _printf_flags                            0x00000000   Number         0  stubs.o ABSOLUTE
    _printf_fp_dec                           0x00000000   Number         0  stubs.o ABSOLUTE
    _printf_fp_hex                           0x00000000   Number         0  stubs.o ABSOLUTE
    _printf_g                                0x00000000   Number         0  stubs.o ABSOLUTE
    _printf_i                                0x00000000   Number         0  stubs.o ABSOLUTE
    _printf_int_dec                          0x00000000   Number         0  stubs.o ABSOLUTE
    _printf_l                                0x00000000   Number         0  stubs.o ABSOLUTE
    _printf_lc                               0x00000000   Number         0  stubs.o ABSOLUTE
    _printf_ll                               0x00000000   Number         0  stubs.o ABSOLUTE
    _printf_lld                              0x00000000   Number         0  stubs.o ABSOLUTE
    _printf_lli                              0x00000000   Number         0  stubs.o ABSOLUTE
    _printf_llo                              0x00000000   Number         0  stubs.o ABSOLUTE
    _printf_llu                              0x00000000   Number         0  stubs.o ABSOLUTE
    _printf_llx                              0x00000000   Number         0  stubs.o ABSOLUTE
    _printf_longlong_dec                     0x00000000   Number         0  stubs.o ABSOLUTE
    _printf_longlong_hex                     0x00000000   Number         0  stubs.o ABSOLUTE
    _printf_longlong_oct                     0x00000000   Number         0  stubs.o ABSOLUTE
    _printf_ls                               0x00000000   Number         0  stubs.o ABSOLUTE
    _printf_mbtowc                           0x00000000   Number         0  stubs.o ABSOLUTE
    _printf_n                                0x00000000   Number         0  stubs.o ABSOLUTE
    _printf_o                                0x00000000   Number         0  stubs.o ABSOLUTE
    _printf_p                                0x00000000   Number         0  stubs.o ABSOLUTE
    _printf_percent                          0x00000000   Number         0  stubs.o ABSOLUTE
    _printf_pre_padding                      0x00000000   Number         0  stubs.o ABSOLUTE
    _printf_return_value                     0x00000000   Number         0  stubs.o ABSOLUTE
    _printf_s                                0x00000000   Number         0  stubs.o ABSOLUTE
    _printf_sizespec                         0x00000000   Number         0  stubs.o ABSOLUTE
    _printf_str                              0x00000000   Number         0  stubs.o ABSOLUTE
    _printf_truncate_signed                  0x00000000   Number         0  stubs.o ABSOLUTE
    _printf_truncate_unsigned                0x00000000   Number         0  stubs.o ABSOLUTE
    _printf_u                                0x00000000   Number         0  stubs.o ABSOLUTE
    _printf_wc                               0x00000000   Number         0  stubs.o ABSOLUTE
    _printf_wctomb                           0x00000000   Number         0  stubs.o ABSOLUTE
    _printf_widthprec                        0x00000000   Number         0  stubs.o ABSOLUTE
    _printf_x                                0x00000000   Number         0  stubs.o ABSOLUTE
    __cpp_initialize__aeabi_                  - Undefined Weak Reference
    __cxa_finalize                            - Undefined Weak Reference
    __decompress                              - Undefined Weak Reference
    _clock_init                               - Undefined Weak Reference
    _microlib_exit                            - Undefined Weak Reference
    __Vectors_End                            0x00000200   Data           0  arm_startup_nrf52840.o(RESET)
    __Vectors_Size                           0x00000200   Number         0  arm_startup_nrf52840.o ABSOLUTE
    __main                                   0x00000201   Thumb Code     0  entry.o(.ARM.Collect$$$$00000000)
    _main_stk                                0x00000201   Thumb Code     0  entry2.o(.ARM.Collect$$$$00000001)
    _main_scatterload                        0x00000205   Thumb Code     0  entry5.o(.ARM.Collect$$$$00000004)
    __main_after_scatterload                 0x00000209   Thumb Code     0  entry5.o(.ARM.Collect$$$$00000004)
    _main_clock                              0x00000209   Thumb Code     0  entry7b.o(.ARM.Collect$$$$00000008)
    _main_cpp_init                           0x00000209   Thumb Code     0  entry8b.o(.ARM.Collect$$$$0000000A)
    _main_init                               0x00000209   Thumb Code     0  entry9a.o(.ARM.Collect$$$$0000000B)
    __rt_final_cpp                           0x00000211   Thumb Code     0  entry10a.o(.ARM.Collect$$$$0000000D)
    __rt_final_exit                          0x00000211   Thumb Code     0  entry11a.o(.ARM.Collect$$$$0000000F)
    __asm___15_app_usbd_core_c_a97d2587__nrf_atomic_internal_mov 0x00000215   Thumb Code    24  app_usbd_core.o(.emb_text)
    __asm___15_app_usbd_core_c_a97d2587__nrf_atomic_internal_orr 0x0000022d   Thumb Code    26  app_usbd_core.o(.emb_text)
    __asm___15_app_usbd_core_c_a97d2587__nrf_atomic_internal_and 0x00000247   Thumb Code    26  app_usbd_core.o(.emb_text)
    __asm___15_app_usbd_core_c_a97d2587__nrf_atomic_internal_eor 0x00000261   Thumb Code    26  app_usbd_core.o(.emb_text)
    __asm___15_app_usbd_core_c_a97d2587__nrf_atomic_internal_add 0x0000027b   Thumb Code    26  app_usbd_core.o(.emb_text)
    __asm___15_app_usbd_core_c_a97d2587__nrf_atomic_internal_sub 0x00000295   Thumb Code    26  app_usbd_core.o(.emb_text)
    __asm___14_nrf_drv_usbd_c_f1d4739e__nrf_atomic_internal_mov 0x000002b1   Thumb Code    24  nrf_drv_usbd.o(.emb_text)
    __asm___14_nrf_drv_usbd_c_f1d4739e__nrf_atomic_internal_orr 0x000002c9   Thumb Code    26  nrf_drv_usbd.o(.emb_text)
    __asm___14_nrf_drv_usbd_c_f1d4739e__nrf_atomic_internal_and 0x000002e3   Thumb Code    26  nrf_drv_usbd.o(.emb_text)
    __asm___14_nrf_drv_usbd_c_f1d4739e__nrf_atomic_internal_eor 0x000002fd   Thumb Code    26  nrf_drv_usbd.o(.emb_text)
    __asm___14_nrf_drv_usbd_c_f1d4739e__nrf_atomic_internal_add 0x00000317   Thumb Code    26  nrf_drv_usbd.o(.emb_text)
    __asm___14_nrf_drv_usbd_c_f1d4739e__nrf_atomic_internal_sub 0x00000331   Thumb Code    26  nrf_drv_usbd.o(.emb_text)
    HardFault_Handler                        0x0000034d   Thumb Code    40  hardfault_handler_keil.o(.emb_text)
    Reset_Handler                            0x00000381   Thumb Code     8  arm_startup_nrf52840.o(.text)
    NMI_Handler                              0x00000389   Thumb Code     2  arm_startup_nrf52840.o(.text)
    MemoryManagement_Handler                 0x0000038d   Thumb Code     2  arm_startup_nrf52840.o(.text)
    BusFault_Handler                         0x0000038f   Thumb Code     2  arm_startup_nrf52840.o(.text)
    UsageFault_Handler                       0x00000391   Thumb Code     2  arm_startup_nrf52840.o(.text)
    SVC_Handler                              0x00000393   Thumb Code     2  arm_startup_nrf52840.o(.text)
    DebugMon_Handler                         0x00000395   Thumb Code     2  arm_startup_nrf52840.o(.text)
    PendSV_Handler                           0x00000397   Thumb Code     2  arm_startup_nrf52840.o(.text)
    SysTick_Handler                          0x00000399   Thumb Code     2  arm_startup_nrf52840.o(.text)
    CCM_AAR_IRQHandler                       0x0000039b   Thumb Code     0  arm_startup_nrf52840.o(.text)
    COMP_LPCOMP_IRQHandler                   0x0000039b   Thumb Code     0  arm_startup_nrf52840.o(.text)
    CRYPTOCELL_IRQHandler                    0x0000039b   Thumb Code     0  arm_startup_nrf52840.o(.text)
    ECB_IRQHandler                           0x0000039b   Thumb Code     0  arm_startup_nrf52840.o(.text)
    FPU_IRQHandler                           0x0000039b   Thumb Code     0  arm_startup_nrf52840.o(.text)
    I2S_IRQHandler                           0x0000039b   Thumb Code     0  arm_startup_nrf52840.o(.text)
    MWU_IRQHandler                           0x0000039b   Thumb Code     0  arm_startup_nrf52840.o(.text)
    NFCT_IRQHandler                          0x0000039b   Thumb Code     0  arm_startup_nrf52840.o(.text)
    PDM_IRQHandler                           0x0000039b   Thumb Code     0  arm_startup_nrf52840.o(.text)
    PWM0_IRQHandler                          0x0000039b   Thumb Code     0  arm_startup_nrf52840.o(.text)
    PWM1_IRQHandler                          0x0000039b   Thumb Code     0  arm_startup_nrf52840.o(.text)
    PWM2_IRQHandler                          0x0000039b   Thumb Code     0  arm_startup_nrf52840.o(.text)
    PWM3_IRQHandler                          0x0000039b   Thumb Code     0  arm_startup_nrf52840.o(.text)
    QDEC_IRQHandler                          0x0000039b   Thumb Code     0  arm_startup_nrf52840.o(.text)
    QSPI_IRQHandler                          0x0000039b   Thumb Code     0  arm_startup_nrf52840.o(.text)
    RADIO_IRQHandler                         0x0000039b   Thumb Code     0  arm_startup_nrf52840.o(.text)
    RNG_IRQHandler                           0x0000039b   Thumb Code     0  arm_startup_nrf52840.o(.text)
    RTC0_IRQHandler                          0x0000039b   Thumb Code     0  arm_startup_nrf52840.o(.text)
    RTC2_IRQHandler                          0x0000039b   Thumb Code     0  arm_startup_nrf52840.o(.text)
    SAADC_IRQHandler                         0x0000039b   Thumb Code     0  arm_startup_nrf52840.o(.text)
    SPIM0_SPIS0_TWIM0_TWIS0_SPI0_TWI0_IRQHandler 0x0000039b   Thumb Code     0  arm_startup_nrf52840.o(.text)
    SPIM1_SPIS1_TWIM1_TWIS1_SPI1_TWI1_IRQHandler 0x0000039b   Thumb Code     0  arm_startup_nrf52840.o(.text)
    SPIM2_SPIS2_SPI2_IRQHandler              0x0000039b   Thumb Code     0  arm_startup_nrf52840.o(.text)
    SPIM3_IRQHandler                         0x0000039b   Thumb Code     0  arm_startup_nrf52840.o(.text)
    SWI1_EGU1_IRQHandler                     0x0000039b   Thumb Code     0  arm_startup_nrf52840.o(.text)
    SWI2_EGU2_IRQHandler                     0x0000039b   Thumb Code     0  arm_startup_nrf52840.o(.text)
    SWI3_EGU3_IRQHandler                     0x0000039b   Thumb Code     0  arm_startup_nrf52840.o(.text)
    SWI4_EGU4_IRQHandler                     0x0000039b   Thumb Code     0  arm_startup_nrf52840.o(.text)
    SWI5_EGU5_IRQHandler                     0x0000039b   Thumb Code     0  arm_startup_nrf52840.o(.text)
    TEMP_IRQHandler                          0x0000039b   Thumb Code     0  arm_startup_nrf52840.o(.text)
    TIMER0_IRQHandler                        0x0000039b   Thumb Code     0  arm_startup_nrf52840.o(.text)
    TIMER1_IRQHandler                        0x0000039b   Thumb Code     0  arm_startup_nrf52840.o(.text)
    TIMER2_IRQHandler                        0x0000039b   Thumb Code     0  arm_startup_nrf52840.o(.text)
    TIMER3_IRQHandler                        0x0000039b   Thumb Code     0  arm_startup_nrf52840.o(.text)
    TIMER4_IRQHandler                        0x0000039b   Thumb Code     0  arm_startup_nrf52840.o(.text)
    UARTE1_IRQHandler                        0x0000039b   Thumb Code     0  arm_startup_nrf52840.o(.text)
    WDT_IRQHandler                           0x0000039b   Thumb Code     0  arm_startup_nrf52840.o(.text)
    __aeabi_uldivmod                         0x000003a5   Thumb Code    98  uldiv.o(.text)
    __rt_ctype_table                         0x00000409   Thumb Code     4  ctype_o.o(.text)
    __aeabi_memcpy                           0x00000411   Thumb Code    36  memcpya.o(.text)
    __aeabi_memcpy4                          0x00000411   Thumb Code     0  memcpya.o(.text)
    __aeabi_memcpy8                          0x00000411   Thumb Code     0  memcpya.o(.text)
    __aeabi_memset                           0x00000435   Thumb Code    14  memseta.o(.text)
    __aeabi_memset4                          0x00000435   Thumb Code     0  memseta.o(.text)
    __aeabi_memset8                          0x00000435   Thumb Code     0  memseta.o(.text)
    __aeabi_memclr                           0x00000443   Thumb Code     4  memseta.o(.text)
    __aeabi_memclr4                          0x00000443   Thumb Code     0  memseta.o(.text)
    __aeabi_memclr8                          0x00000443   Thumb Code     0  memseta.o(.text)
    _memset$wrapper                          0x00000447   Thumb Code    18  memseta.o(.text)
    strlen                                   0x00000459   Thumb Code    14  strlen.o(.text)
    __aeabi_llsl                             0x00000467   Thumb Code    30  llshl.o(.text)
    _ll_shift_l                              0x00000467   Thumb Code     0  llshl.o(.text)
    __aeabi_llsr                             0x00000485   Thumb Code    32  llushr.o(.text)
    _ll_ushift_r                             0x00000485   Thumb Code     0  llushr.o(.text)
    __scatterload                            0x000004a5   Thumb Code    28  init.o(.text)
    __scatterload_rt2                        0x000004a5   Thumb Code     0  init.o(.text)
    GPIOTE_IRQHandler                        0x000004c9   Thumb Code   444  nrf_drv_gpiote.o(i.GPIOTE_IRQHandler)
    HardFault_c_handler                      0x0000068d   Thumb Code    30  hardfault_implementation.o(i.HardFault_c_handler)
    HardFault_process                        0x000006d1   Thumb Code    26  hardfault_implementation.o(i.HardFault_process)
    POWER_CLOCK_IRQHandler                   0x00000737   Thumb Code    14  nrf_drv_common.o(i.POWER_CLOCK_IRQHandler)
    RTC1_IRQHandler                          0x00000745   Thumb Code    32  app_timer.o(i.RTC1_IRQHandler)
    SWI0_EGU0_IRQHandler                     0x00000769   Thumb Code     4  app_timer.o(i.SWI0_EGU0_IRQHandler)
    SystemInit                               0x0000076d   Thumb Code   432  system_nrf52840.o(i.SystemInit)
    UARTE0_UART0_IRQHandler                  0x00000955   Thumb Code    20  nrf_drv_uart.o(i.UARTE0_UART0_IRQHandler)
    USBD_IRQHandler                          0x00000971   Thumb Code   336  nrf_drv_usbd.o(i.USBD_IRQHandler)
    __0snprintf$8                            0x00000e21   Thumb Code    36  printf8.o(i.__0snprintf$8)
    __1snprintf$8                            0x00000e21   Thumb Code     0  printf8.o(i.__0snprintf$8)
    __2snprintf                              0x00000e21   Thumb Code     0  printf8.o(i.__0snprintf$8)
    __0sprintf$8                             0x00000e49   Thumb Code    34  printf8.o(i.__0sprintf$8)
    __1sprintf$8                             0x00000e49   Thumb Code     0  printf8.o(i.__0sprintf$8)
    __2sprintf                               0x00000e49   Thumb Code     0  printf8.o(i.__0sprintf$8)
    __scatterload_copy                       0x00000e71   Thumb Code    14  handlers.o(i.__scatterload_copy)
    __scatterload_null                       0x00000e7f   Thumb Code     2  handlers.o(i.__scatterload_null)
    __scatterload_zeroinit                   0x00000e81   Thumb Code    14  handlers.o(i.__scatterload_zeroinit)
    app_error_fault_handler                  0x00001315   Thumb Code    54  app_error_weak.o(i.app_error_fault_handler)
    app_error_handler_bare                   0x00001381   Thumb Code    22  app_error.o(i.app_error_handler_bare)
    app_usbd_all_call                        0x00001399   Thumb Code    26  app_usbd.o(i.app_usbd_all_call)
    app_usbd_all_until_served_call           0x000013b9   Thumb Code    32  app_usbd.o(i.app_usbd_all_until_served_call)
    app_usbd_cdc_acm_read                    0x000013dd   Thumb Code    40  app_usbd_cdc_acm.o(i.app_usbd_cdc_acm_read)
    app_usbd_cdc_acm_rx_size                 0x00001405   Thumb Code    22  app_usbd_cdc_acm.o(i.app_usbd_cdc_acm_rx_size)
    app_usbd_cdc_acm_write                   0x0000141b   Thumb Code    40  app_usbd_cdc_acm.o(i.app_usbd_cdc_acm_write)
    app_usbd_class_append                    0x00001445   Thumb Code   136  app_usbd.o(i.app_usbd_class_append)
    app_usbd_class_descriptor_find           0x000014d5   Thumb Code    68  app_usbd.o(i.app_usbd_class_descriptor_find)
    app_usbd_class_first_get                 0x00001519   Thumb Code     6  app_usbd.o(i.app_usbd_class_first_get)
    app_usbd_class_sof_register              0x00001571   Thumb Code    20  app_usbd.o(i.app_usbd_class_sof_register)
    app_usbd_class_sof_unregister            0x00001589   Thumb Code    38  app_usbd.o(i.app_usbd_class_sof_unregister)
    app_usbd_core_ep_transfer                0x000015b5   Thumb Code    20  app_usbd_core.o(i.app_usbd_core_ep_transfer)
    app_usbd_core_setup_data_handler_set     0x000016a1   Thumb Code    32  app_usbd_core.o(i.app_usbd_core_setup_data_handler_set)
    app_usbd_core_setup_data_transfer        0x000016c5   Thumb Code    28  app_usbd_core.o(i.app_usbd_core_setup_data_transfer)
    app_usbd_core_setup_rsp                  0x000017a5   Thumb Code    90  app_usbd_core.o(i.app_usbd_core_setup_rsp)
    app_usbd_core_setup_transfer_buff_get    0x00001805   Thumb Code    10  app_usbd_core.o(i.app_usbd_core_setup_transfer_buff_get)
    app_usbd_disable                         0x00001815   Thumb Code    20  app_usbd.o(i.app_usbd_disable)
    app_usbd_enable                          0x00001829   Thumb Code    20  app_usbd.o(i.app_usbd_enable)
    app_usbd_endpoint_std_req_handle         0x00001841   Thumb Code   108  app_usbd.o(i.app_usbd_endpoint_std_req_handle)
    app_usbd_ep_call                         0x000018ad   Thumb Code    28  app_usbd.o(i.app_usbd_ep_call)
    app_usbd_iface_call                      0x00001981   Thumb Code    66  app_usbd.o(i.app_usbd_iface_call)
    app_usbd_init                            0x000019c9   Thumb Code   124  app_usbd.o(i.app_usbd_init)
    app_usbd_interface_std_req_handle        0x00001a59   Thumb Code    34  app_usbd.o(i.app_usbd_interface_std_req_handle)
    app_usbd_setup_data_handled_transfer     0x00001a7d   Thumb Code    28  app_usbd_core.o(i.app_usbd_setup_data_handled_transfer)
    app_usbd_start                           0x00001a9d   Thumb Code    92  app_usbd.o(i.app_usbd_start)
    app_usbd_stop                            0x00001b05   Thumb Code    32  app_usbd.o(i.app_usbd_stop)
    app_usbd_string_desc_get                 0x00001b29   Thumb Code    30  app_usbd_string_desc.o(i.app_usbd_string_desc_get)
    app_util_critical_region_enter           0x00001b51   Thumb Code     4  app_util_platform.o(i.app_util_critical_region_enter)
    app_util_critical_region_exit            0x00001b55   Thumb Code     4  app_util_platform.o(i.app_util_critical_region_exit)
    app_util_disable_irq                     0x00001b59   Thumb Code    12  app_util_platform.o(i.app_util_disable_irq)
    app_util_enable_irq                      0x00001b69   Thumb Code    14  app_util_platform.o(i.app_util_enable_irq)
    assert_nrf_callback                      0x00001c25   Thumb Code    22  nrf_assert.o(i.assert_nrf_callback)
    bsp_board_button_state_get               0x00001c4d   Thumb Code    36  boards.o(i.bsp_board_button_state_get)
    bsp_board_buttons_init                   0x00001c75   Thumb Code    32  boards.o(i.bsp_board_buttons_init)
    bsp_board_led_invert                     0x00001c99   Thumb Code    40  boards.o(i.bsp_board_led_invert)
    bsp_board_led_off                        0x00001cc5   Thumb Code    10  boards.o(i.bsp_board_led_off)
    bsp_board_led_on                         0x00001cd5   Thumb Code    10  boards.o(i.bsp_board_led_on)
    bsp_board_leds_init                      0x00001ce5   Thumb Code    38  boards.o(i.bsp_board_leds_init)
    bsp_board_leds_off                       0x00001d11   Thumb Code    18  boards.o(i.bsp_board_leds_off)
    buffer_is_empty                          0x00001d95   Thumb Code    16  nrf_log_frontend.o(i.buffer_is_empty)
    main                                     0x000021f5   Thumb Code   238  main.o(i.main)
    nrf_drv_clock_hfclk_is_running           0x000024e9   Thumb Code     6  nrf_drv_clock.o(i.nrf_drv_clock_hfclk_is_running)
    nrf_drv_clock_hfclk_request              0x000024f1   Thumb Code    82  nrf_drv_clock.o(i.nrf_drv_clock_hfclk_request)
    nrf_drv_clock_init                       0x00002549   Thumb Code    58  nrf_drv_clock.o(i.nrf_drv_clock_init)
    nrf_drv_clock_onIRQ                      0x0000258d   Thumb Code    84  nrf_drv_clock.o(i.nrf_drv_clock_onIRQ)
    nrf_drv_common_irq_enable                0x000025fb   Thumb Code    56  nrf_drv_common.o(i.nrf_drv_common_irq_enable)
    nrf_drv_power_init                       0x00002649   Thumb Code    68  nrf_drv_power.o(i.nrf_drv_power_init)
    nrf_drv_power_onIRQ                      0x00002699   Thumb Code   138  nrf_drv_power.o(i.nrf_drv_power_onIRQ)
    nrf_drv_power_usbevt_init                0x00002729   Thumb Code    32  nrf_drv_power.o(i.nrf_drv_power_usbevt_init)
    nrf_drv_power_usbevt_uninit              0x0000274d   Thumb Code    20  nrf_drv_power.o(i.nrf_drv_power_usbevt_uninit)
    nrf_drv_systick_delay_ticks              0x00002765   Thumb Code    20  nrf_drv_systick.o(i.nrf_drv_systick_delay_ticks)
    nrf_drv_systick_delay_us                 0x00002779   Thumb Code    18  nrf_drv_systick.o(i.nrf_drv_systick_delay_us)
    nrf_drv_systick_init                     0x00002795   Thumb Code    16  nrf_drv_systick.o(i.nrf_drv_systick_init)
    nrf_drv_uart_init                        0x000027a5   Thumb Code    98  nrf_drv_uart.o(i.nrf_drv_uart_init)
    nrf_drv_uart_tx                          0x0000280d   Thumb Code   262  nrf_drv_uart.o(i.nrf_drv_uart_tx)
    nrf_drv_uart_tx_in_progress              0x00002919   Thumb Code    18  nrf_drv_uart.o(i.nrf_drv_uart_tx_in_progress)
    nrf_drv_uart_uninit                      0x00002931   Thumb Code    74  nrf_drv_uart.o(i.nrf_drv_uart_uninit)
    nrf_drv_usbd_consumer                    0x00002985   Thumb Code    48  nrf_drv_usbd.o(i.nrf_drv_usbd_consumer)
    nrf_drv_usbd_disable                     0x000029b5   Thumb Code    40  nrf_drv_usbd.o(i.nrf_drv_usbd_disable)
    nrf_drv_usbd_enable                      0x000029e9   Thumb Code    70  nrf_drv_usbd.o(i.nrf_drv_usbd_enable)
    nrf_drv_usbd_ep_enable                   0x00002a3d   Thumb Code   128  nrf_drv_usbd.o(i.nrf_drv_usbd_ep_enable)
    nrf_drv_usbd_ep_handled_transfer         0x00002ac9   Thumb Code   116  nrf_drv_usbd.o(i.nrf_drv_usbd_ep_handled_transfer)
    nrf_drv_usbd_ep_max_packet_size_get      0x00002b41   Thumb Code    10  nrf_drv_usbd.o(i.nrf_drv_usbd_ep_max_packet_size_get)
    nrf_drv_usbd_ep_max_packet_size_set      0x00002b4b   Thumb Code    12  nrf_drv_usbd.o(i.nrf_drv_usbd_ep_max_packet_size_set)
    nrf_drv_usbd_ep_stall                    0x00002b59   Thumb Code    18  nrf_drv_usbd.o(i.nrf_drv_usbd_ep_stall)
    nrf_drv_usbd_ep_stall_check              0x00002b71   Thumb Code     4  nrf_drv_usbd.o(i.nrf_drv_usbd_ep_stall_check)
    nrf_drv_usbd_ep_stall_clear              0x00002b75   Thumb Code    14  nrf_drv_usbd.o(i.nrf_drv_usbd_ep_stall_clear)
    nrf_drv_usbd_ep_status_get               0x00002b89   Thumb Code    40  nrf_drv_usbd.o(i.nrf_drv_usbd_ep_status_get)
    nrf_drv_usbd_ep_transfer                 0x00002bcd   Thumb Code   184  nrf_drv_usbd.o(i.nrf_drv_usbd_ep_transfer)
    nrf_drv_usbd_epout_size_get              0x00002ca1   Thumb Code    26  nrf_drv_usbd.o(i.nrf_drv_usbd_epout_size_get)
    nrf_drv_usbd_feeder_buffer_get           0x00002cc5   Thumb Code     4  nrf_drv_usbd.o(i.nrf_drv_usbd_feeder_buffer_get)
    nrf_drv_usbd_feeder_flash                0x00002ccd   Thumb Code    56  nrf_drv_usbd.o(i.nrf_drv_usbd_feeder_flash)
    nrf_drv_usbd_feeder_flash_zlp            0x00002d09   Thumb Code    64  nrf_drv_usbd.o(i.nrf_drv_usbd_feeder_flash_zlp)
    nrf_drv_usbd_feeder_ram                  0x00002d4d   Thumb Code    36  nrf_drv_usbd.o(i.nrf_drv_usbd_feeder_ram)
    nrf_drv_usbd_feeder_ram_zlp              0x00002d71   Thumb Code    54  nrf_drv_usbd.o(i.nrf_drv_usbd_feeder_ram_zlp)
    nrf_drv_usbd_init                        0x00002da9   Thumb Code   148  nrf_drv_usbd.o(i.nrf_drv_usbd_init)
    nrf_drv_usbd_is_enabled                  0x00002e41   Thumb Code    16  nrf_drv_usbd.o(i.nrf_drv_usbd_is_enabled)
    nrf_drv_usbd_is_started                  0x00002e55   Thumb Code    28  nrf_drv_usbd.o(i.nrf_drv_usbd_is_started)
    nrf_drv_usbd_last_setup_dir_get          0x00002e75   Thumb Code     6  nrf_drv_usbd.o(i.nrf_drv_usbd_last_setup_dir_get)
    nrf_drv_usbd_setup_clear                 0x00002e81   Thumb Code     6  nrf_drv_usbd.o(i.nrf_drv_usbd_setup_clear)
    nrf_drv_usbd_setup_data_clear            0x00002e87   Thumb Code    26  nrf_drv_usbd.o(i.nrf_drv_usbd_setup_data_clear)
    nrf_drv_usbd_setup_get                   0x00002ea1   Thumb Code    76  nrf_drv_usbd.o(i.nrf_drv_usbd_setup_get)
    nrf_drv_usbd_setup_stall                 0x00002ef1   Thumb Code     6  nrf_drv_usbd.o(i.nrf_drv_usbd_setup_stall)
    nrf_drv_usbd_start                       0x00002ef9   Thumb Code    34  nrf_drv_usbd.o(i.nrf_drv_usbd_start)
    nrf_drv_usbd_stop                        0x00002f29   Thumb Code    30  nrf_drv_usbd.o(i.nrf_drv_usbd_stop)
    nrf_drv_usbd_transfer_out_drop           0x00002f51   Thumb Code    48  nrf_drv_usbd.o(i.nrf_drv_usbd_transfer_out_drop)
    nrf_log_backend_hexdump_handler_get      0x00003131   Thumb Code     4  nrf_log_backend_serial.o(i.nrf_log_backend_hexdump_handler_get)
    nrf_log_backend_init                     0x00003139   Thumb Code   100  nrf_log_backend_serial.o(i.nrf_log_backend_init)
    nrf_log_backend_std_handler_get          0x000033ed   Thumb Code     4  nrf_log_backend_serial.o(i.nrf_log_backend_std_handler_get)
    nrf_log_blocking_backend_set             0x000033f5   Thumb Code     6  nrf_log_frontend.o(i.nrf_log_blocking_backend_set)
    nrf_log_frontend_dequeue                 0x000033fd   Thumb Code   298  nrf_log_frontend.o(i.nrf_log_frontend_dequeue)
    nrf_log_frontend_init                    0x0000352d   Thumb Code    16  nrf_log_frontend.o(i.nrf_log_frontend_init)
    nrf_log_frontend_std_0                   0x00003541   Thumb Code    68  nrf_log_frontend.o(i.nrf_log_frontend_std_0)
    nrf_log_frontend_std_1                   0x0000358d   Thumb Code    80  nrf_log_frontend.o(i.nrf_log_frontend_std_1)
    nrf_log_frontend_std_2                   0x000035e5   Thumb Code    96  nrf_log_frontend.o(i.nrf_log_frontend_std_2)
    nrf_log_handlers_set                     0x0000364d   Thumb Code    10  nrf_log_frontend.o(i.nrf_log_handlers_set)
    nrf_log_init                             0x0000365d   Thumb Code    36  nrf_log_frontend.o(i.nrf_log_init)
    requestTx                                0x00003985   Thumb Code    50  main.o(i.requestTx)
    usbd_drv_ep_abort                        0x000044e1   Thumb Code     4  nrf_drv_usbd.o(i.usbd_drv_ep_abort)
    m_app_cdc_acm                            0x000046c0   Data          32  main.o(.constdata)
    app_usbd_core_inst                       0x00004734   Data          16  app_usbd_core.o(.constdata)
    app_usbd_cdc_acm_class_methods           0x00004888   Data           8  app_usbd_cdc_acm.o(.constdata)
    __ctype_table                            0x000048e8   Data         129  ctype_o.o(.constdata)
    Region$$Table$$Base                      0x0000497c   Number         0  anon$$obj.o(Region$$Table)
    Region$$Table$$Limit                     0x0000499c   Number         0  anon$$obj.o(Region$$Table)
    countTx                                  0x20000004   Data           4  main.o(.data)
    countRx                                  0x20000008   Data           4  main.o(.data)
    countRequestTx                           0x2000000c   Data           4  main.o(.data)
    countRequestRx                           0x20000010   Data           4  main.o(.data)
    SystemCoreClock                          0x20000098   Data           4  system_nrf52840.o(.data)
    g_extern_serial_number                   0x200008bc   Data          34  main.o(.bss)
    m_ep_feeder_state                        0x20000b7c   Data         108  nrf_drv_usbd.o(.bss)
    m_ep_consumer_state                      0x20000be8   Data         108  nrf_drv_usbd.o(.bss)
    STACK$$Base                              0x200012b8   Number         0  arm_startup_nrf52840.o(STACK)
    STACK$$Limit                             0x200032b8   Number         0  arm_startup_nrf52840.o(STACK)
    __initial_sp                             0x200032b8   Data           0  arm_startup_nrf52840.o(STACK)



==============================================================================

Memory Map of the image

  Image Entry point : 0x00000201

  Load Region LR_IROM1 (Base: 0x00000000, Size: 0x00004a38, Max: 0x00100000, ABSOLUTE)

    Execution Region ER_IROM1 (Base: 0x00000000, Size: 0x0000499c, Max: 0x00100000, ABSOLUTE)

    Base Addr    Size         Type   Attr      Idx    E Section Name        Object

    0x00000000   0x00000200   Data   RO         3664    RESET               arm_startup_nrf52840.o
    0x00000200   0x00000000   Code   RO         3705  * .ARM.Collect$$$$00000000  mc_w.l(entry.o)
    0x00000200   0x00000004   Code   RO         4009    .ARM.Collect$$$$00000001  mc_w.l(entry2.o)
    0x00000204   0x00000004   Code   RO         4012    .ARM.Collect$$$$00000004  mc_w.l(entry5.o)
    0x00000208   0x00000000   Code   RO         4014    .ARM.Collect$$$$00000008  mc_w.l(entry7b.o)
    0x00000208   0x00000000   Code   RO         4016    .ARM.Collect$$$$0000000A  mc_w.l(entry8b.o)
    0x00000208   0x00000008   Code   RO         4017    .ARM.Collect$$$$0000000B  mc_w.l(entry9a.o)
    0x00000210   0x00000000   Code   RO         4019    .ARM.Collect$$$$0000000D  mc_w.l(entry10a.o)
    0x00000210   0x00000000   Code   RO         4021    .ARM.Collect$$$$0000000F  mc_w.l(entry11a.o)
    0x00000210   0x00000004   Code   RO         4010    .ARM.Collect$$$$00002712  mc_w.l(entry2.o)
    0x00000214   0x0000009a   Code   RO          783    .emb_text           app_usbd_core.o
    0x000002ae   0x00000002   PAD
    0x000002b0   0x0000009a   Code   RO         1881    .emb_text           nrf_drv_usbd.o
    0x0000034a   0x00000002   PAD
    0x0000034c   0x00000034   Code   RO         3168    .emb_text           hardfault_handler_keil.o
    0x00000380   0x00000024   Code   RO         3665    .text               arm_startup_nrf52840.o
    0x000003a4   0x00000062   Code   RO         3708    .text               mc_w.l(uldiv.o)
    0x00000406   0x00000002   PAD
    0x00000408   0x00000008   Code   RO         3710    .text               mc_w.l(ctype_o.o)
    0x00000410   0x00000024   Code   RO         3738    .text               mc_w.l(memcpya.o)
    0x00000434   0x00000024   Code   RO         3740    .text               mc_w.l(memseta.o)
    0x00000458   0x0000000e   Code   RO         3742    .text               mc_w.l(strlen.o)
    0x00000466   0x0000001e   Code   RO         4028    .text               mc_w.l(llshl.o)
    0x00000484   0x00000020   Code   RO         4030    .text               mc_w.l(llushr.o)
    0x000004a4   0x00000024   Code   RO         4043    .text               mc_w.l(init.o)
    0x000004c8   0x000001c4   Code   RO         1215    i.GPIOTE_IRQHandler  nrf_drv_gpiote.o
    0x0000068c   0x00000044   Code   RO         3190    i.HardFault_c_handler  hardfault_implementation.o
    0x000006d0   0x00000024   Code   RO         3191    i.HardFault_process  hardfault_implementation.o
    0x000006f4   0x00000016   Code   RO         2739    i.NVIC_ClearPendingIRQ  app_timer.o
    0x0000070a   0x00000016   Code   RO         2740    i.NVIC_EnableIRQ    app_timer.o
    0x00000720   0x00000016   Code   RO         2741    i.NVIC_SetPendingIRQ  app_timer.o
    0x00000736   0x0000000e   Code   RO         1161    i.POWER_CLOCK_IRQHandler  nrf_drv_common.o
    0x00000744   0x00000024   Code   RO         2743    i.RTC1_IRQHandler   app_timer.o
    0x00000768   0x00000004   Code   RO         2744    i.SWI0_EGU0_IRQHandler  app_timer.o
    0x0000076c   0x000001e8   Code   RO         3673    i.SystemInit        system_nrf52840.o
    0x00000954   0x0000001c   Code   RO         1633    i.UARTE0_UART0_IRQHandler  nrf_drv_uart.o
    0x00000970   0x00000160   Code   RO         1882    i.USBD_IRQHandler   nrf_drv_usbd.o
    0x00000ad0   0x00000002   Code   RO         1883    i.USBD_ISR_AccessFault  nrf_drv_usbd.o
    0x00000ad2   0x00000002   PAD
    0x00000ad4   0x0000005c   Code   RO         1884    i.USBD_ISR_EpDataStatus  nrf_drv_usbd.o
    0x00000b30   0x00000044   Code   RO         1885    i.USBD_ISR_Event    nrf_drv_usbd.o
    0x00000b74   0x0000008c   Code   RO         1886    i.USBD_ISR_Setup    nrf_drv_usbd.o
    0x00000c00   0x0000001c   Code   RO         1887    i.USBD_ISR_SetupData  nrf_drv_usbd.o
    0x00000c1c   0x0000003c   Code   RO         1888    i.USBD_ISR_Sof      nrf_drv_usbd.o
    0x00000c58   0x00000034   Code   RO         1889    i.USBD_ISR_Started  nrf_drv_usbd.o
    0x00000c8c   0x00000024   Code   RO         1890    i.USBD_ISR_Usbreset  nrf_drv_usbd.o
    0x00000cb0   0x00000038   Code   RO         1891    i.USBD_ISR_dma_epin0  nrf_drv_usbd.o
    0x00000ce8   0x00000006   Code   RO         1892    i.USBD_ISR_dma_epin1  nrf_drv_usbd.o
    0x00000cee   0x00000006   Code   RO         1893    i.USBD_ISR_dma_epin2  nrf_drv_usbd.o
    0x00000cf4   0x00000006   Code   RO         1894    i.USBD_ISR_dma_epin3  nrf_drv_usbd.o
    0x00000cfa   0x00000006   Code   RO         1895    i.USBD_ISR_dma_epin4  nrf_drv_usbd.o
    0x00000d00   0x00000006   Code   RO         1896    i.USBD_ISR_dma_epin5  nrf_drv_usbd.o
    0x00000d06   0x00000006   Code   RO         1897    i.USBD_ISR_dma_epin6  nrf_drv_usbd.o
    0x00000d0c   0x00000006   Code   RO         1898    i.USBD_ISR_dma_epin7  nrf_drv_usbd.o
    0x00000d12   0x00000002   PAD
    0x00000d14   0x0000004c   Code   RO         1899    i.USBD_ISR_dma_epin8  nrf_drv_usbd.o
    0x00000d60   0x00000048   Code   RO         1900    i.USBD_ISR_dma_epout0  nrf_drv_usbd.o
    0x00000da8   0x00000006   Code   RO         1901    i.USBD_ISR_dma_epout1  nrf_drv_usbd.o
    0x00000dae   0x00000006   Code   RO         1902    i.USBD_ISR_dma_epout2  nrf_drv_usbd.o
    0x00000db4   0x00000006   Code   RO         1903    i.USBD_ISR_dma_epout3  nrf_drv_usbd.o
    0x00000dba   0x00000006   Code   RO         1904    i.USBD_ISR_dma_epout4  nrf_drv_usbd.o
    0x00000dc0   0x00000006   Code   RO         1905    i.USBD_ISR_dma_epout5  nrf_drv_usbd.o
    0x00000dc6   0x00000006   Code   RO         1906    i.USBD_ISR_dma_epout6  nrf_drv_usbd.o
    0x00000dcc   0x00000006   Code   RO         1907    i.USBD_ISR_dma_epout7  nrf_drv_usbd.o
    0x00000dd2   0x00000002   PAD
    0x00000dd4   0x0000004c   Code   RO         1908    i.USBD_ISR_dma_epout8  nrf_drv_usbd.o
    0x00000e20   0x00000028   Code   RO         3956    i.__0snprintf$8     mc_w.l(printf8.o)
    0x00000e48   0x00000028   Code   RO         3957    i.__0sprintf$8      mc_w.l(printf8.o)
    0x00000e70   0x0000000e   Code   RO         4053    i.__scatterload_copy  mc_w.l(handlers.o)
    0x00000e7e   0x00000002   Code   RO         4054    i.__scatterload_null  mc_w.l(handlers.o)
    0x00000e80   0x0000000e   Code   RO         4055    i.__scatterload_zeroinit  mc_w.l(handlers.o)
    0x00000e8e   0x00000002   PAD
    0x00000e90   0x00000410   Code   RO         3962    i._printf_core      mc_w.l(printf8.o)
    0x000012a0   0x00000024   Code   RO         3963    i._printf_post_padding  mc_w.l(printf8.o)
    0x000012c4   0x0000002e   Code   RO         3964    i._printf_pre_padding  mc_w.l(printf8.o)
    0x000012f2   0x00000016   Code   RO         3965    i._snputc           mc_w.l(printf8.o)
    0x00001308   0x0000000a   Code   RO         3966    i._sputc            mc_w.l(printf8.o)
    0x00001312   0x00000002   PAD
    0x00001314   0x0000006c   Code   RO         2587    i.app_error_fault_handler  app_error_weak.o
    0x00001380   0x00000016   Code   RO         2542    i.app_error_handler_bare  app_error.o
    0x00001396   0x00000002   PAD
    0x00001398   0x00000020   Code   RO          545    i.app_usbd_all_call  app_usbd.o
    0x000013b8   0x00000024   Code   RO          546    i.app_usbd_all_until_served_call  app_usbd.o
    0x000013dc   0x00000028   Code   RO         2978    i.app_usbd_cdc_acm_read  app_usbd_cdc_acm.o
    0x00001404   0x00000016   Code   RO         2979    i.app_usbd_cdc_acm_rx_size  app_usbd_cdc_acm.o
    0x0000141a   0x00000028   Code   RO         2981    i.app_usbd_cdc_acm_write  app_usbd_cdc_acm.o
    0x00001442   0x00000002   PAD
    0x00001444   0x00000090   Code   RO          547    i.app_usbd_class_append  app_usbd.o
    0x000014d4   0x00000044   Code   RO          548    i.app_usbd_class_descriptor_find  app_usbd.o
    0x00001518   0x0000000c   Code   RO          549    i.app_usbd_class_first_get  app_usbd.o
    0x00001524   0x00000012   Code   RO          550    i.app_usbd_class_iface_ep_get  app_usbd.o
    0x00001536   0x00000012   Code   RO         2982    i.app_usbd_class_iface_ep_get  app_usbd_cdc_acm.o
    0x00001548   0x00000014   Code   RO          551    i.app_usbd_class_iface_get  app_usbd.o
    0x0000155c   0x00000014   Code   RO         2983    i.app_usbd_class_iface_get  app_usbd_cdc_acm.o
    0x00001570   0x00000018   Code   RO          555    i.app_usbd_class_sof_register  app_usbd.o
    0x00001588   0x0000002c   Code   RO          556    i.app_usbd_class_sof_unregister  app_usbd.o
    0x000015b4   0x00000018   Code   RO          787    i.app_usbd_core_ep_transfer  app_usbd_core.o
    0x000015cc   0x000000c4   Code   RO          788    i.app_usbd_core_event_handler  app_usbd_core.o
    0x00001690   0x00000010   Code   RO          557    i.app_usbd_core_handler_call  app_usbd.o
    0x000016a0   0x00000024   Code   RO          789    i.app_usbd_core_setup_data_handler_set  app_usbd_core.o
    0x000016c4   0x00000020   Code   RO          790    i.app_usbd_core_setup_data_transfer  app_usbd_core.o
    0x000016e4   0x000000c0   Code   RO          791    i.app_usbd_core_setup_req_handler  app_usbd_core.o
    0x000017a4   0x00000060   Code   RO          792    i.app_usbd_core_setup_rsp  app_usbd_core.o
    0x00001804   0x00000010   Code   RO          793    i.app_usbd_core_setup_transfer_buff_get  app_usbd_core.o
    0x00001814   0x00000014   Code   RO          558    i.app_usbd_disable  app_usbd.o
    0x00001828   0x00000018   Code   RO          559    i.app_usbd_enable   app_usbd.o
    0x00001840   0x0000006c   Code   RO          560    i.app_usbd_endpoint_std_req_handle  app_usbd.o
    0x000018ac   0x0000001c   Code   RO          561    i.app_usbd_ep_call  app_usbd.o
    0x000018c8   0x0000001c   Code   RO          562    i.app_usbd_ep_conf_access  app_usbd.o
    0x000018e4   0x0000000a   Code   RO          564    i.app_usbd_ep_instance_get  app_usbd.o
    0x000018ee   0x00000018   Code   RO          565    i.app_usbd_ep_instance_set  app_usbd.o
    0x00001906   0x00000002   PAD
    0x00001908   0x00000078   Code   RO          566    i.app_usbd_event_handler  app_usbd.o
    0x00001980   0x00000048   Code   RO          567    i.app_usbd_iface_call  app_usbd.o
    0x000019c8   0x00000090   Code   RO          568    i.app_usbd_init     app_usbd.o
    0x00001a58   0x00000022   Code   RO          569    i.app_usbd_interface_std_req_handle  app_usbd.o
    0x00001a7a   0x00000002   PAD
    0x00001a7c   0x00000020   Code   RO          796    i.app_usbd_setup_data_handled_transfer  app_usbd_core.o
    0x00001a9c   0x00000068   Code   RO          571    i.app_usbd_start    app_usbd.o
    0x00001b04   0x00000024   Code   RO          572    i.app_usbd_stop     app_usbd.o
    0x00001b28   0x00000028   Code   RO          960    i.app_usbd_string_desc_get  app_usbd_string_desc.o
    0x00001b50   0x00000004   Code   RO         3106    i.app_util_critical_region_enter  app_util_platform.o
    0x00001b54   0x00000004   Code   RO         3107    i.app_util_critical_region_exit  app_util_platform.o
    0x00001b58   0x00000010   Code   RO         3108    i.app_util_disable_irq  app_util_platform.o
    0x00001b68   0x00000014   Code   RO         3109    i.app_util_enable_irq  app_util_platform.o
    0x00001b7c   0x000000a8   Code   RO         1634    i.apply_config      nrf_drv_uart.o
    0x00001c24   0x00000016   Code   RO         3223    i.assert_nrf_callback  nrf_assert.o
    0x00001c3a   0x00000010   Code   RO         1909    i.bit2ep            nrf_drv_usbd.o
    0x00001c4a   0x00000002   PAD
    0x00001c4c   0x00000028   Code   RO          254    i.bsp_board_button_state_get  boards.o
    0x00001c74   0x00000024   Code   RO          255    i.bsp_board_buttons_init  boards.o
    0x00001c98   0x0000002c   Code   RO          257    i.bsp_board_led_invert  boards.o
    0x00001cc4   0x00000010   Code   RO          258    i.bsp_board_led_off  boards.o
    0x00001cd4   0x00000010   Code   RO          259    i.bsp_board_led_on  boards.o
    0x00001ce4   0x0000002c   Code   RO          261    i.bsp_board_leds_init  boards.o
    0x00001d10   0x00000012   Code   RO          262    i.bsp_board_leds_off  boards.o
    0x00001d22   0x00000012   Code   RO         3283    i.buf_len_update    nrf_log_backend_serial.o
    0x00001d34   0x00000060   Code   RO         3378    i.buf_prealloc      nrf_log_frontend.o
    0x00001d94   0x00000014   Code   RO         3379    i.buffer_is_empty   nrf_log_frontend.o
    0x00001da8   0x00000076   Code   RO         2984    i.cdc_acm_event_handler  app_usbd_cdc_acm.o
    0x00001e1e   0x00000008   Code   RO         2985    i.cdc_acm_get_descriptors  app_usbd_cdc_acm.o
    0x00001e26   0x00000026   Code   RO         2986    i.cdc_acm_req_out_data_cb  app_usbd_cdc_acm.o
    0x00001e4c   0x00000098   Code   RO            4    i.cdc_acm_user_ev_handler  main.o
    0x00001ee4   0x00000010   Code   RO         1218    i.channel_port_get  nrf_drv_gpiote.o
    0x00001ef4   0x00000006   Code   RO          574    i.class_event_handler  app_usbd.o
    0x00001efa   0x00000002   PAD
    0x00001efc   0x00000028   Code   RO         1012    i.clock_clk_started_notify  nrf_drv_clock.o
    0x00001f24   0x00000012   Code   RO         2987    i.comm_ep_in_addr_get  app_usbd_cdc_acm.o
    0x00001f36   0x00000002   PAD
    0x00001f38   0x000000ac   Code   RO         2754    i.compare_reg_update  app_timer.o
    0x00001fe4   0x00000012   Code   RO         2988    i.data_ep_in_addr_get  app_usbd_cdc_acm.o
    0x00001ff6   0x00000012   Code   RO         2989    i.data_ep_out_addr_get  app_usbd_cdc_acm.o
    0x00002008   0x00000040   Code   RO         2755    i.elapsed_ticks_acquire  app_timer.o
    0x00002048   0x0000000c   Code   RO         1910    i.ep2bit            nrf_drv_usbd.o
    0x00002054   0x00000018   Code   RO         1911    i.ep_state_access   nrf_drv_usbd.o
    0x0000206c   0x00000078   Code   RO         1635    i.interrupts_enable  nrf_drv_uart.o
    0x000020e4   0x00000016   Code   RO         1014    i.item_enqueue      nrf_drv_clock.o
    0x000020fa   0x00000002   PAD
    0x000020fc   0x000000f8   Code   RO         2756    i.list_insertions_handler  app_timer.o
    0x000021f4   0x00000184   Code   RO            5    i.main              main.o
    0x00002378   0x0000000c   Code   RO         1912    i.nrf_atomic_u32_and  nrf_drv_usbd.o
    0x00002384   0x00000010   Code   RO         1219    i.nrf_bitmask_bit_is_set  nrf_drv_gpiote.o
    0x00002394   0x0000000e   Code   RO         1016    i.nrf_clock_event_check  nrf_drv_clock.o
    0x000023a2   0x00000010   Code   RO         1017    i.nrf_clock_event_clear  nrf_drv_clock.o
    0x000023b2   0x00000002   PAD
    0x000023b4   0x0000001c   Code   RO         1018    i.nrf_clock_hf_is_running  nrf_drv_clock.o
    0x000023d0   0x0000008c   Code   RO            6    i.nrf_delay_us      main.o
    0x0000245c   0x0000008c   Code   RO         2757    i.nrf_delay_us      app_timer.o
    0x000024e8   0x00000006   Code   RO         1021    i.nrf_drv_clock_hfclk_is_running  nrf_drv_clock.o
    0x000024ee   0x00000002   PAD
    0x000024f0   0x00000058   Code   RO         1023    i.nrf_drv_clock_hfclk_request  nrf_drv_clock.o
    0x00002548   0x00000044   Code   RO         1024    i.nrf_drv_clock_init  nrf_drv_clock.o
    0x0000258c   0x00000058   Code   RO         1030    i.nrf_drv_clock_onIRQ  nrf_drv_clock.o
    0x000025e4   0x00000016   Code   RO         1636    i.nrf_drv_common_irq_disable  nrf_drv_uart.o
    0x000025fa   0x00000038   Code   RO         1164    i.nrf_drv_common_irq_enable  nrf_drv_common.o
    0x00002632   0x00000006   Code   RO         1637    i.nrf_drv_get_IRQn  nrf_drv_uart.o
    0x00002638   0x00000010   Code   RO         1638    i.nrf_drv_is_in_RAM  nrf_drv_uart.o
    0x00002648   0x00000050   Code   RO         1478    i.nrf_drv_power_init  nrf_drv_power.o
    0x00002698   0x00000090   Code   RO         1480    i.nrf_drv_power_onIRQ  nrf_drv_power.o
    0x00002728   0x00000024   Code   RO         1486    i.nrf_drv_power_usbevt_init  nrf_drv_power.o
    0x0000274c   0x00000018   Code   RO         1487    i.nrf_drv_power_usbevt_uninit  nrf_drv_power.o
    0x00002764   0x00000014   Code   RO         1569    i.nrf_drv_systick_delay_ticks  nrf_drv_systick.o
    0x00002778   0x0000001c   Code   RO         1570    i.nrf_drv_systick_delay_us  nrf_drv_systick.o
    0x00002794   0x00000010   Code   RO         1572    i.nrf_drv_systick_init  nrf_drv_systick.o
    0x000027a4   0x00000068   Code   RO         1640    i.nrf_drv_uart_init  nrf_drv_uart.o
    0x0000280c   0x0000010c   Code   RO         1648    i.nrf_drv_uart_tx   nrf_drv_uart.o
    0x00002918   0x00000018   Code   RO         1650    i.nrf_drv_uart_tx_in_progress  nrf_drv_uart.o
    0x00002930   0x00000054   Code   RO         1651    i.nrf_drv_uart_uninit  nrf_drv_uart.o
    0x00002984   0x00000030   Code   RO         1913    i.nrf_drv_usbd_consumer  nrf_drv_usbd.o
    0x000029b4   0x00000034   Code   RO         1914    i.nrf_drv_usbd_disable  nrf_drv_usbd.o
    0x000029e8   0x00000054   Code   RO         1915    i.nrf_drv_usbd_enable  nrf_drv_usbd.o
    0x00002a3c   0x0000008c   Code   RO         1917    i.nrf_drv_usbd_ep_enable  nrf_drv_usbd.o
    0x00002ac8   0x00000078   Code   RO         1919    i.nrf_drv_usbd_ep_handled_transfer  nrf_drv_usbd.o
    0x00002b40   0x0000000a   Code   RO         1921    i.nrf_drv_usbd_ep_max_packet_size_get  nrf_drv_usbd.o
    0x00002b4a   0x0000000c   Code   RO         1922    i.nrf_drv_usbd_ep_max_packet_size_set  nrf_drv_usbd.o
    0x00002b56   0x00000002   PAD
    0x00002b58   0x00000018   Code   RO         1923    i.nrf_drv_usbd_ep_stall  nrf_drv_usbd.o
    0x00002b70   0x00000004   Code   RO         1924    i.nrf_drv_usbd_ep_stall_check  nrf_drv_usbd.o
    0x00002b74   0x00000014   Code   RO         1925    i.nrf_drv_usbd_ep_stall_clear  nrf_drv_usbd.o
    0x00002b88   0x00000028   Code   RO         1926    i.nrf_drv_usbd_ep_status_get  nrf_drv_usbd.o
    0x00002bb0   0x0000001c   Code   RO         1927    i.nrf_drv_usbd_ep_to_int  nrf_drv_usbd.o
    0x00002bcc   0x000000d4   Code   RO         1928    i.nrf_drv_usbd_ep_transfer  nrf_drv_usbd.o
    0x00002ca0   0x00000024   Code   RO         1929    i.nrf_drv_usbd_epout_size_get  nrf_drv_usbd.o
    0x00002cc4   0x00000008   Code   RO         1930    i.nrf_drv_usbd_feeder_buffer_get  nrf_drv_usbd.o
    0x00002ccc   0x0000003c   Code   RO         1931    i.nrf_drv_usbd_feeder_flash  nrf_drv_usbd.o
    0x00002d08   0x00000044   Code   RO         1932    i.nrf_drv_usbd_feeder_flash_zlp  nrf_drv_usbd.o
    0x00002d4c   0x00000024   Code   RO         1933    i.nrf_drv_usbd_feeder_ram  nrf_drv_usbd.o
    0x00002d70   0x00000036   Code   RO         1934    i.nrf_drv_usbd_feeder_ram_zlp  nrf_drv_usbd.o
    0x00002da6   0x00000002   PAD
    0x00002da8   0x00000098   Code   RO         1935    i.nrf_drv_usbd_init  nrf_drv_usbd.o
    0x00002e40   0x00000014   Code   RO         1936    i.nrf_drv_usbd_is_enabled  nrf_drv_usbd.o
    0x00002e54   0x00000020   Code   RO         1938    i.nrf_drv_usbd_is_started  nrf_drv_usbd.o
    0x00002e74   0x0000000c   Code   RO         1939    i.nrf_drv_usbd_last_setup_dir_get  nrf_drv_usbd.o
    0x00002e80   0x00000006   Code   RO         1940    i.nrf_drv_usbd_setup_clear  nrf_drv_usbd.o
    0x00002e86   0x0000001a   Code   RO         1941    i.nrf_drv_usbd_setup_data_clear  nrf_drv_usbd.o
    0x00002ea0   0x00000050   Code   RO         1942    i.nrf_drv_usbd_setup_get  nrf_drv_usbd.o
    0x00002ef0   0x00000006   Code   RO         1943    i.nrf_drv_usbd_setup_stall  nrf_drv_usbd.o
    0x00002ef6   0x00000002   PAD
    0x00002ef8   0x00000030   Code   RO         1944    i.nrf_drv_usbd_start  nrf_drv_usbd.o
    0x00002f28   0x00000028   Code   RO         1945    i.nrf_drv_usbd_stop  nrf_drv_usbd.o
    0x00002f50   0x00000034   Code   RO         1946    i.nrf_drv_usbd_transfer_out_drop  nrf_drv_usbd.o
    0x00002f84   0x00000032   Code   RO          266    i.nrf_gpio_cfg      boards.o
    0x00002fb6   0x00000032   Code   RO         1652    i.nrf_gpio_cfg      nrf_drv_uart.o
    0x00002fe8   0x00000012   Code   RO         1653    i.nrf_gpio_cfg_default  nrf_drv_uart.o
    0x00002ffa   0x00000012   Code   RO         1654    i.nrf_gpio_cfg_input  nrf_drv_uart.o
    0x0000300c   0x00000014   Code   RO         1655    i.nrf_gpio_cfg_output  nrf_drv_uart.o
    0x00003020   0x00000030   Code   RO         1245    i.nrf_gpio_cfg_sense_set  nrf_drv_gpiote.o
    0x00003050   0x0000001c   Code   RO          267    i.nrf_gpio_pin_port_decode  boards.o
    0x0000306c   0x0000001c   Code   RO         1247    i.nrf_gpio_pin_port_decode  nrf_drv_gpiote.o
    0x00003088   0x0000001c   Code   RO         1656    i.nrf_gpio_pin_port_decode  nrf_drv_uart.o
    0x000030a4   0x00000014   Code   RO         1657    i.nrf_gpio_pin_set  nrf_drv_uart.o
    0x000030b8   0x00000026   Code   RO          268    i.nrf_gpio_pin_write  boards.o
    0x000030de   0x00000002   PAD
    0x000030e0   0x0000002c   Code   RO         1250    i.nrf_gpio_ports_read  nrf_drv_gpiote.o
    0x0000310c   0x00000014   Code   RO         1251    i.nrf_gpiote_event_clear  nrf_drv_gpiote.o
    0x00003120   0x00000010   Code   RO         1252    i.nrf_gpiote_event_is_set  nrf_drv_gpiote.o
    0x00003130   0x00000008   Code   RO         3285    i.nrf_log_backend_hexdump_handler_get  nrf_log_backend_serial.o
    0x00003138   0x00000070   Code   RO         3286    i.nrf_log_backend_init  nrf_log_backend_serial.o
    0x000031a8   0x0000012e   Code   RO         3287    i.nrf_log_backend_serial_hexdump_handler  nrf_log_backend_serial.o
    0x000032d6   0x00000114   Code   RO         3288    i.nrf_log_backend_serial_std_handler  nrf_log_backend_serial.o
    0x000033ea   0x00000002   PAD
    0x000033ec   0x00000008   Code   RO         3289    i.nrf_log_backend_std_handler_get  nrf_log_backend_serial.o
    0x000033f4   0x00000006   Code   RO         3381    i.nrf_log_blocking_backend_set  nrf_log_frontend.o
    0x000033fa   0x00000002   PAD
    0x000033fc   0x00000130   Code   RO         3382    i.nrf_log_frontend_dequeue  nrf_log_frontend.o
    0x0000352c   0x00000014   Code   RO         3384    i.nrf_log_frontend_init  nrf_log_frontend.o
    0x00003540   0x0000004c   Code   RO         3385    i.nrf_log_frontend_std_0  nrf_log_frontend.o
    0x0000358c   0x00000058   Code   RO         3386    i.nrf_log_frontend_std_1  nrf_log_frontend.o
    0x000035e4   0x00000068   Code   RO         3387    i.nrf_log_frontend_std_2  nrf_log_frontend.o
    0x0000364c   0x00000010   Code   RO         3393    i.nrf_log_handlers_set  nrf_log_frontend.o
    0x0000365c   0x00000024   Code   RO         3394    i.nrf_log_init      nrf_log_frontend.o
    0x00003680   0x00000014   Code   RO         1488    i.nrf_power_event_get_and_clear  nrf_drv_power.o
    0x00003694   0x0000000a   Code   RO         1658    i.nrf_uart_event_check  nrf_drv_uart.o
    0x0000369e   0x0000000c   Code   RO         1659    i.nrf_uart_event_clear  nrf_drv_uart.o
    0x000036aa   0x0000000c   Code   RO         1660    i.nrf_uart_int_enable_check  nrf_drv_uart.o
    0x000036b6   0x0000000a   Code   RO         1661    i.nrf_uarte_event_check  nrf_drv_uart.o
    0x000036c0   0x0000000c   Code   RO         1662    i.nrf_uarte_event_clear  nrf_drv_uart.o
    0x000036cc   0x00000018   Code   RO          575    i.nrf_usbd_dtoggle_get  app_usbd.o
    0x000036e4   0x00000018   Code   RO          576    i.nrf_usbd_dtoggle_set  app_usbd.o
    0x000036fc   0x00000018   Code   RO          797    i.nrf_usbd_dtoggle_set  app_usbd_core.o
    0x00003714   0x0000002c   Code   RO         1948    i.nrf_usbd_ep_is_stall  nrf_drv_usbd.o
    0x00003740   0x0000003c   Code   RO         1949    i.nrf_usbd_epin_dma_handler  nrf_drv_usbd.o
    0x0000377c   0x00000068   Code   RO         1950    i.nrf_usbd_epout_dma_handler  nrf_drv_usbd.o
    0x000037e4   0x00000010   Code   RO         1951    i.nrf_usbd_event_check  nrf_drv_usbd.o
    0x000037f4   0x00000018   Code   RO         1952    i.nrf_usbd_event_clear  nrf_drv_usbd.o
    0x0000380c   0x00000014   Code   RO         1953    i.nrf_usbd_eventcause_clear  nrf_drv_usbd.o
    0x00003820   0x00000018   Code   RO          798    i.nrf_usbd_task_trigger  app_usbd_core.o
    0x00003838   0x00000018   Code   RO         1954    i.nrf_usbd_task_trigger  nrf_drv_usbd.o
    0x00003850   0x00000078   Code   RO         1663    i.pins_to_default   nrf_drv_uart.o
    0x000038c8   0x000000bc   Code   RO            7    i.power_usb_event_handler  main.o
    0x00003984   0x0000006c   Code   RO            8    i.requestTx         main.o
    0x000039f0   0x0000003c   Code   RO         2758    i.rtc1_stop         app_timer.o
    0x00003a2c   0x00000032   Code   RO         1664    i.rx_byte           nrf_drv_uart.o
    0x00003a5e   0x00000018   Code   RO         1665    i.rx_done_event     nrf_drv_uart.o
    0x00003a76   0x00000002   PAD
    0x00003a78   0x0000000c   Code   RO         3290    i.serial_is_busy    nrf_log_backend_serial.o
    0x00003a84   0x0000002c   Code   RO         3291    i.serial_tx         nrf_log_backend_serial.o
    0x00003ab0   0x00000004   Code   RO          799    i.setup_data_handler_empty  app_usbd_core.o
    0x00003ab4   0x0000008c   Code   RO         2990    i.setup_event_handler  app_usbd_cdc_acm.o
    0x00003b40   0x000000ac   Code   RO         2991    i.setup_req_class_out  app_usbd_cdc_acm.o
    0x00003bec   0x000000e0   Code   RO          800    i.setup_req_get_descriptor  app_usbd_core.o
    0x00003ccc   0x00000074   Code   RO          801    i.setup_req_std_in  app_usbd_core.o
    0x00003d40   0x00000064   Code   RO          802    i.setup_req_std_out  app_usbd_core.o
    0x00003da4   0x000000cc   Code   RO          803    i.setup_req_std_set_configuration  app_usbd_core.o
    0x00003e70   0x00000080   Code   RO         2759    i.timer_list_handler  app_timer.o
    0x00003ef0   0x0000003c   Code   RO         2760    i.timer_list_insert  app_timer.o
    0x00003f2c   0x00000060   Code   RO         2761    i.timer_list_remove  app_timer.o
    0x00003f8c   0x00000074   Code   RO         2763    i.timer_timeouts_check  app_timer.o
    0x00004000   0x00000034   Code   RO         3292    i.timestamp_process  nrf_log_backend_serial.o
    0x00004034   0x00000020   Code   RO         1667    i.tx_byte           nrf_drv_uart.o
    0x00004054   0x0000001c   Code   RO         1668    i.tx_done_event     nrf_drv_uart.o
    0x00004070   0x00000010   Code   RO         3293    i.uart_event_handler  nrf_log_backend_serial.o
    0x00004080   0x0000011e   Code   RO         1669    i.uart_irq_handler  nrf_drv_uart.o
    0x0000419e   0x000000f0   Code   RO         1670    i.uarte_irq_handler  nrf_drv_uart.o
    0x0000428e   0x00000002   PAD
    0x00004290   0x00000010   Code   RO          804    i.usb_core_ep0_handler_check  app_usbd_core.o
    0x000042a0   0x000000b6   Code   RO          805    i.usbd_descriptor_conf_feeder  app_usbd_core.o
    0x00004356   0x00000002   PAD
    0x00004358   0x00000188   Code   RO         1955    i.usbd_dmareq_process  nrf_drv_usbd.o
    0x000044e0   0x00000004   Code   RO         1956    i.usbd_drv_ep_abort  nrf_drv_usbd.o
    0x000044e4   0x000000c4   Code   RO         1957    i.usbd_ep_abort     nrf_drv_usbd.o
    0x000045a8   0x00000040   Code   RO         1958    i.usbd_ep_abort_all  nrf_drv_usbd.o
    0x000045e8   0x00000040   Code   RO         1959    i.usbd_ep_data_handler  nrf_drv_usbd.o
    0x00004628   0x00000010   Code   RO         1960    i.usbd_int_rise     nrf_drv_usbd.o
    0x00004638   0x00000022   Code   RO            9    i.usbd_user_ev_handler  main.o
    0x0000465a   0x00000002   PAD
    0x0000465c   0x00000010   Code   RO          577    i.user_event_handler  app_usbd.o
    0x0000466c   0x0000000a   Code   RO         2992    i.user_event_handler  app_usbd_cdc_acm.o
    0x00004676   0x00000042   Data   RO           12    .constdata          main.o
    0x000046b8   0x00000028   Data   RO           13    .constdata          main.o
    0x000046e0   0x00000008   Data   RO          269    .constdata          boards.o
    0x000046e8   0x00000018   Data   RO          579    .constdata          app_usbd.o
    0x00004700   0x0000002b   Data   RO          807    .constdata          app_usbd_core.o
    0x0000472b   0x00000001   PAD
    0x0000472c   0x00000008   Data   RO          808    .constdata          app_usbd_core.o
    0x00004734   0x00000010   Data   RO          809    .constdata          app_usbd_core.o
    0x00004744   0x00000004   Data   RO          961    .constdata          app_usbd_string_desc.o
    0x00004748   0x0000002a   Data   RO          962    .constdata          app_usbd_string_desc.o
    0x00004772   0x00000026   Data   RO          963    .constdata          app_usbd_string_desc.o
    0x00004798   0x0000000e   Data   RO          964    .constdata          app_usbd_string_desc.o
    0x000047a6   0x00000005   Data   RO          966    .constdata          app_usbd_string_desc.o
    0x000047ab   0x00000001   PAD
    0x000047ac   0x00000008   Data   RO         1256    .constdata          nrf_drv_gpiote.o
    0x000047b4   0x00000001   Data   RO         1489    .constdata          nrf_drv_power.o
    0x000047b5   0x00000003   PAD
    0x000047b8   0x000000ce   Data   RO         1962    .constdata          nrf_drv_usbd.o
    0x00004886   0x00000002   PAD
    0x00004888   0x00000008   Data   RO         2993    .constdata          app_usbd_cdc_acm.o
    0x00004890   0x00000014   Data   RO         2994    .constdata          app_usbd_cdc_acm.o
    0x000048a4   0x00000020   Data   RO         3296    .constdata          nrf_log_backend_serial.o
    0x000048c4   0x00000024   Data   RO         3397    .constdata          nrf_log_frontend.o
    0x000048e8   0x00000081   Data   RO         3711    .constdata          mc_w.l(ctype_o.o)
    0x00004969   0x00000003   PAD
    0x0000496c   0x00000004   Data   RO         3712    .constdata          mc_w.l(ctype_o.o)
    0x00004970   0x0000000b   Data   RO         3398    .conststring        nrf_log_frontend.o
    0x0000497b   0x00000001   PAD
    0x0000497c   0x00000020   Data   RO         4051    Region$$Table       anon$$obj.o


    Execution Region RW_IRAM1 (Base: 0x20000000, Size: 0x000032b8, Max: 0x00040000, ABSOLUTE)

    Base Addr    Size         Type   Attr      Idx    E Section Name        Object

    0x20000000   0x00000014   Data   RW           14    .data               main.o
    0x20000014   0x0000000c   Data   RW          580    .data               app_usbd.o
    0x20000020   0x00000010   Data   RW          810    .data               app_usbd_core.o
    0x20000030   0x00000008   Data   RW          811    .data               app_usbd_core.o
    0x20000038   0x00000014   Data   RW          967    .data               app_usbd_string_desc.o
    0x2000004c   0x00000010   Data   RW         1490    .data               nrf_drv_power.o
    0x2000005c   0x00000014   Data   RW         1963    .data               nrf_drv_usbd.o
    0x20000070   0x00000014   Data   RW         2766    .data               app_timer.o
    0x20000084   0x00000004   Data   RW         3112    .data               app_util_platform.o
    0x20000088   0x0000000c   Data   RW         3297    .data               nrf_log_backend_serial.o
    0x20000094   0x00000004   Data   RW         3399    .data               nrf_log_frontend.o
    0x20000098   0x00000004   Data   RW         3674    .data               system_nrf52840.o
    0x2000009c   0x00000020   Zero   RW           10    .bss                main.o
    0x200000bc   0x00000822   Zero   RW           11    .bss                main.o
    0x200008de   0x00000002   PAD
    0x200008e0   0x00000090   Zero   RW          578    .bss                app_usbd.o
    0x20000970   0x00000050   Zero   RW          806    .bss                app_usbd_core.o
    0x200009c0   0x00000014   Zero   RW         1032    .bss                nrf_drv_clock.o
    0x200009d4   0x00000068   Zero   RW         1255    .bss                nrf_drv_gpiote.o
    0x20000a3c   0x00000020   Zero   RW         1671    .bss                nrf_drv_uart.o
    0x20000a5c   0x00000238   Zero   RW         1961    .bss                nrf_drv_usbd.o
    0x20000c94   0x0000010c   Zero   RW         2765    .bss                app_timer.o
    0x20000da0   0x00000100   Zero   RW         3294    .bss                nrf_log_backend_serial.o
    0x20000ea0   0x00000418   Zero   RW         3396    .bss                nrf_log_frontend.o
    0x200012b8   0x00002000   Zero   RW         3662    STACK               arm_startup_nrf52840.o


==============================================================================

Image component sizes


      Code (inc. data)   RO Data    RW Data    ZI Data      Debug   Object Name

        22          0          0          0          0       2137   app_error.o
       108         54          0          0          0      27357   app_error_weak.o
      1190         80          0         20        268      40304   app_timer.o
         0          0          0          0          0       5752   app_uart_fifo.o
      1236        118         24         12        144      44203   app_usbd.o
       680         14         28          0          0      30670   app_usbd_cdc_acm.o
      1672        106         67         24         80      45779   app_usbd_core.o
        40         10        103         20          0       3404   app_usbd_string_desc.o
        44         10          0          4          0       3228   app_util_platform.o
        36          8        512          0       8192        916   arm_startup_nrf52840.o
       330         36          8          0          0      11031   boards.o
         0          0          0          0          0       1340   bsp.o
        52         14          0          0          0        600   hardfault_handler_keil.o
       104         48          0          0          0       2746   hardfault_implementation.o
      1010        356        106         20       2114      89569   main.o
        22          0          0          0          0       2598   nrf_assert.o
       370         30          0          0         20      13526   nrf_drv_clock.o
        70          0          0          0          0      28100   nrf_drv_common.o
       640         34          8          0        104      18952   nrf_drv_gpiote.o
       304         26          1         16          0      14688   nrf_drv_power.o
        64         10          0          0          0       5020   nrf_drv_systick.o
      1830         68          0          0         32      65543   nrf_drv_uart.o
      3970        384        206         20        568     105106   nrf_drv_usbd.o
       848         56         32         12        256       9915   nrf_log_backend_serial.o
       766         56         47          4       1048      11077   nrf_log_frontend.o
       488         56          0          4          0       2351   system_nrf52840.o

    ----------------------------------------------------------------------
     15946       1574       1182        156      12828     585912   Object Totals
         0          0         32          0          0          0   (incl. Generated)
        50          0          8          0          2          0   (incl. Padding)

    ----------------------------------------------------------------------

      Code (inc. data)   RO Data    RW Data    ZI Data      Debug   Library Member Name

         8          4        133          0          0         68   ctype_o.o
         0          0          0          0          0          0   entry.o
         0          0          0          0          0          0   entry10a.o
         0          0          0          0          0          0   entry11a.o
         8          4          0          0          0          0   entry2.o
         4          0          0          0          0          0   entry5.o
         0          0          0          0          0          0   entry7b.o
         0          0          0          0          0          0   entry8b.o
         8          4          0          0          0          0   entry9a.o
        30          0          0          0          0          0   handlers.o
        36          8          0          0          0         68   init.o
        30          0          0          0          0         68   llshl.o
        32          0          0          0          0         68   llushr.o
        36          0          0          0          0         68   memcpya.o
        36          0          0          0          0        108   memseta.o
      1234         54          0          0          0        572   printf8.o
        14          0          0          0          0         68   strlen.o
        98          0          0          0          0         92   uldiv.o

    ----------------------------------------------------------------------
      1580         74        136          0          0       1180   Library Totals
         6          0          3          0          0          0   (incl. Padding)

    ----------------------------------------------------------------------

      Code (inc. data)   RO Data    RW Data    ZI Data      Debug   Library Name

      1574         74        133          0          0       1180   mc_w.l

    ----------------------------------------------------------------------
      1580         74        136          0          0       1180   Library Totals

    ----------------------------------------------------------------------

==============================================================================


      Code (inc. data)   RO Data    RW Data    ZI Data      Debug   

     17526       1648       1318        156      12828     562576   Grand Totals
     17526       1648       1318        156      12828     562576   ELF Image Totals
     17526       1648       1318        156          0          0   ROM Totals

==============================================================================

    Total RO  Size (Code + RO Data)                18844 (  18.40kB)
    Total RW  Size (RW Data + ZI Data)             12984 (  12.68kB)
    Total ROM Size (Code + RO Data + RW Data)      19000 (  18.55kB)

==============================================================================

